:020000040800F2
:1000000000040020E1010008090E00080D0E0008A0
:10001000610E00080D0E0008350E0008E30100080F
:10002000E3010008E3010008E3010008352F0008A0
:10003000E3010008E3010008E3010008E301000810
:10004000E3010008E3010008E3010008E301000800
:10005000E3010008E301000895310008C131000800
:10006000ED3100081932000845320008E3010008AC
:10007000E3010008E3010008E3010008E3010008D0
:10008000E3010008E3010008E3010008E3010008C0
:10009000E3010008E3010008E301000871320008F1
:1000A000E3010008E3010008E3010008E3010008A0
:1000B000B12F0008E3010008E3010008E301000894
:1000C000E3010008E3010008E3010008E301000880
:1000D000E3010008E3010008E3010008E301000870
:1000E000D9320008E3010008E3010008E301000839
:1000F000E3010008E3010008E3010008E301000850
:10010000E3010008E3010008E3010008E30100083F
:10011000E3010008E3010008E3010008E30100082F
:10012000E3010008E3010008E3010008E30100081F
:10013000E3010008E3010008E3010008E30100080F
:10014000E3010008E3010008E30100088926000834
:10015000E3010008E3010008E3010008E3010008EF
:10016000E3010008E3010008E3010008E3010008DF
:10017000E3010008E3010008E3010008E3010008CF
:10018000E3010008E3010008E3010008E3010008BF
:10019000E3010008E3010008E3010008E3010008AF
:1001A000E3010008E3010008E3010008E30100089F
:1001B000E3010008E3010008E3010008E30100088F
:1001C000E3010008E3010008E3010008E30100087F
:1001D000E3010008E3010008E3010008E30100086F
:1001E00002E000F000F8FEE772B6394880F30888B4
:1001F000384880F3098838484EF60851CEF200019D
:10020000086040F20000CCF200004EF63471CEF2ED
:1002100000010860BFF34F8FBFF36F8F40F2000003
:10022000C0F2F0004EF68851CEF200010860BFF334
:100230004F8FBFF36F8F4FF00000E1EE100A4EF6C4
:100240003C71CEF200010860062080F31488BFF3F1
:100250006F8F01F0E1FE02F003FE4FF055301F49B1
:100260001B4A91423CBF41F8040BFAE71C49194A6A
:1002700091423CBF41F8040BFAE71A491A4A1B4B5A
:100280009A423EBF51F8040B42F8040BF8E70020F5
:100290001749184A91423CBF41F8040BFAE701F0B4
:1002A000BFFE02F039FE144C144DAC4203DA54F890
:1002B000041B8847F9E700F03FF8114C114DAC42A0
:1002C00003DA54F8041B8847F9E701F0A7BE0000E1
:1002D000000400200024002000000008000000208E
:1002E00000040020F036000800240020282400200C
:1002F0002824002018300020E0010008E001000858
:10030000E0010008E00100082DE9F04F2DED108A12
:10031000C1F80CD0C3689D46BDEC108ABDE8F08FD3
:10032000002383F311882846A047002001F0FAFA41
:1003300001F0AAFA00DFFEE71A4B6FF07C0270B5FD
:1003400000241A700F225C709C70DC701C715C7150
:100350009C71DC711C725C729A72DC7201F02EFE70
:10036000064601F053FE054650B90F4B9E4217D08A
:1003700001339E4241F2883412BF05460024012514
:10038000002001F025FE0DB100F0B4F800F010FDE2
:1003900000F0F4FB204600F00BF900F0ABF8F9E7B1
:1003A0000446EDE728240020010007B008B500F05E
:1003B00087FBA0F120035842584108BD07B5054B03
:1003C00002211B88ADF8043001A800F0C7FB03B080
:1003D0005DF804FBBC330008064991F8243033B1C2
:1003E00000230822086A81F8243000F0E9BB0120CC
:1003F000704700BF482400202DE9F84F234C94F8A3
:1004000024300546884617468BBB2E46DFF87C9085
:10041000002F38D094F824A0BAF1000F05D1202283
:10042000FF214846266200F0B1FCCAF10805BD4232
:1004300028BF3D465FFA85FBAD0041462A4604EBE6
:100440008A0000F079FC94F82430A7EB0B079B445A
:100450005FFA8BFBBBF1080F2E44A844FFB284F86F
:1004600024B0D5D1FFF7B8FF0028D1D108E0266A23
:1004700006EB8306B042C9D0FFF7AEFF0028C4D117
:100480000020BDE8F88F0120BDE8F88F4824002047
:1004900010B5202383F311881248C3680BB101F013
:1004A000C7FA0023104A0F484FF47A7101F084FA1A
:1004B000002383F311880D4C236813B12368013B9B
:1004C0002360636813B16368013B6360084B1B786A
:1004D00033B9636823B9022000F024FC322363603F
:1004E00010BD00BF342400209104000878250020AE
:1004F0007024002010B5254B254953F8042F0132F4
:1005000000D110BD8B42F8D1224C234B22689A4275
:100510003AD9224B9B6803F1006303F580339A427A
:1005200032D2002000F044FB1D4B0220187000F076
:10053000F1FB1C4B1A6C00221A64196E1A66196EB4
:10054000596C5A64596E5A665A6E5A6942F0800262
:100550005A615A6922F080025A615A691A6942F056
:1005600000521A611A6922F000521A611B6972B6B0
:100570000D4A0E4B13601B682268202181F31188FD
:100580009D4683F30888104710BD00BFFCFF00089C
:100590001C00010804000108FFFF000828240020B7
:1005A000702400200038024008ED00E0000001083F
:1005B0002DE9F04F99B0B34C01902022FF2110A8F3
:1005C000A66800F0E3FBB04A1378A346A3B9AF488E
:1005D0000121C3601170202383F31188C3680BB11C
:1005E00001F026FA0023AA4AA8484FF47A7101F0D4
:1005F000E3F9002383F31188019B13B1A54B019A02
:100600001A60A54AA349019F0292002313704B6010
:1006100099461C461D469846012000F07BFB002FA2
:1006200000F012829B4B1B68002B40F00D8219B02A
:10063000BDE8F08F0220FFF7B9FE002840F0FB81F3
:10064000019BB9F1000F08BF1F46944B1B88ADF802
:100650002C3002210BA800F081FADDE74FF47A700C
:1006600000F02EFA031E0393EADB0220FFF79EFE42
:1006700082460028E4D0039B581E042800F2DD8146
:10068000DFE800F0030E1114170018A8052340F846
:10069000343D042100F062FA54464FF0000856E061
:1006A00004217848F6E704217D48F3E704217D48DA
:1006B000F0E71C24204600F07DFA04340B9004215E
:1006C0000BA800F04BFA2C2CF4D1E5E7002DB7D0A5
:1006D000002CB5D00220FFF769FE0546002800F087
:1006E000AF8101206C4C00F063FA0220207000F012
:1006F00011FB4FF000095FFA89FA504600F068FAE2
:10070000074658B1504600F073FA09F10109002874
:10071000F1D12C46A9460027634B97E7012302201D
:10072000237000F0EDFA3E46DBF808309E4206D218
:10073000304600F03FFA0130EBD10436F4E7029B7B
:1007400000261E70534BA9465E602C46374600F0CB
:1007500025FB15B1002C18BF0027FFF72FFE5BE724
:10076000002D3FF46DAF002C3FF46AAF029B0220D6
:10077000187000F0CFFA322000F0A2F9B0F1000AB0
:10078000C0F25E811AF0030540F05A81DBF80820C0
:1007900006EB0A03934200F25381BAF5807F00F220
:1007A0004F8155450DDA4FF47A7000F089F90490C5
:1007B000049B002BC0F244813C4A049BAB5401359E
:1007C000EFE7C820FFF7F2FD0546002800F038816A
:1007D0001F2E11D8C6F12004544528BF544610AB33
:1007E00026F0030022463149184400F0A5FA2246BB
:1007F000FF212E4800F0CAFA4FEAAA0A5FFA8AF2ED
:100800002A493046FFF7F8FD0446002800F01A8117
:1008100006EB8A0605469AE70220FFF7C7FD002887
:100820003FF40EAFFFF7D8FD00283FF409AF4FF0BB
:10083000000A5346DBF8082092451CD2BAF11F0F7C
:1008400012D8109A01320FD02AF0030218A90A44D4
:1008500052F8202C0B92184604220BA900F014FB2E
:100860000AF1040A0346E5E75046039300F0A2F9B3
:10087000039B0B90EFE718A8042140F84C3D00F0D3
:100880006DF964E72824002074250020342400201A
:10089000910400087825002070240020BE33000851
:1008A0002C24002030240020C033000874240020B1
:1008B00018A8002340F8343D642100F02BF90028EB
:1008C0007FF4BEAE0220FFF771FD00283FF4B8AE02
:1008D0000B9800F09FF918AB43F8480D0421184617
:1008E000CDE718A8002340F8343D642100F012F948
:1008F00000287FF4A5AE0220FFF758FD00283FF442
:100900009FAE0B9800F094F918AB43F8440DE5E75F
:100910000220FFF74BFD00283FF492AE00F08EF965
:1009200018AB43F8400DD9E70220FFF73FFD002840
:100930003FF486AE0BA9142000F086F9824618A871
:10094000042140F83CAD00F009F951460BA896E7A8
:10095000322000F0B5F8B0F1000AFFF671AE1AF0DF
:10096000030F7FF46DAEDBF808200AEB0803934217
:100970003FF666AE0220FFF719FD00283FF460AE97
:100980002AF0030AC244D0453FF4E1AE404600F0ED
:1009900011F904210A900AA800F0E0F808F104080F
:1009A000F1E74FF47A70FFF701FD00283FF448AEFD
:1009B000FFF712FD00283FF4AFAE109B01330CD0BF
:1009C000082210A90020FFF717FD00283FF4A4AE6D
:1009D0002022FF2110A800F0D9F9FFF7EFFC3748DB
:1009E00000F0A6FF23E6002D3FF42AAE002C3FF4D2
:1009F00027AE18A8002340F8343D642100F08AF89F
:100A0000824600287FF41CAE0220FFF7CFFC0028AE
:100A10003FF416AE0390FFF7D1FC41F2883000F0AE
:100A200087FF0B9800F0EEF900F0B8F9039B5746EA
:100A30001C461D46F0E5054689E64FF00008FFE537
:100A40002546FDE52C4667E6002000F039F80490C5
:100A5000049B002BFFF6E3AD012000F051F9049B4D
:100A6000213B122B3FF6D8AD01A252F823F000BF74
:100A7000350600085D060008CD06000819060008C6
:100A80001906000819060008610700085109000846
:100A900019080008B1080008E30800081109000857
:100AA000190600082909000819060008A30900080A
:100AB0004F07000819060008E7090008A086010092
:100AC00037B5114B1A780132D2B20024012A0146FF
:100AD0008DF8074011D80D4803681D6A4FF47A73EA
:100AE0004B4301220DF10701A847012805D1084B0E
:100AF0009DF807001C7003B030BD4FF4FA7000F091
:100B000017FF4FF0FF30F6E70024002048260020B2
:100B10008425002038B50E4B1A780132D2B2012A52
:100B200005460ED80B4803681C6A4FF47A734B4392
:100B300004222946A047042803D1074B002018703F
:100B400038BD4FF4FA7000F0F3FE4FF0FF3038BDBF
:100B500000240020482600208425002030B4054CC5
:100B60002368DD69044B0A46AC460146204630BC8A
:100B7000604700BF48260020A086010070B501F044
:100B800021F9094C094E20700025306823788342F2
:100B900008D901F011F9336805440133B5F5803FF8
:100BA0003360F2D370BD00BF852500208025002072
:100BB00001F0B6B900F1006000F5803000687047C0
:100BC00000F10060920000F5803001F041B90000B2
:100BD000054B1A68054B1B789B1A834202D91044B7
:100BE00001F0EAB80020704780250020852500200C
:100BF00038B5074D04462868204401F0E5F828B9C7
:100C000028682044BDE8384001F0F6B838BD00BF80
:100C10008025002010F0030308D1B0F5007F05D82F
:100C200000F10050A0F508400068704700207047B0
:100C3000014BC058704700BF107AFF1F014B186866
:100C4000704700BF002004E070B52A4B1C68C4F355
:100C50000B03240C63B140F21342934231D040F2B3
:100C6000194293422FD040F2214293422DD10323C7
:100C7000214A0C2505FB03235D6893F9082042F205
:100C800001039C4224D0B4F5805F23D041F20103DC
:100C90009C4221D041F203039C421FD041F2070342
:100CA0009C4208BF3122441E0C44013D0B46A34226
:100CB0001ED215F9016F581C96B1034600F8016C5D
:100CC000F5E70123D4E70223D2E73F220B4DD6E715
:100CD0003322E3E74122E1E75A22E4E75922E2E73F
:100CE0002C2584421D7001D9981C5A70401A70BD81
:100CF0001846FBE7002004E0D0330008C4330008A6
:100D0000022802BF024B4FF400129A61704700BFE5
:100D100000040240022802BF014B20229A61704762
:100D200000040240022801BF024A536983F02003F5
:100D3000536170470004024010B50023934203D072
:100D4000CC5CC4540133F9E710BD000030B5441E3B
:100D500014F9010F0B4660B193F90050854201F17F
:100D6000010106D11AB993F90020801A30BD013A69
:100D7000EEE7002AF7D1104630BD000002460346D8
:100D8000981A13F9011B0029FAD17047024403464F
:100D9000934202D003F8011BFAE77047024B1A781E
:100DA000024B1A70704700BF8425002000240020E9
:100DB00038B5104D104C284600F002F9214628465F
:100DC00000F02AF924680D48626DD2F8043843F027
:100DD0000203C2F8043800F0ABFD0949204600F0D8
:100DE00027FA626DD2F8043823F00203C2F80438FF
:100DF00038BD00BF482600209C34000840420F0048
:100E0000C434000870470000FEE7000000B59BB046
:100E1000EFF3098168226846FFF78EFFEFF3058341
:100E2000034B9A6B9A6A9A6A9A6A9A6A9B6AFEE775
:100E300000ED00E000B59BB0EFF309816822684641
:100E4000FFF77AFFEFF30583044B9A6B9A6A9A6A6D
:100E50009A6A9A6A9A6A9B6AFEE700BF00ED00E010
:100E600000B59BB0EFF3098168226846FFF764FF85
:100E7000EFF30583034B5A6B9A6A9A6A9A6A9A6AE5
:100E80009B6AFEE700ED00E030B5084D0A44914250
:100E90000BD011F8013B09245840013CF7D040F336
:100EA00000032B4083EA5000F7E730BD2083B8ED04
:100EB000002304491A465A50C8180833802B426050
:100EC000F9D170478825002002684368114301600A
:100ED00003B118477047000013B5446BD4F894343D
:100EE0001A681178042915D1217C022912D11979A7
:100EF000128901238B4013420CD101A904F14C004B
:100F000001F028FED4F89444019B21790246206820
:100F100000F0DAF902B010BD143001F0ABBD0000F2
:100F20004FF0FF33143001F0A5BD00004C3001F04C
:100F30007DBE00004FF0FF334C3001F077BE000063
:100F4000143001F079BD00004FF0FF31143001F092
:100F500073BD00004C3001F049BE00004FF0FF327D
:100F60004C3001F043BE0000D0F8942438B513682B
:100F700019780429054601D0012038BD017C0229D9
:100F8000FAD112795C89012090400440F4D105F136
:100F9000140001F00BFD02460028EDD0D5F8945462
:100FA0004FF480732868697900F07CF9204638BDD9
:100FB000406BFFF7D9BF000000207047704700006A
:100FC0007FB5124B0360002343608360C36001253B
:100FD00002260F4B057404460290019300F184022F
:100FE000294600964FF48073143001F0BBFC094B86
:100FF0000193029400964FF4807304F523722946FE
:1010000004F14C0001F082FD04B070BD20340008F2
:10101000B10F0008D90E00080B68202282F3118856
:101020000A7903EB820290614A79093243F822007F
:101030008A7912B103EB8203986102230374C0F82A
:101040009414002383F311887047000038B5037FA0
:10105000044613B190F85430ABB9201D012502218C
:10106000FFF732FF04F1140025776FF0010100F063
:1010700087FC84F8545004F14C006FF00101BDE886
:10108000384000F07DBC38BD10B501210446043065
:10109000FFF71AFF0023237784F8543010BD0000B7
:1010A00038B504460025143001F074FC04F14C00FE
:1010B000257701F043FD201D84F854500121FFF7EE
:1010C00003FF2046BDE83840FFF74EBF90F844309C
:1010D00003F06003202B19D190F84520212A0AD073
:1010E000222A4FF000030ED0202A0FD1084A826333
:1010F0000722C26304E0064B83630723C363002314
:101100000364012070478363C363F9E700207047DD
:1011100001240020D0F8943437B51A6811780429D6
:1011200004461AD1017C022917D1197912890123A9
:101130008B40134211D100F14C05284601F0BEFD51
:1011400058B101A9284601F005FDD4F89444019B4B
:1011500021790246206800F0B7F803B030BD0000E6
:1011600000EB8103F7B59C6905460E46F4B12023D8
:1011700083F3118805EB8607201D0821FFF7A4FEE5
:10118000FB685B691B684C3413B1204601F0F0FC2E
:1011900001A9204601F0DEFC024648B1019B314620
:1011A000284600F091F8002383F3118803B0F0BDC6
:1011B000FB685A691268002AF5D01B8A013B13406C
:1011C000F1D105F14402EAE7093138B550F8214080
:1011D000DCB1202383F31188D4F894241368527966
:1011E00003EB8203DB689B695D6845B104216018ED
:1011F000FFF76AFE294604F1140001F0E1FB2046E6
:10120000FFF7B2FE002383F3118838BD704700005A
:1012100000F08CBF0123037000234360C36183622D
:101220000362C3624362036303814381704700002A
:1012300038B50446202383F3118800254160C5603A
:1012400005614561856100F081FF0223237085F30C
:10125000118838BD70B500EB810305465069DA602E
:101260000E46144618B110220021FFF78FFDA06929
:1012700018B110220021FFF789FD31462846BDE84C
:10128000704001F02DB80000028902F001020281D5
:10129000428902F0010242810022026142618261C0
:1012A00001F0B2B8F0B400EB81044789E46801258D
:1012B000A4698D403D43458123600023A2606360A3
:1012C000F0BC01F0CDB80000F0B400EB8104078958
:1012D000E468012564698D403D4305812360002356
:1012E000A2606360F0BC01F047B9000070B5022352
:1012F000002504460370A0F84C5080F84E5080F84A
:101300004F5005814581C56005614561856180F863
:10131000345000F081FF63681B6823B129462046E2
:10132000BDE87040184770BD436802781B6880F8BC
:101330005020052202700BB10421184770470000AD
:10134000436890F850201B6802700BB105211847C4
:101350007047000090F8343070B5044613B1002394
:1013600080F8343004F14402204601F06FF86368DD
:101370009B6863BB94F8445015F0600615D194F84F
:10138000453005F07F0545EA032540F202339D42D2
:1013900000F00E815BD8022D00F0DC803FD8002DDC
:1013A00000F08780012D00F0CF800021204601F061
:1013B000A5FA0021204601F097FA63681B6813B173
:1013C000062120469847062384F8343070BD204615
:1013D00098470028CED094F84B2094F84A3043EA3E
:1013E0000223E26B934238BFE36394F94430E56B28
:1013F000002B4FF0200380F2FD80002D00F0EC80E8
:10140000092284F8342083F311880021E36BA26B56
:101410002046FFF759FF002383F3118870BDB5F50F
:10142000817F00F0B180B5F5407F49D0B5F5807F70
:10143000BBD194F84630012BB7D1B4F84C3023F02F
:101440000203A4F84C30A663E6632664C3E740F2C7
:1014500001639D421ED8B5F5C06F3BD2B5F5A06FB4
:10146000A3D1B4F84430B3F5A06F0ED194F8463050
:1014700084F84E30204600F027FF63681B6813B1E4
:10148000012120469847032323700023A363E363CD
:101490002364A0E7B5F5106F32D040F602439D42B9
:1014A00052D0B5F5006F80D104F14F03A36301233F
:1014B00024E004F14C03A3630223E36325648AE779
:1014C00094F84630012B7FF470AFB4F84C3043F001
:1014D0000203B6E794F84920616894F848304D68F3
:1014E00094F8471043EA0223204694F84620A84780
:1014F00000283FF45AAF4368A3630368E363A4E79B
:101500002378042B10D1202383F311882046FFF782
:10151000BBFE86F31188636884F84F601B68032163
:1015200021700BB12046984794F84630002BACD080
:1015300084F84F300423237063681B68002BA4D009
:10154000022120469847A0E7374BA3630223E363B9
:1015500000239DE794F8481011F0800F204601F019
:101560000F010ED000F064FF012806D002287FF49E
:101570001CAF2E4BA363E06367E72D4BA363E563CA
:1015800063E700F047FFEFE794F84630002B7FF465
:101590000CAF94F8483013F00F013FF476AF1A0601
:1015A000204602D501F0BEF96FE701F0B1F96CE712
:1015B00094F84630002B7FF4F8AE94F8483013F0DE
:1015C0000F013FF462AF1B06204602D501F096F9E9
:1015D0005BE701F089F958E7142284F8342083F39B
:1015E00011882B462A4629462046FFF75BFE85F3E5
:1015F000118870BD5DB1152284F8342083F3118801
:101600000021E36BA26B2046FFF74CFE03E70B22A1
:1016100084F8342083F311882B462A462946204635
:10162000FFF752FEE3E700BF5034000848340008DB
:101630004C34000838B590F834300446152B29D8BE
:10164000DFE803F03E28282828283E28280B2939DF
:1016500028282828282828283E3E90F84B1090F863
:101660004A20C36B42EA01229A4214D9C268128A04
:10167000B3FBF2F502FB15356DB9202383F3118816
:101680002B462A462946FFF71FFE85F311880A23B9
:1016900084F8343038BD142384F83430202383F3A5
:1016A000118800231A4619462046FFF7FBFD002348
:1016B00083F3118838BD036C03B198470023E7E733
:1016C000002101F01BF90021204601F00DF96368AB
:1016D0001B6813B10621204698470623D8E700006F
:1016E00090F83420152A38B5044622D801239340B7
:1016F00040F6416213421DD113F480150FD19B02B5
:1017000017D50B2380F83430202383F311882B4620
:101710002A462946FFF7D8FD85F3118838BDC368EE
:101720009B695B682BB9036C03B19847002384F86D
:10173000343038BD002101F0E1F80021204601F0ED
:10174000D3F863681B6813B1062120469847062327
:10175000EDE70000024B00221B605B609A6070475F
:1017600008260020002303748268054B1B689968D3
:101770009142FBD25A680360426010605860704723
:101780000826002008B5202383F31188037C032B4F
:1017900005D0042B0DD02BB983F3118808BD436904
:1017A00000221A604FF0FF334361FFF7DBFF002395
:1017B000F2E790E80C001A6002685360F2E700005C
:1017C000002303748268054B1B6899689142FBD81B
:1017D0005A68036042601060586070470826002015
:1017E000054B19690874186802681A60536018611B
:1017F00001230374FEF788BD0826002030B54B1C7A
:1018000087B005460A4C10D023690A4A01A800F0A7
:10181000D3F82846FFF7E4FF049B13B101A800F0BA
:1018200007F92369586907B030BDFFF7D9FFF8E71A
:10183000082600208517000838B50C4D41612B693A
:1018400081689A689142044603D8BDE83840FFF7A2
:1018500089BF1846FFF786FF01232C6101462374D8
:101860002046BDE83840FEF74FBD00BF08260020E7
:10187000044B1A681B6990689B68984294BF0020CB
:10188000012070470826002010B5084C2368206905
:101890001A6822605460012223611A74FFF790FFD6
:1018A00001462069BDE81040FEF72EBD0826002045
:1018B0008260022202740022427470478368A3F19E
:1018C0007C0243F80C2C026943F83C2C426943F833
:1018D000382C074A43F81C2CC26843F8102C02220B
:1018E00003F8082C002203F8072CA3F11800704716
:1018F0002103000810B5202383F31188FFF7DEFFD2
:1019000000210446FFF798FF002383F31188204647
:1019100010BD0000024B1B6958610F20FFF760BF2C
:1019200008260020202383F31188FFF7F3BF00006F
:1019300008B50146202383F311880820FFF75EFFD6
:10194000002383F3118808BD49B1064B42681B6927
:1019500018605A60136043600420FFF74FBF4FF0D8
:10196000FF307047082600200368984206D01A68A6
:101970000260506059611846FFF7F4BE70470000DE
:1019800038B504460D462068844200D138BD03684E
:1019900023605C604561FFF7E5FEF4E7054B03F16A
:1019A00014025A619A614FF0FF32DA6100221A6222
:1019B000704700BF08260020F8B503614FF0804350
:1019C000C2605C6A194B1A46022952F8145F38BF8C
:1019D0000221954206461F460AD1586198611C6251
:1019E0000560456081600819BDE8F84001F088B9DC
:1019F000186AAB68241A0C1902D3E41A2D6804E0A3
:101A00009C4202D2204401F089F9AB689C42F4D890
:101A10006B68736035601E606E60B460A9684FF0DB
:101A2000FF33091BA960FB61F8BD00BF0826002039
:101A300010B41B4C234653F8141F814210D0416848
:101A400002680A60026851609A424FF00001C1606A
:101A500003D0936881680B4493605DF8044B704732
:101A60000A68626100209A425360C86003D15DF841
:101A7000044B01F04DB993688868034493604FF0BC
:101A80008042206A526A121A9342E6D9991A0129B1
:101A900098BF931C18445DF8044B01F03FB900BF98
:101AA0000826002000207047FEE700007047000075
:101AB0004FF0FF3070470000022906D0032906D0FE
:101AC0000129064818BF0020704705487047032ABF
:101AD0009ABF044800EBC200002070472035000880
:101AE000D43400080824002070B59AB001AD064631
:101AF00008462946144600F095F82846FFF73EF9B7
:101B0000C0B2431C5B0086E8180023700323637097
:101B1000002302341946DAB2904204F1020401D8DB
:101B20001AB070BDEA5C04F8022C04F8011C013301
:101B3000F1E7000008B5202383F311880348FFF77D
:101B4000E9FA002383F3118808BD00BF482600206E
:101B500010B50446052916D8DFE801F0161503165E
:101B6000161D202383F311880E4A0121FFF772FB13
:101B700020460D4A0221FFF76DFB0C48FFF790FA53
:101B8000002383F3118810BD202383F311880748B5
:101B9000FFF75CFAF4E7202383F311880348FFF78B
:101BA00073FAEDE754340008783400084826002022
:101BB00038B50C4D0C4C0D492A4604F10800FFF7CE
:101BC00093FF05F1CA0204F110000949FFF78CFFE9
:101BD00005F5CA7204F118000649BDE83840FFF760
:101BE00083BF00BF102B002008240020A43400086D
:101BF000AE340008B934000870B5044608460D46F6
:101C0000FFF7BCF8C6B22046013403780BB918467A
:101C100070BD32462946FFF799F80028F3D101201C
:101C200070BD00002DE9F84F05460C46FFF7A6F8F9
:101C30002B49C6B22846FFF7DFFF08B10536F6B2DA
:101C400028492846FFF7D8FF08B11036F6B2632EB0
:101C50000DD8DFF88C80DFF88C90234FDFF890A050
:101C6000DFF890B02E7846B92670BDE8F88F294687
:101C70002046BDE8F84F01F099BB252E2CD1072254
:101C800041462846FFF762F858B9DBF80030236078
:101C9000DBF804306360DBF80830A36007350C34F0
:101CA000E0E7082249462846FFF750F8A0B90F4B55
:101CB000A21C13F8011F09095345C95D02F8021C53
:101CC000197801F00F0102F10202C95D02F8031C4C
:101CD000EFD118340835C5E7267001350134C1E766
:101CE00040350008B9340008553500080F7AFF1F49
:101CF0001B7AFF1F48350008BFF34F8F024AD36895
:101D0000DB03FCD4704700BF003C024008B5094B20
:101D10001B7873B9FFF7F0FF074B1A69002ABFBFA2
:101D2000064A5A6002F188325A601A6822F48062C8
:101D30001A6008BD6E2D0020003C0240230167455B
:101D400008B50B4B1B7893B9FFF7D6FF094B1A69FF
:101D500042F000421A611A6842F480521A601A680E
:101D600022F480521A601A6842F480621A6008BD38
:101D70006E2D0020003C02400B2870B513D80B4A92
:101D80000B4C137863B90B4E4FF0006144F82310ED
:101D900056F8235001330C2B2944F7D1012313703B
:101DA00054F8200070BD002070BD00BFA02D0020A1
:101DB000702D002068350008014B53F82000704753
:101DC000683500080C2070470B2810B5044601D96F
:101DD000002010BDFFF7D0FF064B53F82430184405
:101DE000C21A0BB9012010BD12680132F0D1043BB8
:101DF000F6E700BF683500080B2810B5044621D867
:101E0000FFF77AFFFFF782FF0F4AF323D360C30087
:101E1000DBB243F4007343F002031361136943F42C
:101E200080331361FFF768FFFFF7A6FF074B53F8F6
:101E3000241000F0DDF8FFF783FF2046BDE81040D6
:101E4000FFF7C2BF002010BD003C0240683500080B
:101E50002DE9F84312F00103154640D18218B2F182
:101E6000016F3CD22C4B1B6813F0010337D02B4C75
:101E7000FFF74CFFF323E360FFF73EFF40F201273B
:101E8000032D01D9830713D0244C0F46401A40F28A
:101E90000118EB1B0B44012B00EB0706236924D828
:101EA00023F001032361FFF74BFF0120BDE8F88316
:101EB000236923F44073236123693B43236151F871
:101EC000046B0660BFF34F8FFFF716FF03689E4257
:101ED00008D0236923F001032361FFF731FF0020BD
:101EE000BDE8F883043D0430CAE723F4407323615E
:101EF000236943EA08032361B94637F8023B33807C
:101F0000BFF34F8FFFF7F8FE3688B9F80030B6B24E
:101F1000B342BED0DDE700BF00380240003C0240C3
:101F2000084908B50B7828B153B9FFF7EFFE012334
:101F30000B7008BD23B1BDE808400870FFF700BF73
:101F400008BD00BF6E2D002010B50244064B0439B9
:101F5000D2B2904200D110BD441C00B253F8200010
:101F600041F8040FE0B2F4E750280040104B30B5C0
:101F70001C6F240407D41C6F44F400741C671C6F8E
:101F800044F400441C670B4C236843F480732360C3
:101F90000244094B0439D2B2904200D130BD441CF6
:101FA00000B251F8045F43F82050E0B2F4E700BFFC
:101FB00000380240007000405028004007B5012260
:101FC00001A90020FFF7C0FF019803B05DF804FBF2
:101FD00013B50446FFF7F2FFA04206D002A9012282
:101FE00041F8044D0020FFF7C1FF02B010BD000012
:101FF00070470000034B1B689B0042BF024B01224D
:102000001A70704774380240A12D0020014B1878D7
:10201000704700BFA12D002070470000FEE70000C0
:10202000084A094B09498B4204D3094A00219342CB
:1020300005D3704752F8040F43F8040BF3E743F855
:10204000041BF4E714370008183000201830002073
:1020500018300020836D30B500229D68446D114614
:102060004FF0FF3004EB421301329542C3F80019E0
:10207000C3F81019C3F80809C3F8001BC3F8101BF4
:10208000C3F8080BEED24FF00113C4F81C3830BD72
:10209000890141F02001016103699B06FCD41220F3
:1020A00000F0C4BE204B03EB80022DE9F047D2F8CC
:1020B0000CE05D6DDEF81420461CD2F800C005EB84
:1020C000063605EB4018516861450BD3D5F8342826
:1020D000012303FA00F022EA0000C5F8340818468C
:1020E000BDE8F087BEF81040ACEB0103A34228BF67
:1020F0002346D8F81849A4B2B3EB840F10D89468DB
:102100001F46A4F1040959F804AFC6F800A0042F33
:1021100001D9043FF7E71C440B4494605360D2E7B5
:102120000020BDE8F08700BFA42D002010B5054CAD
:102130002046FFF76FF84FF0A0436365024BA3659D
:1021400010BD00BFA42D0020BC3500080378012B72
:1021500070B5054650D12A4B446D98421BD1294B8E
:102160005A6B42F080025A635A6D42F080025A65FF
:102170005A6D5A6942F080025A615A6922F080020F
:102180005A610E2143205B6900F0D6FB1E4BE360D1
:102190001E4BC4F800380023C4F8003EC02323605F
:1021A0006E6D4FF40413A3633369002BFCDA012333
:1021B00033610C2000F03AFE3369DB07FCD41220B7
:1021C00000F034FE3369002BFCDA0026A6602846B6
:1021D000FFF740FF6B68C4F81068DB68C4F8146848
:1021E000C4F81C684BB90A4BA3614FF0FF3363611D
:1021F000A36843F00103A36070BD064BF4E700BF82
:10220000A42D0020003802404014004003002002AA
:10221000003C30C0083C30C0F8B5446D0546002194
:102220002046FFF735FFA96D00234FF001128F689C
:10223000C4F834384FF00066C4F81C284FF0FF3063
:1022400004EB431201339F42C2F80069C2F8006BED
:10225000C2F80809C2F8080BF2D20B686A6DEB6588
:10226000636210231361166916F01006FBD1122069
:1022700000F0DCFDD4F8003823F4FE63C4F8003825
:10228000A36943F4402343F01003A3610923C4F876
:102290001038C4F814380A4BEB604FF0C043C4F850
:1022A000103B084BC4F8003BC4F81069C4F800396F
:1022B000EB6D03F1100243F48013EA65A362F8BDED
:1022C0009835000840800010426D90F84E10D2F80A
:1022D000003823F4FE6343EA0113C2F80038704764
:1022E0002DE9F0410EB200EB86080D46D8F80C102F
:1022F0000F6807F00303022B50D0032B50D03D4A48
:102300003D4F012B18BF1746446D4FEA451E04EBA5
:102310000E030022C3F8102B8A6905F1100C002A65
:1023200040D04A8A05F158035B013A43E250012349
:10233000D4F81C2803FA0CF31343A6444A69C4F8E2
:102340001C380023CEF8103905F13F03002A39D09C
:102350000A8A898B9208012988BF4A43C16D04EB20
:102360008303561841EA0242C66529465A60204650
:10237000FFF78EFED8F80C301B8A43EA85531F43C3
:1023800005F148035B01E7500123D4F81C2803FA48
:1023900005F51543C4F81C58BDE8F081174FB3E7A5
:1023A000174FB1E704EB4613D3F8002B22F4004299
:1023B000C3F8002BD4F81C28012303FA0CF322EAFB
:1023C0000303BAE704EB83030E4A5A6004EB461694
:1023D00029462046FFF75CFED6F8003923F4004377
:1023E000C6F80039D4F81C38012202FA05F523EAB0
:1023F0000505CFE700800010008004100080081061
:1024000000800C1000040002826D1268C265FFF7A4
:1024100021BE00005831436D49015B5813F4004060
:1024200004D013F4001F14BF0120022070470000E5
:102430004831436D49015B5813F4004004D013F454
:10244000001F14BF012002207047000000EB810133
:10245000CB68196A0B6813604B68536070470000C3
:1024600000EB810330B5DD68AA691368D36019B940
:10247000402B84BF402313606B8A1468426D1C4458
:10248000013CB4FBF3F46343033323F0030302EB97
:10249000411043EAC44343F0C043C0F8103B2B68EB
:1024A00003F00303012B09B20ED1D2F8083802EB76
:1024B000411013F4807FD0F8003B14BF43F08053E9
:1024C00043F00053C0F8003B02EB4112D2F8003B4E
:1024D00043F00443C2F8003B30BD00002DE9F04159
:1024E000244D6E6D06EB40130446D3F8087BC3F809
:1024F000087B38070AD5D6F81438190706D505EB36
:1025000084032146DB6828465B689847FA072FD585
:10251000D6F81438DB072BD505EB8403D968CCB982
:102520008B69488A5E68B6FBF0F200FB12628AB9DA
:102530001868DA6890420DD2121A83E8140020233A
:1025400083F311880B482146FFF78AFF84F3118833
:10255000BDE8F081012303FA04F26B8923EA020348
:102560006B81CB6823B121460248BDE8F041184792
:10257000BDE8F081A42D002000EB810370B5DD687B
:10258000436D6C692668E6604A0156BB1A444FF4F5
:102590000020C2F810092A6802F00302012A0AB2D8
:1025A0000ED1D3F8080803EB421410F4807FD4F85E
:1025B000000914BF40F0805040F00050C4F80009FA
:1025C00003EB4212D2F8000940F00440C2F80009BF
:1025D000D3F83408012202FA01F10143C3F8341898
:1025E00070BD19B9402E84BF4020206020682E8A1B
:1025F000841940F00050013C1A44B4FBF6F440EA60
:10260000C440C6E7F8B504461E48456D05EB4413C3
:10261000D3F80869C3F80869F10717D5D5F8103859
:10262000DA0713D500EB8403D9684B691F68DA68B1
:10263000974218D2D21B00271A605F60202383F3D1
:1026400011882146FFF798FF87F31188330617D5C5
:10265000D5F834280123A340134211D02046BDE809
:10266000F840FFF71FBD012303FA04F2038923EAB0
:10267000020303818B68002BE8D021469847E5E7E9
:10268000F8BD00BFA42D002096482DE9F84F456DF8
:102690006E69AB691E4016F4805F6E61044605D01A
:1026A000FEF724FEBDE8F84F00F054BC002E12DA0D
:1026B000D5F8003E8B489B071EBFD5F8003E23F09F
:1026C0000303C5F8003ED5F8043823F00103C5F82C
:1026D0000438FEF735FE370502D58248FEF724FEA2
:1026E000B0040CD5D5F8083813F0060FEB6823F4C6
:1026F00070530CBF43F4105343F4A053EB60310705
:1027000004D56368DB680BB176489847F2025AD467
:10271000B3020CD5D4F85480DFF8C8A100274FF0DD
:102720000109A36D9B68F9B28B4280F08780F706A0
:1027300019D5616D0A6AC2F30A1702F00F0302F499
:10274000F012B2F5802F00F0A180B2F5402F0AD12F
:1027500004EB830301F58051DB68186A00231A46F5
:102760009F4240F087803003D5F8184813D5E10325
:1027700002D50020FFF7B2FEA20302D50120FFF729
:10278000ADFE630302D50220FFF7A8FE270302D5A2
:102790000320FFF7A3FE750384D5E00702D50020D0
:1027A000FFF730FFA10702D50120FFF72BFF6207DB
:1027B00002D50220FFF726FF23077FF573AF032022
:1027C000FFF720FF6EE7D4F85480DFF818A1002748
:1027D0004FF00109A36D9B685FFA87FB5B4597D3B8
:1027E00008EB4B13D3F8002902F44022B2F5802FF6
:1027F00022D1D3F80029002A1EDAD3F8002942F0AA
:102800009042C3F80029D3F80029002AFBDB59467F
:10281000606DFFF73DFC228909FA0BF322EA0303FE
:10282000238104EB8B03DB689B6813B15946504648
:1028300098475846FFF736FC0137CBE708EB4112C3
:10284000D2F8003B03F44023B3F5802F10D1D2F827
:10285000003B002B0CDA628909FA01F322EA030338
:10286000638104EB8103DB68DB680BB1504698475A
:10287000013756E79C0708BF0A68072B98BF02700C
:1028800003F101039CBF120A013069E7023304EB34
:10289000830201F58051526890690268D0F808C03F
:1028A0004068A2EB000E0022104697420AD104EBCA
:1028B000830463689B699A683A449A605A6817442B
:1028C0005F6050E712F0030F08BF0868964588BFA5
:1028D0008CF8000002F1010284BF000A0CF1010C27
:1028E000E3E700BFA42D0020436D03EB4111D1F8B5
:1028F000003B43F40013C1F8003B7047436D03EB0A
:102900004111D1F8003943F40013C1F80039704780
:10291000436D03EB4111D1F8003B23F40013C1F8E0
:10292000003B7047436D03EB4111D1F8003923F4AC
:102930000013C1F80039704700F1604300F01F0236
:10294000400903F5614309018000C9B200F160400C
:1029500083F8001300F5614001239340C0F88031F3
:102960000360704730B5039C0172043304FB0325F8
:10297000C361049B03630021059B00604060C1604C
:10298000426102618561046242628162C1624363A5
:1029900030BD00000022416A41610161C260826273
:1029A000C2626FF00101FEF7EBBF000003694269EC
:1029B000934203D1C2680AB100207047181D7047C6
:1029C00003691960C2680132C260C2691344826936
:1029D0000361934224BF436A03610021FEF7C4BF31
:1029E00038B504460D46E3683BB16269131D1268B1
:1029F000A3621344E362002038BD237A33B9294629
:102A00002046FEF7A1FF0028EDDA38BD6FF0010087
:102A1000FBE70000C368C269013BC360436913441C
:102A200082694361934224BF436A43610023836206
:102A3000036B03B11847704770B52023044683F336
:102A40001188866A3EB9FFF7CBFF054618B186F3B9
:102A50001188284670BDA36AE26A13F8015BA3627D
:102A6000934202D32046FFF7D5FF002383F311885A
:102A7000EFE700002DE9F84F04460E4690469946D0
:102A8000202787F311880025AA46D4F828B0BBF187
:102A9000000F09D149462046FFF7A2FF20B18BF372
:102AA00011882846BDE8F88FA16AE36AA8EB050BF8
:102AB0005B1A9B4528BF9B46BBF1400F1BD9334691
:102AC00001F1400251F8040B43F8040B9142F9D193
:102AD000A36A40334036A3624035A26AE36A9A4251
:102AE00002D32046FFF796FF8AF311884545D8D2D6
:102AF00087F31188C9E730465A46FEF71DF9A36AE5
:102B00005B445E44A3625D44E7E7000010B5029CAD
:102B10000172043303FB0421C36100238362C36297
:102B2000039B0363049B00604060C46042610261D8
:102B3000816104624262436310BD0000026AC260A8
:102B4000426A4261026100228262C2626FF0010148
:102B5000FEF716BF436902699A4203D1C2680AB1FF
:102B600000207047184650F8043B0B607047000087
:102B7000C368C2690133C360436913448269436116
:102B8000934224BF436A43610021FEF7EDBE00007B
:102B900038B504460D46E3683BB123691A1DA262AD
:102BA000E2691344E362002038BD237A33B9294631
:102BB0002046FEF7C9FE0028EDDA38BD6FF00100AF
:102BC000FBE7000003691960C268013AC260C2698C
:102BD000134482690361934224BF436A0361002363
:102BE0008362036B03B118477047000070B5202360
:102BF00004460E4683F31188856A35B91146FFF7FE
:102C0000C7FF10B185F3118870BDA36A1E70A36A57
:102C1000E26A01339342A36204D3E1692046043996
:102C2000FFF7D0FF002080F3118870BD2DE9F84F29
:102C300004460D4691469A464FF0200888F31188C5
:102C40000026B346A76A4FB951462046FFF7A0FFBA
:102C500020B187F311883046BDE8F88FA06AE76A93
:102C6000A9EB06033F1A9F4228BF1F46402F1BD9DE
:102C700005F1400355F8042B40F8042B9D42F9D18F
:102C8000A36A4033A3624036A26AE36A9A4204D33D
:102C9000E16920460439FFF795FF8BF311884E4513
:102CA000D9D288F31188CDE729463A46FEF744F891
:102CB000A36A3B443D44A3623E44E5E7026943699D
:102CC0009A4203D1C3681BB9184670470023FBE73B
:102CD000836A002BF8D0043B9B1AF5D01360C368BD
:102CE000013BC360C3691A44836902619A4224BFED
:102CF000436A0361002383620123E5E700F06CB9B6
:102D00004FF08043002258631A610222DA60704754
:102D10004FF080430022DA60704700004FF080439C
:102D200058637047FEE7000010B5174CFEF712FD20
:102D3000FEF734FE802215492046FEF7B9FD012337
:102D400044F8180C0374124B124AD96821F4E0615C
:102D50000904090C0A431049DA60CA6842F080721B
:102D6000CA600E490A6842F001020A601022DA774E
:102D7000202283F82220002383F3118862B60848BA
:102D8000BDE81040FEF7B6BD30260020C83500086B
:102D900000ED00E00003FA05F0ED00E0001000E0B7
:102DA000D03500082DE9F84F1F4C4FF00008656939
:102DB00004F11407C1464FF08043266A5B6AAA6893
:102DC0009E1B96421DD34FF0200AAA68236AD5F8AD
:102DD0000CB0134423622B68BB425F60A6EB020673
:102DE0006361C5F80C8001D1FFF792FF89F3118868
:102DF0002869D8478AF311886569AB689E42E4D296
:102E0000D9E76269BA420CD0916823628E1B966042
:102E1000A86802282CBF1818981CBDE8F84FFFF7C7
:102E20007DBFBDE8F88F00BF08260020034B59681E
:102E30005A68521A9042FBD8704700BF001000E059
:102E40004B6843608B688360CB68C3600B694361E8
:102E50004B6903628B6943620B6803607047000033
:102E600008B5224B22481A6940F2FF110A431A6141
:102E70001A6922F4FF7222F001021A611A691A6BB0
:102E80000A431A631A6D0A431A651A4A1B6D1146E2
:102E9000FFF7D6FF184802F11C01FFF7D1FF1748D2
:102EA00002F13801FFF7CCFF154802F15401FFF79A
:102EB000C7FF144802F17001FFF7C2FF124802F188
:102EC0008C01FFF7BDFF114802F1A801FFF7B8FF21
:102ED0000F4802F1C401FFF7B3FF0E4802F1E00111
:102EE000FFF7AEFFBDE8084000F0E0B80038024050
:102EF00000000240F03500080004024000080240D3
:102F0000000C024000100240001402400018024071
:102F1000001C02400020024008B500F037FAFFF71D
:102F200003FFFFF767F8BDE80840FEF741BE000069
:102F300070470000064A536823F001035360EFF323
:102F40000983683383F30988002383F3118870476A
:102F500030EF00E010B5202383F31188104B5B683D
:102F600013F4006318D0F1EE103AEFF309844FF038
:102F7000807344F84C3C0B4BDB6844F8083CA4F1EC
:102F8000680383F30988FEF773FC18B1064B44F815
:102F9000503C10BD054BFAE783F3118810BD00BF0C
:102FA00000ED00E030EF00E03103000834030008DA
:102FB0004FF0804310B51A69920708D500241C61B0
:102FC000202383F31188FFF7EDFE84F31188BDE819
:102FD0001040FFF7BFBF0000104B1A6C42F0010217
:102FE0001A641A6E42F001021A660D4A1B6E93684B
:102FF00043F0010393604FF0804353229A624FF0F5
:10300000FF32DA6200229A615A63DA605A60012262
:103010005A6108211A601C20FFF78EBC003802405C
:10302000002004E01F4B1A696FEAC2526FEAD252C5
:103030001A611A69C2F308021A614FF0FF301A6967
:103040005A69586100215A6959615A691A6A62F0CD
:1030500080521A621A6A02F080521A621A6A5A6A16
:1030600058625A6A59625A6A1A6C42F080521A645B
:103070001A6E42F080521A661A6E0B4A106840F4BB
:1030800080701060186F00F44070B0F5007F1EBFB4
:103090004FF4803018671967536823F40073536046
:1030A00000F054B90038024000700040304B4FF03F
:1030B00080521A642F4A4FF4404111601A6842F05E
:1030C00001021A601A689207FCD59A6822F003027E
:1030D0009A60274B19469A6812F00C02FBD11868C7
:1030E00000F0F90018609A601A6842F480321A60A1
:1030F0000B689B03FCD54B6F43F001034B671C4BE4
:103100005A6F9007FCD51C4A5A601A6842F08072C8
:103110001A60184A53685904FCD5154B1A68920175
:10312000FCD5164A9A60164B1A68164B9A42164BF3
:103130001BD1164A1168164A914216D140F2051267
:103140001A600B4B9A6842F002029A609A6802F089
:103150000C02082AFAD15A6C42F480425A645A6E20
:1031600042F480425A665B6E704740F20572E7E7B0
:10317000003802400070004008544007009488382E
:10318000002004E011640020003C024000ED00E05B
:1031900041C20F41084A08B5536911680B4003F05A
:1031A0000103536123B1054A13680BB15068984776
:1031B000BDE80840FFF7CEBE003C01408825002056
:1031C000084A08B5536911680B4003F002035361C4
:1031D00023B1054A93680BB1D0689847BDE8084011
:1031E000FFF7B8BE003C014088250020084A08B51A
:1031F000536911680B4003F00403536123B1054A7E
:1032000013690BB150699847BDE80840FFF7A2BEAB
:10321000003C014088250020084A08B55369116820
:103220000B4003F00803536123B1054A93690BB1C6
:10323000D0699847BDE80840FFF78CBE003C0140CC
:1032400088250020084A08B5536911680B4003F02F
:103250001003536123B1054A136A0BB1506A9847B2
:10326000BDE80840FFF776BE003C014088250020FD
:10327000174B10B55C691A68144004F478725A61EF
:10328000A30604D5134A936A0BB1D06A9847600627
:1032900004D5104A136B0BB1506B9847210604D527
:1032A0000C4A936B0BB1D06B9847E20504D5094AE1
:1032B000136C0BB1506C9847A30504D5054A936C69
:1032C0000BB1D06C9847BDE81040FFF743BE00BF7C
:1032D000003C0140882500201A4B10B55C691A6833
:1032E000144004F47C425A61620504D5164A136DF9
:1032F0000BB1506D9847230504D5134A936D0BB15C
:10330000D06D9847E00404D50F4A136E0BB1506E90
:103310009847A10404D50C4A936E0BB1D06E984720
:10332000620404D5084A136F0BB1506F9847230409
:1033300004D5054A936F0BB1D06F9847BDE8104094
:10334000FFF708BE003C014088250020062108B593
:103350000846FFF7F1FA06210720FFF7EDFA0621EC
:103360000820FFF7E9FA06210920FFF7E5FA062110
:103370000A20FFF7E1FA06211720FFF7DDFA062100
:103380002820BDE80840FFF7D7BA000008B5FFF7CE
:1033900049FEFDF78DFDFDF73BFFFDF70FFEFFF743
:1033A000C7FDBDE80840FFF7A9BC0000034611F8BF
:1033B000012B03F8012B002AF9D1704712101213C8
:1033C0001211000053544D3332463F3F3F0000007E
:1033D00000000000C43300083F0000001304000098
:1033E000003400083F000000190400000A340008FF
:1033F0003F00000021040000143400083F000000DA
:1034000053544D3332463430780053544D333246A2
:103410003432780053544D333246343436585800E1
:1034200000000000350F0008210F00085D0F0008A4
:10343000490F0008550F0008410F00082D0F000824
:10344000190F0008B90F000800000000010000007B
:1034500000000000020000000000000061110008F0
:10346000C911000840004000E02A0020F02A002096
:103470000200000000000000030000000000000047
:103480000D1200080000000010000000002B0020BA
:10349000000000000100000000000000A42D00203A
:1034A000010102004172647550696C6F740025421D
:1034B0004F415244252D424C002553455249414C21
:1034C00025000000511B0008B91A0008CD100008A3
:1034D000351B000843000000DC34000809024300EB
:1034E000020100C0320904000001020201000524AB
:1034F0000010010524010001042402020524060035
:1035000001070582030800FF09040100020A000008
:10351000000705010240000007058102400000008D
:1035200012000000283500081201100102000040BE
:1035300009124157000201020301000004030904BB
:1035400025424F41524425006F6D6E696275736666
:103550003470726F00303132333435363738394198
:103560004243444546000000004000000040000087
:1035700000400000004000000000010000000200C8
:103580000000020000000200000002000000020033
:1035900000000200000002000000000055130008B7
:1035A00035160008E116000840004000042E0020F7
:1035B000042E002001000000142E002080000000D6
:1035C00040010000030000006D61696E0000000012
:1035D000E8350008202E00201830002001000000EF
:1035E000252D00080000000069646C6500000000E3
:1035F0000001804200000000AAAAAAAA000100401F
:10360000FFFF00000000000000A00A0040050001CC
:1036100000000000AAAAAAAA40020001CFFF0000F1
:10362000000000000000000000000000000000009A
:10363000AAAAAAAA00000000FFFF000000000000E4
:10364000000000000000000000000000AAAAAAAAD2
:1036500000000000FFFF000000000000000000006C
:103660000000000000000000AAAAAAAA00000000B2
:10367000FFFF00000000000000000000000000004C
:1036800000000000AAAAAAAA00000000FFFF000094
:10369000000000000000000000000000000000002A
:1036A000AAAAAAAA00000000FFFF00000000000074
:1036B0000000000000000000000000000A00000000
:1036C00000000000030000000000000000000000F7
:1036D00000000000000000000000000000000000EA
:1036E00000000000000000000000000000000000DA
:1036F000FF00960000000008040000003C350008B0
:1037000000000000000000000000000000000000B9
:103710000000000000000000FFFFFFFFFFFFFFFFB1
:10372000FFFFFFFFFFFFFFFFFFFFFFFFFFFFFFFFA9
:10373000FFFFFFFFFFFFFFFFFFFFFFFFFFFFFFFF99
:10374000FFFFFFFFFFFFFFFFFFFFFFFFFFFFFFFF89
:10375000FFFFFFFFFFFFFFFFFFFFFFFFFFFFFFFF79
:020000040801F1
:1000000000060020B5120108755C0908D15B0908DB
:100010003D5C0908D15B0908095C0908B7120108B1
:10002000B7120108B7120108B7120108858B0B0837
:10003000B7120108B7120108B7120108B712010878
:10004000B7120108B7120108B7120108B712010868
:10005000B7120108B71201081D970B0845970B0846
:100060006D970B0895970B08BD970B08453C0B083F
:100070006D3C0B08993C0B08C53C0B08F13C0B0888
:10008000193D0B08453D0B08C93B0B08B712010889
:10009000B7120108B7120108B7120108E5970B085B
:1000A00009990B080D990B0821990B0825990B0844
:1000B00029990B083D990B0851990B08B7120108B3
:1000C000B7120108D1420B0879440B08B712010896
:1000D000B7120108B9980B08B7120108CD980B08A0
:1000E00049980B08B7120108B712010875990B0857
:1000F00079990B088D990B0891990B08713D0B08A4
:10010000B7120108B712010865990B08B712010868
:10011000E1980B08B7120108B7120108B7120108DD
:100120009D3D0B08C53D0B08F13D0B081D3E0B081E
:10013000493E0B08B7120108B7120108B7120108AF
:10014000B7120108B7120108B7120108B1920B08E3
:10015000713E0B089D3E0B08C93E0B08F5980B0835
:10016000B7120108B7120108B7120108B712010847
:10017000B7120108B7120108B7120108B712010837
:10018000B7120108B7120108B7120108B712010827
:10019000B7120108B7120108B7120108B712010817
:1001A000B7120108B7120108B7120108B712010807
:1001B000B7120108B7120108B7120108B7120108F7
:1001C000B7120108B7120108B7120108B7120108E7
:1001D000B7120108B7120108B7120108B7120108D7
:1001E0009D580108D184020805FA0308FDB70508E7
:1001F00021BE0508CD1C0608558106081989060888
:10020000518C0608C9F10608E518070859EE0708D9
:1002100049490808A1560808294E09080D5309083C
:10022000112B0A0889860A08E1AC0A0899B70A085E
:1002300061E70A0841EE0A08000000000000000023
:1002400081F0004102E000BF83F0004330B54FEA87
:1002500041044FEA430594EA050F08BF90EA020FF4
:100260001FBF54EA000C55EA020C7FEA645C7FEA87
:10027000655C00F0E2804FEA5454D4EB5555B8BFAA
:100280006D420CDD2C4480EA020281EA030382EA1B
:10029000000083EA010180EA020281EA0303362DAD
:1002A00088BF30BD11F0004F4FEA01314FF4801C80
:1002B0004CEA113102D0404261EB410113F0004F92
:1002C0004FEA03334CEA133302D0524263EB430349
:1002D00094EA050F00F0A780A4F10104D5F1200EE7
:1002E0000DDB02FA0EFC22FA05F2801841F1000142
:1002F00003FA0EF2801843FA05F359410EE0A5F116
:1003000020050EF1200E012A03FA0EFC28BF4CF046
:10031000020C43FA05F3C01851EBE37101F00045FC
:1003200007D54FF0000EDCF1000C7EEB00006EEB09
:100330000101B1F5801F1BD3B1F5001F0CD3490893
:100340005FEA30004FEA3C0C04F101044FEA4452EA
:1003500012F5800F80F09A80BCF1004F08BF5FEA71
:10036000500C50F1000041EB045141EA050130BD51
:100370005FEA4C0C404141EB0101013C28BFB1F563
:10038000801FE9D291F0000F04BF01460020B1FAAE
:1003900081F308BF2033A3F10B03B3F120020CDA81
:1003A0000C3208DD02F1140CC2F10C0201FA0CF05F
:1003B00021FA02F10CE002F11402D8BFC2F1200CC4
:1003C00001FA02F120FA0CFCDCBF41EA0C0190407A
:1003D000E41AA2BF01EB0451294330BD6FEA0404C3
:1003E0001F3C1CDA0C340EDC04F11404C4F12002AE
:1003F00020FA04F001FA02F340EA030021FA04F3C0
:1004000045EA030130BDC4F10C04C4F1200220FA16
:1004100002F001FA04F340EA0300294630BD21FA54
:1004200004F0294630BD94F0000F83F4801306BF1A
:1004300081F480110134013D4EE77FEA645C18BF0E
:100440007FEA655C29D094EA050F08BF90EA020FA5
:1004500005D054EA000C04BF1946104630BD91EA9D
:10046000030F1EBF0021002030BD5FEA545C05D1A0
:100470004000494128BF41F0004130BD14F58004DF
:100480003CBF01F5801130BD01F0004545F0FE4153
:1004900041F470014FF0000030BD7FEA645C1ABF88
:1004A000194610467FEA655C1CBF0B46024650EABF
:1004B000013406BF52EA033591EA030F41F40021EB
:1004C00030BD00BF90F0000F04BF0021704730B571
:1004D0004FF4806404F132044FF000054FF0000146
:1004E00050E700BF90F0000F04BF0021704730B507
:1004F0004FF4806404F1320410F0004548BF4042DC
:100500004FF000013EE700BF42004FEAE2014FEA30
:1005100031014FEA02701FBF12F07F4393F07F4F0B
:1005200081F06051704732F07F4208BF704793F00E
:100530007F4F04BF41F40021704730B54FF4607421
:1005400001F0004521F000411CE700BF50EA010224
:1005500008BF704730B54FF000050AE050EA0102CD
:1005600008BF704730B511F0004502D5404261EB3D
:1005700041014FF4806404F132045FEA915C3FF47E
:10058000D8AE4FF003025FEADC0C18BF03325FEA1B
:10059000DC0C18BF033202EBDC02C2F1200300FACC
:1005A00003FC20FA02F001FA03FE40EA0E0021FAF1
:1005B00002F11444BDE600BF70B54FF0FF0C4CF4DF
:1005C000E06C1CEA11541DBF1CEA135594EA0C0F91
:1005D00095EA0C0F00F0DEF82C4481EA030621EACC
:1005E0004C5123EA4C5350EA013518BF52EA033507
:1005F00041F4801143F4801338D0A0FB02CE4FF0B9
:100600000005E1FB02E506F00042E0FB03E54FF0E8
:100610000006E1FB03569CF0000F18BF4EF0010EE0
:10062000A4F1FF04B6F5007F64F5407404D25FEADC
:100630004E0E6D4146EB060642EAC62141EA55518F
:100640004FEAC52040EA5E504FEACE2EB4F1FD0CD1
:1006500088BFBCF5E06F1ED8BEF1004F08BF5FEA4F
:10066000500E50F1000041EB045170BD06F0004601
:1006700046EA010140EA020081EA0301B4EB5C04AE
:10068000C2BFD4EB0C0541EA045170BD41F48011A6
:100690004FF0000E013C00F3AB8014F1360FDEBFCB
:1006A000002001F0004170BDC4F10004203C35DAA7
:1006B0000C341BDC04F11404C4F1200500FA05F32A
:1006C00020FA04F001FA05F240EA020001F00042CB
:1006D00021F0004110EBD37021FA04F642EB060141
:1006E0005EEA430E08BF20EAD37070BDC4F10C046B
:1006F000C4F1200500FA04F320FA05F001FA04F22F
:1007000040EA020001F0004110EBD37041F100011A
:100710005EEA430E08BF20EAD37070BDC4F1200525
:1007200000FA05F24EEA020E20FA04F301FA05F28D
:1007300043EA020321FA04F001F0004121FA04F235
:1007400020EA020000EBD3705EEA430E08BF20EA05
:10075000D37070BD94F0000F0FD101F0004640003F
:1007600041EB010111F4801F08BF013CF7D041EAC1
:10077000060195F0000F18BF704703F000465200C5
:1007800043EB030313F4801F08BF013DF7D043EA96
:100790000603704794EA0C0F0CEA135518BF95EA4C
:1007A0000C0F0CD050EA410618BF52EA4306D1D1D3
:1007B00081EA030101F000414FF0000070BD50EAF2
:1007C000410606BF1046194652EA430619D094EA7C
:1007D0000C0F02D150EA013613D195EA0C0F05D166
:1007E00052EA03361CBF104619460AD181EA0301BA
:1007F00001F0004141F0FE4141F470014FF0000072
:1008000070BD41F0FE4141F4780170BD70B54FF00C
:10081000FF0C4CF4E06C1CEA11541DBF1CEA13558C
:1008200094EA0C0F95EA0C0F00F0A7F8A4EB05046E
:1008300081EA030E52EA03354FEA013100F0888065
:100840004FEA03334FF0805545EA131343EA12632E
:100850004FEA022245EA111545EA10654FEA0026E3
:100860000EF000419D4208BF964244F1FD0404F59C
:10087000407402D25B084FEA3202B61A65EB0305F8
:100880005B084FEA32024FF480104FF4002CB6EBB5
:10089000020E75EB030E22BFB61A754640EA0C0035
:1008A0005B084FEA3202B6EB020E75EB030E22BF75
:1008B000B61A754640EA5C005B084FEA3202B6EBB6
:1008C000020E75EB030E22BFB61A754640EA9C0075
:1008D0005B084FEA3202B6EB020E75EB030E22BF45
:1008E000B61A754640EADC0055EA060E18D04FEA03
:1008F000051545EA16754FEA06164FEAC30343EAA3
:1009000052734FEAC2025FEA1C1CC0D111F4801F6F
:100910000BD141EA00014FF000004FF0004CB6E768
:1009200011F4801F04BF01430020B4F1FD0C88BF07
:10093000BCF5E06F3FF6AFAEB5EB030C04BFB6EB12
:10094000020C5FEA500C50F1000041EB045170BD05
:100950000EF0004E4EEA113114EB5C04C2BFD4EB32
:100960000C0541EA045170BD41F480114FF0000EB6
:10097000013C90E645EA060E8DE60CEA135594EA32
:100980000C0F08BF95EA0C0F3FF43BAF94EA0C0F35
:100990000AD150EA01347FF434AF95EA0C0F7FF4AA
:1009A00025AF104619462CE795EA0C0F06D152EAFE
:1009B00003353FF4FDAE1046194622E750EA4106E2
:1009C00018BF52EA43067FF4C5AE50EA41047FF4F3
:1009D0000DAF52EA43057FF4EBAE12E74FF0FF3C58
:1009E00006E000BF4FF0010C02E000BF4FF0010C29
:1009F0004DF804CD4FEA410C7FEA6C5C4FEA430CA2
:100A000018BF7FEA6C5C1BD001B050EA410C0CBFF0
:100A100052EA430C91EA030F02BF90EA020F002052
:100A2000704710F1000F91EA030F58BF994208BFB9
:100A300090422CBFD8176FEAE37040F00100704776
:100A40004FEA410C7FEA6C5C02D150EA013C07D1CD
:100A50004FEA430C7FEA6C5CD6D152EA033CD3D018
:100A60005DF8040B704700BF8446104662468C4612
:100A70001946634600E000BF01B5FFF7B7FF002845
:100A800048BF10F1000F01BD4DF808EDFFF7F4FF6E
:100A90000CBF012000205DF808FB00BF4DF808EDF9
:100AA000FFF7EAFF34BF012000205DF808FB00BF1C
:100AB0004DF808EDFFF7E0FF94BF012000205DF83E
:100AC00008FB00BF4DF808EDFFF7CEFF94BF0120F3
:100AD00000205DF808FB00BF4DF808EDFFF7C4FFEC
:100AE00034BF012000205DF808FB00BF4FEA410C35
:100AF0007FEA6C5C02D150EA013C0AD14FEA430C18
:100B00007FEA6C5C02D152EA033C02D14FF0000054
:100B100070474FF0010070474FEA410212F5001292
:100B200015D211D56FF47873B3EB625212D94FEA34
:100B3000C12343F0004343EA505311F0004F23FA1E
:100B400002F018BF404270474FF00000704750EA73
:100B5000013005D111F0004008BF6FF00040704730
:100B60004FF00000704700BF4A0011D212F500128A
:100B700011D20DD56FF47873B3EB62520ED44FEAF5
:100B8000C12343F0004343EA505323FA02F0704775
:100B90004FF00000704750EA013002D14FF0FF30B3
:100BA00070474FF0000070474FEA4102B2F1E04356
:100BB00024BFB3F5001CDCF1FE5C0DD901F0004C44
:100BC0004FEAC0024CEA5070B2F1004F40EB830094
:100BD00008BF20F00100704711F0804F21D113F1C0
:100BE0003872BCBF01F00040704741F480114FEAF9
:100BF0005252C2F11802C2F1200C10FA0CF320FA82
:100C000002F018BF40F001004FEAC1234FEAD3239E
:100C100003FA0CFC40EA0C0023FA02F34FEA430308
:100C2000CCE77FEA625307D150EA01331EBF4FF091
:100C3000FE4040F44000704701F0004040F0FE40AC
:100C400040F40000704700BF80F0004002E000BFA9
:100C500081F0004142001FBF5FEA410392EA030FA7
:100C60007FEA226C7FEA236C6AD04FEA1262D2EBF1
:100C70001363C1BFD218414048404140B8BF5B42F6
:100C8000192B88BF704710F0004F40F4000020F08F
:100C90007F4018BF404211F0004F41F4000121F0A5
:100CA0007F4118BF494292EA030F3FD0A2F10102EF
:100CB00041FA03FC10EB0C00C3F1200301FA03F12D
:100CC00000F0004302D5494260EB4000B0F5000F50
:100CD00013D3B0F1807F06D340084FEA310102F10F
:100CE0000102FE2A51D2B1F1004F40EBC25008BFC1
:100CF00020F0010040EA03007047490040EB00008B
:100D0000013A28BFB0F5000FEDD2B0FA80FCACF18B
:100D1000080CB2EB0C0200FA0CF0AABF00EBC250B8
:100D200052421843BCBFD0401843704792F0000FA6
:100D300081F4000106BF80F400000132013BB5E7F9
:100D40004FEA41037FEA226C18BF7FEA236C21D06F
:100D500092EA030F04D092F0000F08BF08467047D4
:100D600090EA010F1CBF0020704712F07F4F04D1A2
:100D7000400028BF40F00040704712F100723CBFB5
:100D800000F50000704700F0004343F0FE4040F4DF
:100D9000000070477FEA226216BF08467FEA23639D
:100DA0000146420206BF5FEA412390EA010F40F488
:100DB000800070474FF0000304E000BF10F00043D4
:100DC00048BF40425FEA000C08BF704743F09643BB
:100DD00001464FF000001CE050EA010208BF7047D6
:100DE0004FF000030AE000BF50EA010208BF70475D
:100DF00011F0004302D5404261EB41015FEA010C72
:100E000002BF84460146002043F0B64308BFA3F169
:100E10008053A3F50003BCFA8CF2083AA3EBC2534B
:100E200010DB01FA02FC634400FA02FCC2F120026A
:100E3000BCF1004F20FA02F243EB020008BF20F0A1
:100E40000100704702F1200201FA02FCC2F1200207
:100E500050EA4C0021FA02F243EB020008BF20EAFC
:100E6000DC7070477BB972B90029BEBF00204FF01B
:100E7000004106E008BF00281CBF6FF000414FF0A2
:100E8000FF3000F015BAADF1080C6DE904CE002971
:100E900009DB002B1ADB00F0A3F8DDF804E0DDE944
:100EA000022304B07047404261EB4101002B1BDB81
:100EB00000F096F8DDF804E0DDE9022304B04042DA
:100EC00061EB4101524263EB43037047524263EBD3
:100ED000430300F085F8DDF804E0DDE9022304B007
:100EE000404261EB41017047524263EB430300F023
:100EF00077F8DDF804E0DDE9022304B0524263EB49
:100F00004303704753B94AB9002908BF00281CBFE2
:100F10004FF0FF314FF0FF3000F0CAB9ADF1080CCF
:100F20006DE904CE00F05CF8DDF804E0DDE90223B1
:100F300004B0704730B1012390FAA0F0B0FA80F00D
:100F40001844704708460029FBD02123F4E700BF6E
:100F5000430803F05533C01A830803F0333300F01D
:100F60003330184400EB101000F00F3000EB00207D
:100F700000EB0040000E704707EE900AF5EEC07AD5
:100F8000F1EE10FA01D400F00BB8F1EE677A08B573
:100F900017EE900A00F004F8404261EB410108BDF1
:100FA000D0B5FFF7B1FA0C4B002206460F46FFF70B
:100FB00003FBFFF7D9FD0446FFF784FA074B002235
:100FC000FFF7FAFA02460B4630463946FFF73CF97E
:100FD000FFF7CAFD2146D0BD0000F03D0000F04102
:100FE0002DE9F047089D04468E46002B4DD18A42DC
:100FF000944669D9B2FA82F252B101FA02F3C2F10F
:10100000200120FA01F10CFA02FC41EA030E94409F
:101010004FEA1C48210CBEFBF8F61FFA8CF708FBC0
:1010200016E341EA034306FB07F199420AD91CEB98
:10103000030306F1FF3080F01F81994240F21C81CA
:10104000023E63445B1AA4B2B3FBF8F008FB103312
:1010500044EA034400FB07F7A7420AD91CEB040447
:1010600000F1FF3380F00A81A74240F20781644417
:10107000023840EA0640E41B00261DB1D44000239C
:10108000C5E900433146BDE8F0878B4209D9002D00
:1010900000F0EF800026C5E9000130463146BDE88A
:1010A000F087B3FA83F6002E4AD18B4202D38242F4
:1010B00000F2F980841A61EB030301209E46002DA3
:1010C000E0D0C5E9004EDDE702B9FFDEB2FA82F2F8
:1010D000002A40F09280A1EB0C014FEA1C471FFA56
:1010E0008CFE0126200CB1FBF7F307FB131140EA3D
:1010F00001410EFB03F0884208D91CEB010103F10A
:10110000FF3802D2884200F2CB804346091AA4B2CB
:10111000B1FBF7F007FB101144EA01440EFB00FE9F
:10112000A64508D91CEB040400F1FF3102D2A64504
:1011300000F2BB800846A4EB0E0440EA03409CE7A3
:10114000C6F12007B34022FA07FC4CEA030C20FA50
:1011500007F401FA06F31C43F9404FEA1C4900FA70
:1011600006F3B1FBF9F8200C1FFA8CFE09FB1811ED
:1011700040EA014108FB0EF0884202FA06F20BD960
:101180001CEB010108F1FF3A80F08880884240F2B0
:101190008580A8F102086144091AA4B2B1FBF9F0F4
:1011A00009FB101144EA014100FB0EFE8E4508D9EF
:1011B0001CEB010100F1FF346CD28E456AD9023874
:1011C000614440EA0840A0FB0294A1EB0E01A14259
:1011D000C846A64656D353D05DB1B3EB080261EBC7
:1011E0000E0101FA07F722FA06F3F1401F43C5E9A1
:1011F000007100263146BDE8F087C2F12003D840D7
:101200000CFA02FC21FA03F3914001434FEA1C4718
:101210001FFA8CFEB3FBF7F007FB10360B0C43EA0A
:10122000064300FB0EF69E4204FA02F408D91CEBBA
:10123000030300F1FF382FD29E422DD902386344B8
:101240009B1B89B2B3FBF7F607FB163341EA034158
:1012500006FB0EF38B4208D91CEB010106F1FF38A7
:1012600016D28B4214D9023E6144C91A46EA00469E
:1012700038E72E46284605E70646E3E61846F8E630
:101280004B45A9D2B9EB020864EB0C0E0138A3E779
:101290004646EAE7204694E74046D1E7D0467BE75A
:1012A000023B614432E7304609E76444023842E7D2
:1012B000704700BF02E000F000F8FEE772B6374862
:1012C00080F30888364880F3098836483649086034
:1012D00040F20000CCF200004EF63471CEF2000174
:1012E0000860BFF34F8FBFF36F8F40F20000C0F272
:1012F000F0004EF68851CEF200010860BFF34F8F28
:10130000BFF36F8F4FF00000E1EE100A4EF63C7114
:10131000CEF200010860062080F31488BFF36F8FBF
:10132000A7F08EFCA6F0F6FC4FF055301F491B4A83
:1013300091423CBF41F8040BFAE71D49184A91421B
:101340003CBF41F8040BFAE71A491B4A1B4B9A426F
:101350003EBF51F8040B42F8040BF8E7002018498F
:10136000184A91423CBF41F8040BFAE7A7F06CFC25
:10137000A6F024FD144C154DAC4203DA54F8041BBE
:101380008847F9E701F010F9114C124DAC4203DA2D
:1013900054F8041B8847F9E7A7F054BC0006002066
:1013A000002200200000010808ED00E000000020FD
:1013B00000060020581B0E0800220020842C00206C
:1013C000882C0020A0520120E00101083802010809
:1013D00038020108380201082DE9F04F2DED108A7E
:1013E000C1F80CD0C3689D46BDEC108ABDE8F08FF3
:1013F000002383F311882846A0470020A6F010FAA6
:10140000FEE7A6F06DF800DFFEE7000001F0FF0147
:10141000102A2BDB10F0070F08D010F8013B013A1F
:101420008B422DD010F0070F42B3F6D1F0B441EA51
:10143000012141EA014122F007047FF00007002367
:10144000F0E80256083C85EA010586EA010685FABD
:1014500047F5A3FA87F586FA47F6A5FA87F68EB917
:10146000EED1F0BC01F0FF0102F0070232B110F83A
:10147000013B013A83EA010313B1F8D10020704720
:1014800001387047002D06BF35460338073815F080
:10149000010F07D1013015F4807F02BF013015F430
:1014A000C03F0130F0BC0138704700BF10F8012B7D
:1014B00011F8013B012A28BF9A42F7D0D01A704791
:1014C000034613F8012B002AFBD1181A0138704784
:1014D00038B50022002304460D46FFF7DFFA28B98D
:1014E00020462946BDE8384000F00AB8204605F1FC
:1014F000004100F005F8404261EB410138BD00BFFA
:10150000D0B50C4B002206460F46FFF755F8FFF703
:101510002BFB0446FEF7D6FF074B0022FFF74CF8E3
:1015200002460B4630463946FEF78EFEFFF71CFB9F
:101530002146D0BD0000F03D0000F04103680022CC
:101540001B68184710B503685B680446984708B1E4
:1015500094F84D0010BD000038B504467CF060FCE6
:101560000E4B1D680146E86A02681268904752F007
:1015700051FBEB6A93F89C1051F038FB94F837302C
:101580005BB184F0ADFBEB6AD3F8A030C01AB0F5C4
:10159000FA6F24BF002384F8373038BD942C002024
:1015A00070B50E4605465EF02FF85DF0F1FF10B9FC
:1015B0000124204670BD0A4B93F97E35012BF7D1EB
:1015C0005EF022F8437A002BF2D15EF01DF8847AA7
:1015D000002CEDD1034A314628467CF067FEE8E74F
:1015E000984C0020800F0C08034BD3F8E8350BB95A
:1015F0007CF0CCBB01207047984C00202DE9F043D3
:101600002DED028BC47F91B006460F468CB990F940
:101610000430002B00F00881844B1D68A86A036821
:101620005B6B9847044650B9814A394630467CF096
:101630003DFE204611B0BDEC028BBDE8F083B368DF
:101640004BB933685B6B3946304611B0BDEC028B49
:10165000BDE8F0431847E86AFFF774FF0446002826
:10166000E7D1394630467DF015FDDFF8F8810546B3
:10167000394630467CF042FE08F5B26208F28C53DF
:1016800092ED007AD3ED007AB4EEE77A2840F1EEDD
:1016900010FAC5B209D598F98835032B05D0654AEB
:1016A000394630467CF002FE254608F5A663D3EDA8
:1016B000007AB0EE088AF4EEC87AF1EE10FA0BD593
:1016C00017EE900AFEF720FF5B4ACDE9000139468C
:1016D00030467CF0EBFD002508F23453D3ED007A60
:1016E000F4EEC87AF1EE10FA0BD517EE900AFEF779
:1016F0000BFF524ACDE90001394630467CF0D6FD59
:10170000002508F5A763D3ED007AB8EE087AF4EE69
:10171000C77AF1EE10FA0BDD17EE900AFEF7F4FE31
:10172000474ACDE90001394630467CF0BFFD00252F
:10173000B8F91C35042B07DC052200923946414AD2
:1017400030467CF0B3FD0025D8F8CC0D5DF0B8FF35
:1017500080B198F97E356BB1D8F8CC3DB8F98025C9
:10176000B3F90E309A4205DA374A394630467CF0F2
:101770009DFD0025DFF8F09039463046FFF710FF59
:1017800099F8913F002B48D100EA05042F484FF407
:10179000806100F0FFFE78B1D8F8CC3DB3F90C3091
:1017A000A3F2E24292B2B2F5FA7F05D9284A39464D
:1017B00030467CF07BFD0024264890F82C365BB147
:1017C00000F224602DF09EF9054628B9224A3946D8
:1017D00030467CF06BFD2C4600212E2204A80DF132
:1017E0000C080391ABF08EF9D9F87C0F42463221F8
:1017F00008F09AF9054600287FF41BAFD9F87C0F52
:1018000003689B689847154ACDF80080034639461F
:1018100030467CF04BFD2C460BE7114A39463046EA
:101820007CF044FD0024B1E7012402E7942C002061
:10183000900F0C08A70F0C08CA0F0C08EA0F0C0831
:101840000C100C082E100C084D100C08982C0020C1
:1018500088100C08987C0020B0100C089CC10C0863
:1018600073100C08984C0020986C002070B5054649
:101870000E46FFF795FE3146044628467DF0B6FA3F
:101880002040C0B270BD0000F0B591B005460E46D4
:101890007CF0EAFD0446D8B1102128467CF0DCFA41
:1018A000B0B100212E2204A803AF0391ABF02AF9B6
:1018B00010F0E4F932233A4601210FF0EDFC044622
:1018C00030B9054B00973246102128467CF0CCFAFF
:1018D000204611B0F0BD00BFC4100C0870B505461D
:1018E0000E46B1B990F910408CB116480BF0A4F82F
:1018F000DFED157AB0EEC00AB4EEE70AF1EE10FAA9
:1019000007D4124A012128467CF0D0FC34462046F8
:1019100070BDAB689BB10E4B1B68D86AFFF712FE17
:10192000044630B15CF07EF90A4A042155F0A2FA6F
:10193000EDE731462846BDE870407DF061B80124EE
:10194000E5E700BF982C002000000034D0100C0800
:10195000942C0020E2100C0838B504467DF05AFCA7
:101960000546B0B10C4805F07BFB40B10B49A1F531
:1019700098400FF0D1FD10B1074800F0DFFD204680
:10198000FFF7EAFD0123064984F8373020467DF051
:1019900051FB284638BD00BF982C0020988D0020B0
:1019A00004110C08F8B505460E461746C2B12329A6
:1019B00001D0012914D81E4807F028FC044668B15C
:1019C00000242046F8BD95F91030022B08D05CF0B9
:1019D00029F9184A062155F04DFAF2E7002EF2D007
:1019E0003A46314628467DF0CBFC04460028E7D035
:1019F000114ED6F87C2F06F571639A4203D003F29C
:101A000014702DF0B5FCD6F87C0F03689B6B9847DB
:101A10000A4B83F8F8052846FFF79EFD4FF0FF3389
:101A20000749C6F8AC3F28467DF004FBC9E700BF74
:101A3000982C002014110C08986C0020987C002031
:101A40002C110C08F8B505460E467CF0B1FA104B87
:101A500093F953750446CFB90E48BD212DF01EFCF5
:101A600038B10D4B32464FF4804128467CF0FCF9EA
:101A70003C460848BC212DF011FC38B1074B3246DA
:101A80004FF4804128467CF0EFF900242046F8BD51
:101A9000984C0020BC82002040110C086C110C08EE
:101AA00000207047014800F0F1BC00BF982C0020D6
:101AB00003685B68184700000DF036B965F054B94B
:101AC0005DF0F0BC25F05CBC51F012BA07F0D4BC5C
:101AD0004FF0CEBA0AF0A8BA02F056BE4DF064BE7E
:101AE00014F0CAB861F058B960F0D6BD0CF0DAB99C
:101AF00046F028BE0BF01EB813F01CBC66F0E8BE22
:101B00005DF0F2B95BF0FCBA06F0DCBE04F054BA4A
:101B100009F00ABE0AF0F2B90BF0F4BF0CF07EBA7D
:101B20000AF03EBE0CF016B901F040B900F2845044
:101B300017F06CB907F00ABA90F8F432B02202FB41
:101B4000030390F8382393F8D13012B1012B28BF4A
:101B50000123184670470000034808602C211170CB
:101B600008221A60704700BFB0140C0870B5044614
:101B700000F5C4400C3004F5A855FFF7EDFC00213A
:101B8000284610F001F8802120460CF0B7FC18B16F
:101B900027F07AFA25F00EF804F5005303F5A76252
:101BA00092ED007ADFED216A03F5A662D2ED007AAC
:101BB00067EEA67AD5ED936AFDEEE77A03F55E63EC
:101BC000F8EEE77A04F5C15167EEA67A1831FDEE1A
:101BD000E77A05F5457017EE902A43F8042CD5ED09
:101BE000927AF0EEE77A67EE877A04F5AA46C3EDBB
:101BF000007A2AF061FA94ED467AD6ED1D7AE7EE86
:101C0000007AC6ED1D7AB0EE670A27F0A5FF4FF403
:101C1000001186ED1D0A20460CF070FC20B128460C
:101C2000BDE870400EF0DCBA70BD00BF0000C842D5
:101C3000FFF79CBF10B500F580430446D3F87C0F36
:101C400003689B6B984704F5A04393F8B3353BB901
:101C500030B104F539503830BDE8104081F046BD50
:101C600010BD0000FFF7E6BF38B54FF48011044601
:101C70000CF044FC054620B9012120460CF03EFC46
:101C80000546022120460CF039FC40B115B920462A
:101C900002F020FD04F5A8500EF0A0F901E0002D9F
:101CA000F8D14FF4805120460CF028FC30B104F5F7
:101CB000C3400830BDE8384061F094B938BD000039
:101CC000FFF7D2BF38B54FF4801104460CF016FC74
:101CD0000121054620460CF011FC18B115B920462B
:101CE00002F0F8FC102120460CF008FC60B1204600
:101CF00002F062FD4FF4800120460CF0FFFB18B9A2
:101D000027F0C2F925F052F8202120460CF0F6FB0E
:101D100028B1204602F0C6FD204602F0E1FE4FF455
:101D2000005120460CF0EAFB10B1204602F0C0FE44
:101D3000802120460CF0E2FB28B127F0A5F9BDE890
:101D4000384024F05BBF38BDFFF7BCBF00F58043CF
:101D500000F5C040D3F8A01F64307EF009BF00003A
:101D6000FFF7F4BF10B5044617F040F990F92130A1
:101D70008BB190F8403373B194F9A8355BB1064B41
:101D80001B68DB6A93F89C302BB904F28450BDE8E1
:101D9000104016F053BE10BD942C0020FFF7E2BF98
:101DA0002DE9F843434B1B68DB6A93F89C300446EB
:101DB000002B7CD000F5805898F80938002B76D09D
:101DC00007F024FA002872D004F5005504F50857EE
:101DD00095F84E1338460DF0A5FC002867D004F5A1
:101DE00090763046FFF7A8FE022860D994F81424B4
:101DF0004FF0B00909FB024292ED837AF1EE007ACE
:101E0000B4EEE77AF1EE10FA51D495F84E13384655
:101E10000DF038FFB5F91C3507EE903AB8EEE77AC9
:101E2000B4EEC07AF1EE10FA0CDD94F8143409FB2C
:101E30000343F8EE677A93ED837AF4EEC77AF1EE16
:101E400010FA34DCD8F8F836D5F8DC2D002BB8BF02
:101E50005B4293422BDC08F2FC63D3ED007A9FEDEA
:101E6000166A05F23453D3ED006AF8EEE77A66EEAF
:101E7000866AF4EEE67AF1EE10FA18DC05F55E6398
:101E800093ED007A27EE067AF4EEC77AF1EE10FAB7
:101E90000DD494F81414B5F91E25B02303FB016189
:101EA000384601F58271BDE8F8430DF025BBBDE869
:101EB000F88300BF942C00200000C842FFF770BFD9
:101EC0002DE9F04190F814342D4D00EB03132F68E9
:101ED000D3F8C48100F5907604463046FFF72CFE17
:101EE000474514D0022814D904F58047C5F800806E
:101EF00097F8A43F012B15D817D104F5C045D5F8A4
:101F00000831E3B9D5F80C31CBB905230BE0022831
:101F100010D804F5804393F8A42F5AB1052283F812
:101F2000A42F07E0013B87F8A43F04F5C9501C30FB
:101F300011F024F82046BDE8F04109F09FBD114B97
:101F40001B68D86A03685B68984780460028ECD114
:101F500094F81414B02303FB0161DC31204605F032
:101F6000EFF8D5F8EC300FCB05F1F00605F58875E4
:101F700086E80F0085E80F0087F8A48FD5E700BF3B
:101F8000882C0020942C0020FFF79ABF10B500F594
:101F9000A04300F5805493F8B3251AB1002384F8C8
:101FA00009380AE0D3F80036042B07D100F5BF400A
:101FB000583081F039FE84F8090810BD0123EEE79E
:101FC00010B500F5804400F59E43D4F87C1F103313
:101FD000994200F5A04308D000F59E425432914248
:101FE0001CBF4FF0FF32C3F86C2503F25C52074967
:101FF000116003F5AC63064A1A60FFF7C7FFD4F817
:102000007C0F0368BDE810401B6918470000C842F8
:102010000000C8C2FFF7D4BFF7B500F5A0460446DC
:10202000D6F800368B420D463FD00B1F00F5BF4758
:10203000594207F1580759413846019181F0E4FCB3
:102040000199384681F0E0FC042D02D118486DF06A
:10205000C5FAD6F80036012B18D1032D16D104F598
:10206000C4400C307BF0E6FE40B1204607F0CEF8CD
:1020700020B104F5355034306DF0AAFA2046C6F888
:10208000005603B0BDE8F04002F078BC072DF5D152
:1020900004F55650D6F87C256423052192FBF3F312
:1020A0000830044A54F0E6FEE8E703B0F0BD00BF94
:1020B0000C5A002010120C0838B500F58045044673
:1020C000D5F87C0F03689B6B9847002843D004F534
:1020D000A04393F8F825002A3DD1D5F87C1F04F5DC
:1020E0009E421032914238D193F8AC252AB9012191
:1020F0002046BDE83840FFF78FBFB3F86226152AA7
:1021000029D193F8DC1F11F0010122D1D3F8003658
:10211000072B1ED004F5C04393F952300BB90421AC
:10212000E6E720460AF088FCDFED0F7AB4EEE70A16
:10213000F1EE10FAF3DB04F5BF40583081F0B4FC47
:102140000028ECD004F55650084A0621083054F017
:1021500091FE0721CCE70321CAE704F59E435433DF
:102160009942F8D138BD00BF0000B44234120C08C7
:1021700038B5224CD4F87C2F04F571639A422DEDCA
:10218000028BB0EE408A03D00020BDEC028B38BD3C
:1021900004F58055D5F80036042B25D194F8A53FD9
:1021A00033B11749A1F6DC202DF05AFB0028ECD101
:1021B0009FED147AF0EEC87AF4EEC77AF1EE10FAD9
:1021C00009D49FED110A28EE008ABDEEC88A18EEE8
:1021D000103AC5F87C350D4881F066FC0028D3D054
:1021E000002385F8AF35D0E7B5F86216A4F5804036
:1021F00006F0CAF90028D1D1C6E700BF986C0020CC
:10220000988D0020000000340000C842708C00202F
:1022100010B52DED028B00F5A0430446D3F800362F
:10222000042B0BD104F07AF92046B0EE408A04F07A
:1022300045FA38EE400ABDEC028B10BD00F5C044F3
:1022400094ED4F0AF7E700002DE9F0412DED028BE8
:1022500000F58C658AB00446284612F093F80023F6
:1022600007A904F5A8500793089309930FF018FBEA
:10227000002800F089809DED090ADFED597A04F508
:10228000A04505F28C5393ED007A20EE270ADFED8E
:10229000557AA7EE270A04F5AE401C3004F58046B7
:1022A00083ED000A66F028FD2046FFF705FFD6F80B
:1022B0007C0F03689B6B984795F8B335002B5ED174
:1022C00000285CD095F8F835002B58D1D5F80036A9
:1022D000042B70D09FED448A204604F011FA04F5D7
:1022E000C04204F59E43C2F8C402D6F87C1F2833CE
:1022F00099421CD192F88031CBB904F50053B3F95F
:10230000AC3D002B04DC3949D1F86C1DC9060ED553
:10231000D2F8EC70D2F8F4107F680A33C91B642736
:102320007B438142ACBF5B181B18C2F8C432D5F89E
:102330000036D2F8C412D6F8A82F05912046049290
:1023400003930CF05DFBB6F9B68F07462046FFF706
:102350005FFFCDE9007804F5165605F21C6504F51B
:102360003950F0EE400ADDE90332D6ED0E1A95ED54
:10237000001A0599B0EE480A383080F05BFE0AB0CA
:10238000BDEC028BBDE8F08104F59070FFF7D4FB43
:1023900002280AD994F81434B02202FB034393F8BC
:1023A000402212B193ED8B0A67E7284611F084FEB4
:1023B000B1EE400A61E704F5C2484746103704F51C
:1023C000C1413A467031404615F054FF002881D093
:1023D0003946404615F0E2FFB0EE408A7CE700BF88
:1023E000CDCC4C3ECDCC4C3F00000000984C0020A2
:1023F000FFF72ABF00F5804200F59E43D2F87C2FFC
:102400004C339A421FBF00F5AB4043690B60143058
:1024100014BF01200020704710B500F5804200F580
:102420009E43D2F87C2F4C339A420C4612D000F5D2
:102430004050D0F8B00703681B69984707EE900A30
:102440009FED057AF8EEE77A012067EE877AC4ED12
:10245000007A10BD0020FCE70AD7233C10B500F538
:10246000804200F59E43D2F87C2F4C339A420C46B2
:102470000AD000F54050D0F8B00703685B69984770
:10248000012084ED000A10BD0020FCE730B50546B0
:102490000FC985B06C4684E80F0040F279322146BE
:1024A000284604F0E3FC0C4B03F63872D3F87C3F6B
:1024B00093420ED19DF8001011F0040102D1204684
:1024C00015F0D4FC0548214604F088FD012005B034
:1024D00030BD0020FBE700BF986C0020982C002046
:1024E00000F58040D0F87C0F03689B6C1847000013
:1024F00000F58040D0F87C0F0368DB6C18470000C3
:1025000010B500F5A85300F50050D3F80842146048
:10251000D3F804320B60D0F86C3D9B050BD400F56A
:10252000B760D0ED006AD2ED007A9FED037AE6EE57
:10253000C77AC2ED007A10BD35FA8E3C38B50D4D24
:1025400004462946A5F598400FF0F8F804F58043B5
:1025500005F13C0183F8A50F04F5A85004F5C0442B
:102560000EF084FFD4ED4F7AF1EE677AC4ED4F7A26
:1025700038BD00BF988D002010B5044600F590705E
:102580001FF0DEF82046BDE81040FFF7D7BF00007F
:10259000FFF7F2BF00F50050D0F86C3D194214BFB0
:1025A000012000207047000038B5054B1C682368E7
:1025B0000A461D68034B01462046A847002038BD47
:1025C000942C0020982C002070B52DED028B044631
:1025D000036804F500559B6D9847D5F86C3D1B06C4
:1025E00017D5B5F91C35B5F91E15CA1A0B4402EBFF
:1025F000D27203EBD37352105B1000EE902A00EE00
:10260000103AF8EEE00AB8EEC00A04F5A8500EF051
:10261000EBFC5B4BB5F84E251A7004F5C4455FF032
:102620005BF90C355EF0AAFD00212846FEF7E6FFB7
:10263000544E0123B0712846F3717BF0F1FB28B9A9
:1026400028467CF00BFDB0FA80F04009307104217F
:1026500020460BF053FF20B104F5AE403C304EF065
:10266000B9FD28467BF0DCFBE8B994F8143404F596
:10267000C04504EB031341F28832D3F8C461D5F8A6
:102680008431F31A93420ED904F59070FFF754FA8F
:10269000022808D9C5F88461204604F0E1FC04F55D
:1026A000BF4300229A65B4F9A4301BB9B4F8A23034
:1026B000A4F8A430B4F8A430DFED338A07EE903AE2
:1026C000F8EEE77AB7EE008A88EE270AD4ED2B7A87
:1026D000F0EEE77AF4EEE87AF1EE10FA09D5B4F903
:1026E000A23007EE903AF8EEE77A88EE277A84ED8A
:1026F0002B7AD4ED2B0A27F031F920BB4FF078FC70
:1027000040F27D124FF480114FF02AFC4DF002F997
:102710004CF06AFD04F544503430B0EE408A74F059
:10272000DFFC04F54A50B0EE480A103074F0D8FCD3
:10273000B0EE480ABDEC028B04F54F500430BDE802
:10274000704074F0CDBCD4ED2B7A94ED460AF0EED7
:10275000E77AF4EEE87AF1EE10FA09D5B4F9A2308E
:1027600007EE903AF8EEE77A88EE277A84ED2B7A36
:10277000D4ED2B0A27F0F2F80028BFD0C6E700BF3F
:10278000A02300200D90002000000034FFF71CBFA4
:1027900070B500F5C046044696F95030002B2ADD8E
:1027A00006F034FD38BB04F5C4450C3528467CF0F2
:1027B00055FC00B328467BF033FBE0B183F090FA80
:1027C00004F5A0434FF47A72D3F89C35C01A96F9F9
:1027D0005030534398420ED301221C212846FFF764
:1027E000E1F840B104F55650034ABDE870400621B7
:1027F000083054F03FBB70BD54120C0830B52DEDBD
:10280000028B83B0044601A900F5A8500FF01AF816
:10281000002874D004F5AB4595ED017ADDED017A21
:10282000B4EEE77AF1EE10FA05F1040507D504F5E8
:10283000C4400C307BF0FEFA08B1019B2B6004F51C
:1028400000541820B4F91C35052BB8BF052307EE3A
:10285000903A04F5AE63D3ED006AB4F91E3507EE85
:10286000103AB8EEC77AF8EEE77A37EE077AC6EE96
:10287000870AB6EE007AF4EE470AF1EE10FAC8BF06
:10288000F0EE470A9FED2D7A67EE877A9FED2C7A5E
:1028900086EEA71AF0EE007AB4EE671AF1EE10FA9F
:1028A00048BFB0EE671ADDED017AF4EEC77AF1EEBB
:1028B00010FACCBF86EEA70AB0EE410A27F060F905
:1028C000B0EE408A1F480DF0C7FF90B91E48402166
:1028D000FFF760FE68B11D4BD3F80036012B08D11D
:1028E000F7EE007AB4EEE78AF1EE10FA58BFB0EED8
:1028F000678AB0EE480A03B0BDEC028B30BD04F528
:10290000C4400C307BF096FAB7EE008A0028D9D08C
:1029100046205EF083FAB4EEC80ADFED0D7AF1EEE0
:1029200010FAD8BFB0EE480A87EE800AA8F03EF849
:102930002F209FED081ADFED080ABFE73333333F3E
:1029400017B7D13898410020982C0020987C00209F
:10295000000034428FC2D53F9A99193FF8B504461A
:102960005CF052FE0368DB689847054610B9002505
:102970002846F8BD204606F0D7FA04F580460746FB
:10298000D6F87C0F03689B6B984780B10E4BD3F849
:102990007C0F03685B6B984748B104F5005494F9C9
:1029A000C535002BE3D0032BE1D03D46E0E796F898
:1029B000903F002BDCD004F5005494F98855023D7B
:1029C00018BF0125D4E700BF986C002073B500F54F
:1029D000804202F6C47393ED000AD2F87C2F00F512
:1029E0009D432C339A422BD100F50053D3F8C43DBC
:1029F000B3F90840003C18BF012400F5A04300F5DE
:102A0000435500F58050D3F81466D0F8F82693F8B3
:102A100010363C35B61A5BB10A488DED010A4FF409
:102A20000061FFF7B7FD9DED010A80F00100C3B220
:102A300022463146284602B0BDE870407DF0BCB960
:102A40000024DAE7982C002010B5044605F094FE27
:102A500098B104F5A042D2F8143603F58C415031F8
:102A6000C2F8141604F58051D1F8F8160029BEBF3B
:102A7000A3F58C43503BC2F814362046FFF7A6FF5F
:102A8000BDE8104004205EF0B5B900002DE9F0412A
:102A90002DED048B00F5804800F5005608F6C47350
:102AA00093ED009ADFED378A06F5B76393ED008A60
:102AB00028EE288A00F5A047BDEEC88AD7F8183658
:102AC00018EE102A1A4408EE102A054646205EF039
:102AD000A5F906F5AC63D3ED007AD8F87C0FB8EE13
:102AE000C88A05F59D43A0EE278A2C339842FDEE57
:102AF000C87A17EE904A42D1D6F8C83DB3F90860BB
:102B0000003E18BF012603685B699847C0B9D8F832
:102B10007C0F03689B6B984790B905F5C048D8F8BF
:102B2000BC32022B0CD1284609F0D2FD40B1D8EDC1
:102B30000C7A67EEA87AFDEEE77A17EE903A1CB2AF
:102B400005F5495805F5805508F11408D5F8FC3607
:102B5000E41A97F810363BB10B484FF40061FFF7C9
:102B600019FD80F00100C3B2B0EE490ABDEC048B40
:102B7000324621464046BDE8F0417CF059BE002671
:102B8000C1E700BF0000C842982C002010B50446E1
:102B90000CF082F868B100B200EB4000C0EB00130B
:102BA00000EE103AB8EEC00ABDE8104013205EF007
:102BB00021B92046FFF76AFFF6E7000010B50E487E
:102BC000FFF7CCFEB0B10D4C04205EF027F9D4F82D
:102BD000C40D5CF089FF04205EF00CF913205EF058
:102BE0001DF9D4F8C80D5CF07FFFBDE8104013203C
:102BF0005EF000B910BD00BF982C0020984C00205A
:102C0000F8B52DED028B0446FFF7A8FE002800F072
:102C1000838004F5804704F59D42D7F87C3F3C3221
:102C2000934279D004F59D426432934274D004F506
:102C30009E42083293426FD004F59D426C3293421B
:102C40006AD004F59D427432934265D004F59D42EA
:102C50003432934260D004F50055F6EE008AD5F880
:102C6000C40D5CF001FEB4EEE80AF1EE10FA40DDAE
:102C7000B0EE087AFFEE007AE0EE077AB0EE670A6F
:102C8000D5F8DC2D04F5A04607EE902AD6F81436C8
:102C9000B8EEE77A07EE903AF8EEE77A5142E7EEBF
:102CA000007AFDEEE77A17EE900AC6F8140627F0D0
:102CB00007F8C6F81406D7F87C2F04F59E43303386
:102CC0009A4222D0D5F8C80D5CF0CEFDB4EEE80AE9
:102CD000F1EE10FAB0EE408A21DCFEEE007AB4EE9E
:102CE000E70AF1EE10FA22D5B0EE087AF7EE007A94
:102CF00019E0FEEE007AB4EEE70AF1EE10FABFD565
:102D0000B0EE087AF7EE007AB6E726484FF4805125
:102D1000FFF740FC0028D5D0BDEC028BF8BDB0EE2B
:102D2000087AFFEE007AE8EE077AB0EE678A20466E
:102D300005F022FD08B1B1EE488A05F23453D3ED17
:102D4000006AD6F818369FED186A05F55E6595EDB0
:102D5000007AB5EEC08A07EE903AF1EE10FACCBFD9
:102D600028EE268A27EE488AF8EEE77A66EE866A2B
:102D7000E8EE067A27EE067AFDEEE77AFDEEE66AE1
:102D800017EE903ABDEEC77A16EE902A17EE101A9B
:102D900017EE900AC6F8183626F092FFC6F8180605
:102DA000BAE700BF982C00200000C84270B5044666
:102DB00004F5804582F094FFD5F88C3FC31AB3F533
:102DC000FA6F064603D9D5F87C0F06F0C7FE2E4BE6
:102DD000C5F88C6FD3F87C0F026813689847002100
:102DE000204609F029FEDFED297AB0EEC00AB4EEE4
:102DF000E70AF1EE10FA45D504F5C043D3ED4F7A5A
:102E0000B1EE047AF0EEE77AF4EEC77AF1EE10FA5A
:102E100038D504F58C6011F04FF9F6EE007AB0EE7B
:102E2000C00AB4EEE70AF1EE10FA2BD504F5C85546
:102E300095ED017AF0EE087AB4EEE77AF1EE10FA49
:102E400005F104051ED504F543503C307DF024F80F
:102E500004F5495014307CF09BFD04F54E502C30A5
:102E60007DF0C8FC95ED007AF7EE007AB4EEE77AD3
:102E7000F1EE10FA06D504F554502030BDE870404C
:102E80007DF00EBA70BD00BF986C002000000034C9
:102E900000F5005090F91335012BC3BF00F67860A0
:102EA00090ED290ADFED047A9FED040AC8BF20EEF9
:102EB000270A46205DF09EBF0000C84200000000C7
:102EC0002DE9F8432DED028B00F5804909F6C47316
:102ED000D3ED008A054609F019FA8046D9F87C0F2F
:102EE00003681B6A984705F54E562C3698B1504C2E
:102EF000D4F8D835002B0EDD82F0F2FED4F8D835A8
:102F0000C01A40F6B733984205D8B4F9CC453046DC
:102F10007DF07CFC7CE005F5C04305F5005793F897
:102F2000B13243B1B7F9A435002B04DD05F54053A8
:102F300093F9C23313BBD9F87C3F05F59D452C3579
:102F4000AB426FD00021B0EE680A30467DF0F6F952
:102F5000054604205DF062FF2BB207EE903A07F5BC
:102F6000AB67F8EEE77A97ED007AE0EE077AFDEED0
:102F7000E77A17EE904A444424B2C8E72846012174
:102F800009F09CFB9FED2B7AB7F9A435C0EE077AC8
:102F900005F5A04505F5C46508EE103A55F80C3C5A
:102FA0009FED250AB8EEC88A28EE278A07EE903AE8
:102FB000F8EEE77A67EE807A9FED200A27EE800A26
:102FC000A7F018FBB7F91C35DFED1D7A95ED007AF7
:102FD00020EE270A07EE903AF8EEE77A0021B4EEE9
:102FE000E77AF1EE10FA58BFF0EE477A80EE277AD2
:102FF0003046DFED147AB0EE480AA7EE270AF0EE6D
:10300000680A7DF0F7FABDEEC00A10EE103A1CB265
:10301000BDEC028B20460C49BDE8F84341F2941206
:1030200026F05EBEB8F1000118BF01218BE700BF9A
:10303000987C002000A08C450AD7233C35FA8E3CB2
:103040000AE81C41E02E65426CEEFFFF38B500F542
:1030500040530546D3F8B0070368DB68984701463C
:1030600005F5545020307DF0FDF804B22846FFF7F6
:1030700075FC70B107EE904A05F50055B8EEE70A09
:10308000D5F8D00D5CF030FDBDEEC00A10EE103A60
:103090001CB220460349BDE8384041F2941226F0A4
:1030A0001FBE00BF6CEEFFFF38B590F81434B0229D
:1030B00002FB030393ED837AF7EE007AB4EEE77A2E
:1030C000F1EE10FA054600F5A0441DD5002109F0E7
:1030D000B3FCDFED427AB0EEC00AB4EEE70AF1EEDF
:1030E00010FA11D5D4F80036012B0DD0072B0BD0D8
:1030F000002384F8703504F27454002323602846BA
:10310000BDE8384009F002B982F0EAFDD4F878351C
:10311000C4F87805C31AB3F57A7F84BF002384F816
:103120007035284609F0F2F8D4F80036012B07EE86
:10313000100A2DD0072B2BD0B8EEC77ADFED286A06
:10314000C7EE267A05F50052B2F9682500EE102A7E
:10315000B8EEC00A27EE800ADFED207AB0EEC07A22
:10316000B4EEE77AF1EE10FA14D4002384F8703547
:1031700094F8703505F554502030DBB97CF05AFFD7
:10318000BDE83840174900B241F2941226F0A8BDBC
:103190009FED150A94F87025002AE9D10122934287
:1031A00084F87025E4D0072B1EBF04F2745300226C
:1031B0001A60DDE704F2745494ED007ADFED0B7AC7
:1031C00067EEC77A9FED0A7A67EE877AFDEEE77AB7
:1031D00017EE901A7DF046F8D2E700BF00000034E9
:1031E00000A08C456CEEFFFF00000000E02E654261
:1031F0000000C84270B52DED028B00F5BF46583671
:1032000082B00546304680F07FFB0446E8B905F5FC
:103210000053D3F8C42DB2F9082082B905F5C04295
:10322000D2ED4F7A03F2645393ED007AF0EEE77A31
:10323000F4EEC77AF1EE10FA4CBF012400243046B8
:1032400080F076FB002808BF0024304680F05CFB4D
:1032500028BB05F5A043D3F86C35013319D0F4B978
:103260009FED1A8A2846FFF72BFE07EE900AB8EE6C
:10327000E70A8DED010AD4B915205DF0BBFD9DED87
:10328000010A1A2002B0BDEC028BBDE870405DF06F
:10329000B1BD002CE4D02846FFF706FF02E0284627
:1032A000FFF7D4FE07EE900AB8EEE78ADAE71A20B5
:1032B0005EF042F89DED010A08B9B0EE480A15200B
:1032C0005DF098FDB0EE480ADBE700BF00000000AB
:1032D00010B500F5005303F23452D2ED006ADFED71
:1032E000137A9FED136A03F55E6292ED007A03F69E
:1032F000786366EEA76A27EE277AD3ED2A7A67EE1F
:10330000867AFDEEE66ABDEEC77AFDEEE77A044600
:1033100016EE902A17EE101A17EE900A26F0D0FC3F
:1033200004F5A044C4F8180610BD00BF0000C84250
:10333000A00CB34510B504460BF0E4F8031E2CDBDB
:1033400004F5005191F913259A4226DD04F5A040B9
:10335000D0F80046022C20D001F26C51D1ED007A59
:10336000DFED0E6AD31A66EEE76A07EE102A07EE63
:10337000903AB8EEC77AF8EEE77AD0F8183687EECA
:10338000876A07EE903AF8EEE77AE6EE867AFDEE87
:10339000E77A17EE903AC0F8183610BD0000C84220
:1033A000F8B52DED028B00F5A0459FED440AD5F848
:1033B00014369FED437A07EE903AF8EEE77A04462A
:1033C00067EE807A9FED3F0AF0EEE76AF4EE476A17
:1033D000F1EE10FAC8BFF0EE477A27EE800AA6F0A9
:1033E00049FF26F0EFFAB7EE008AC8EE007A05F240
:1033F0001C6704F50056C7ED007A96F9443553B3BF
:10340000204605F0B9F930BBB6F91C35012BB8BF21
:10341000012307EE903A05F5C462F8EEE77AD2EDA3
:10342000006A86EEA77AB4EEC87AF1EE10FA15D8E3
:1034300040F6C4122449D5F8140626F041FCC5F81C
:103440001406D6F8DC2D40F6C4139A42D4BFC6F851
:10345000DC2DC6F8DC3DBDEC028BF8BDD7ED007A63
:10346000B4EEE77AF1EE10FAF5D588EE070A20EE11
:10347000000AA7F0E9F8DFED157AD5F8140620EE7A
:10348000270ADFED137A20EE270A40F6C413FDEE7B
:10349000C07A17EE904A9C42B8BF1C462246614251
:1034A00026F00EFCC5F81406D6F8DC3DA342D4BFC6
:1034B000C6F8DC3DC6F8DC4DCDE700BF0AD7233C9B
:1034C0000000AA4235FA8E3C3CF6FFFFE02E654232
:1034D0000000C84210B500F540530446D3F8B007C9
:1034E00003681B68984704F50053D3F8DC2D51425C
:1034F00026F0E6FB04F5A043C3F814062046BDE819
:103500001040FFF74DBF00007047000001207047DA
:10351000082070470120704770470000014B93F866
:1035200050057047984C0020034B93F9600D00380C
:1035300018BF0120704700BF984C0020014B93F941
:1035400052057047984C002013B5064BD3F87C0FFA
:103550004B690468009308310EC9646CA04702B03F
:1035600010BD00BF986C002070470000002070471D
:103570007047000038B5254DD5F87C0F03685B68AF
:1035800098470F2834D80F2839D8DFE800F00836DC
:103590000808080808080838363636363636102443
:1035A0001B4B93F8812512B193F880350BB944F089
:1035B0001004184BD5F87C2F9A42A3F1080303D0CE
:1035C0009A4218BF44F01004134991F9C515C1B1CE
:1035D0009A4218D0032902D1104B9A4201D144F0EB
:1035E00040040F487AF01CFC68B144F080040AE003
:1035F000182814BF01241824D2E71824D0E7012486
:10360000CEE79A42EDD144F0010038BD986C00201D
:10361000985C0020E47B0020984C0020A87B0020D0
:10362000A48E002008B5044805F0F0FD00280CBF6A
:103630000120022008BD00BF982C0020F0B52DED20
:10364000028B8BB005460EF019FB4FF48071D0F859
:10365000047290ED828AD0F80C6204461448FEF79A
:1036600099FF30B9134BDFED147A93ED007AA7EE92
:10367000678A2D7C82F034FBD4F81823D4F81C33ED
:10368000D4F814130892099327221C23CDE90032A1
:103690000390079103AA1E21284604978DED058A01
:1036A000069654F01BFC0BB0BDEC028BF0BD00BFC6
:1036B000982C00205052002035FA8E3C2DE9F04322
:1036C0002DED068B424ED6F87C2F06F64C739A42AF
:1036D0008BB077D006F58059A6F5805390F810800E
:1036E000D3F8B077D9F814369FED3A9A07EE903AAE
:1036F000D9F81836B8EEE7AA07EE903A3B68384694
:103700009B68F8EEE79A984707EE900AF8EEE77A9A
:10371000384667EE897A09F29459FDEEE77A2AEE87
:1037200009AA17EE903A1DB23B681B69984707EE4D
:10373000900AF8EEE77AD9ED008A67EE897AA6F565
:103740008040FDEEE77A06F57B6617EE903ADFEDF6
:10375000227AF4EEE78AF1EE10FA58BFF0EE678AAB
:103760001CB202F033FE3B68D6ED00AADFED1B7AF7
:103770005B6908EE100A38466AEEA7AA9847FCEE85
:10378000E88AB8EEC88A18EE903AB72269EE899AAC
:1037900028EE098AADF824301A23CDE900323E2103
:1037A00003AA40468DED03AACDED049A8DED058A5E
:1037B000CDED06AA8DED070AADF82050ADF82240F8
:1037C00054F08CFB0BB0BDEC068BBDE8F08300BF62
:1037D000986C00200AD7233C00FF7F470000C842B6
:1037E00008B502480AF08EFE00B208BD982C0020F1
:1037F00055F036BE37B50D46134840F2EF2203F0C0
:1038000035FB2C7814F004040AD0696803220F48B1
:1038100014F068FA0C4803B0BDE8304002F0EEBC8A
:1038200001AA2146284614F031FB0028F2D0DDED34
:10383000017A9FED077A67EE877A2246FDEEE77AF6
:1038400017EE901AE3E700BF982C0020A88D002007
:103850000000C84210B5054C012384F8833556F0AA
:103860003FF8002384F8833510BD00BF985C00202A
:1038700059F0E6BA2DE9F0412DED028B4FF000082A
:1038800082B0CDE900281E4F9FED1E8A0C461546DA
:10389000B0EE480AB1F90220D7F8C41D4FF47A738C
:1038A000064659F0B5FD0123CDE90053B4F90020D7
:1038B000D7F8C81DB0EE480A30464FF47A7359F075
:1038C000A7FDB4F90420D7F8CC1D9FED0F0A43469D
:1038D0003046CDE9005859F09BFDCDE90058B4F9C8
:1038E0000620D7F8D01DB0EE480A4FF47A73304660
:1038F00059F08EFD02B0BDEC028BBDE8F08100BF37
:10390000984C00200000FA4400007A4438B5C5788D
:103910000B46352D044628BF352535220021184693
:10392000A9F0F0F82A4604F10C01BDE83840A9F0EE
:103930009FB8000010B5074B93F93C2740F24D3477
:1039400040F24D13002A08BF1C4655F011FE2043DB
:1039500010BD00BF987C002010B5044614F0C6FDD1
:10396000204610BD10B50B4C002384F8AF3556F03F
:10397000B1FC54F8842CA4F1F0039A4208D194F8D5
:1039800028362BB904F22460BDE810402BF0C2BEEB
:1039900010BD00BF987C002013B5124C94F84E1354
:1039A00004F500700BF0BEFE78B194F84E1304F5E8
:1039B00000700CF025F940B194F84E1304F5007036
:1039C00002B0BDE810400CF05DB90EF057F901A946
:1039D0000DF038FF18B19DED010A02B010BD9FED4A
:1039E000020AFAE7984C00200000000008B51248CF
:1039F000D0F87C2F00F644739A4216D0B0F9943F69
:103A0000ABB900F5805393F8392582B990F8912F1E
:103A10006AB993F8E93563B9A0F5804005F0F6FB83
:103A200000280CBF0320042008BD0220FCE705206D
:103A3000FAE70620F8E700BF986C002010B5214B8C
:103A400003F64C72D3F87C3F934290B0044636D0D4
:103A500000231D48029314F02FF9014618B91A48A3
:103A600002AA14F075F9247C82F03AF9174BDDEDC7
:103A7000027A9FED177AD3E9462305930023F8EEE7
:103A8000E77A0793089309930A930B930C930D938A
:103A90000E934FF6F853ADF83C300023CDE9030206
:103AA00067EE877A96228DF83E303323CDE90032D7
:103AB000572103AA2046CDED067A54F00FFA10B034
:103AC00010BD00BF986C0020A88D0020988C0020AD
:103AD0000AD7233C10B555F045FF044678B909488C
:103AE00050F8842C80F8AF45A0F1F0039A4206D13B
:103AF00090F828361BB900F224602BF00BFE20460C
:103B000010BD00BF987C00200120704708B5034B12
:103B1000D3F87C0F03685B68984708BD986C002059
:103B200030B587B005460EF0A9F804462D7C82F02A
:103B3000CBF8D4F88422D4F888320492059300217B
:103B40001023CD22CDE900320290039102AA42F661
:103B50000C31284654F0C2F907B030BD30B52DED18
:103B6000028B89B005460EF089F800F55A7393E888
:103B7000070002AC84E80700DDED020A9DED030AB0
:103B80002D7CF1EE600AB1EE400AA6F0C5FD20469C
:103B9000B0EE408A28F076FEDFED0B7A049B0793A7
:103BA00028EE278A0C230122CDE90032A82105AA9C
:103BB00028468DED058A8DED060A54F08FF909B07F
:103BC000BDEC028B30BD00BFE02E6542282938B520
:103BD000054623D007D824292BD0272911D01B290B
:103BE00008D1012413E0432937D008D84029F8D060
:103BF000422928D02846BDE8384059F065BD5329F0
:103C0000EEE7122153F068FB044610B90024204669
:103C100038BD297C13484CF01DFAF8E7162153F003
:103C20005BFB04460028F1D0297C0E484CF0ECFAEE
:103C3000EDE70C2153F050FB04460028E6D028465F
:103C4000FFF78CFFE3E7102153F046FB0446002802
:103C5000DCD02846FFF764FFD9E7017C02487FF0FB
:103C600051FEBEE7D4830020708C0020F0B52DED0E
:103C7000028B05468DB01646B0EE408A0C460029F0
:103C800030D0007C54F0C0F80746287C54F0C0FFC8
:103C900000F121039F4207D2287C0DB0BDEC028BBE
:103CA000BDE8F04053F006BB63690893636A22697C
:103CB000CDF82530236AA069E1680792CDF8293054
:103CC0006222212327680590CDE900320691287CE5
:103CD0000397192303AAC2218DED048A8DF824606D
:103CE00054F0FCF80DB0BDEC028BF0BD70B52E4960
:103CF000D1F87C2F01F64C739A42044652D0A1F5BC
:103D00000055B5F8F635DE0708D5A1F5805393EDDB
:103D10008A0A0122A1F6DC51FFF7A8FFB5F8F635B3
:103D2000980708D52149022291EDE10A204601F5C4
:103D30006071FFF79BFFB5F8F635590708D51C49A8
:103D40000B4693ED000A043903222046FFF78EFF4D
:103D5000B5F8F6351A0708D516490B4693ED000A53
:103D6000043905222046FFF781FFB5F8F635DB065A
:103D700018D5114ED6F80036042B13D10DF07EFF66
:103D8000054606F6D8707FF0EDFD95EDC70ADFED2C
:103D90000B7A014620EE270A20460622BDE8704035
:103DA000FFF764BF70BD00BF986C0020985C0020D6
:103DB00090610020EC610020987C0020E02E65429C
:103DC00070B504460E461DF0F9FC90F8F412B023CD
:103DD00003FB0101DC31204603F0B2F9054698B13E
:103DE0003EB10DF04BFF90F87C3243F0020380F8B7
:103DF0007C3204F5804304F59E44D3F87C0F2834CC
:103E0000A04201D105F0F6FD284670BD73B51646F7
:103E1000019104460DF032FF01990DF07DFB05463E
:103E200098B13EB10DF02AFF90F87C3243F00203C6
:103E300080F87C3204F58043D3F87C0F04F59E4370
:103E40002833984201D105F0D5FD284602B070BD57
:103E500030B5054685B00C46D1E9040126F0FAF8E4
:103E600040B1684613F038FF6A462146284659F0AB
:103E70003FFA08B9022067E0344840F24F32694601
:103E800002F0F4FFD4ED037AF4EE677AF1EE10FA63
:103E900022D69FED2F7AF0EEE77AF4EEC77AF1EEB4
:103EA00010FA54BF012200229DF80030294962F324
:103EB000410368468DF8003014F078F80028D9D115
:103EC0002548694669F02AFC40B94FF0A3FE052257
:103ED00016214FF057FCCDE70022E5E7D4ED017A3B
:103EE000FDEEE77A17EE903ADB0706D41B4B03F69C
:103EF0003872D3F87C3F934225D1194913480222E6
:103F00000AF00EF99DF8001011F0040102D1684684
:103F100013F0ACFF0D48694603F060F894ED020A17
:103F2000B4EE400AF1EE10FA0BD6B5EEC00AF1EE8F
:103F300010FA06DD9DF800100948C1F3400106F0B3
:103F4000C5FD002000E0042005B030BD982C002005
:103F500000000034988D002050500020986C002004
:103F6000D07B002010B52DED028BD1ED017A91EDC3
:103F7000008AFCEEE77A8AB0CDED037A9DF80C104A
:103F800005AA044659F09EF9C8B1DFED0E7A059BEB
:103F9000009368EE277A0022FDEEE77A114617EECD
:103FA000903A06A813F0B8FE23682046D3F8CC3028
:103FB00006A9984700200AB0BDEC028B10BD022074
:103FC000F9E700BF0000C84237B5124DD5F87C0FA5
:103FD00003681B6A0C46984740B9D5F87C2F05F555
:103FE00071639A4202D0042003B030BDD4ED007A50
:103FF000D4ED020A94ED010A0748FCEEE77ACDED14
:10400000017A9DF8041003F049FE0028EBD000204F
:10401000EAE700BF986C0020982C002008B5D1ED8D
:10402000007A9FED087A0848F0EEE77AF4EEC77A56
:10403000F1EE10FA54BF0121002104F097FB00209B
:1040400008BD00BF00000034982C002010B5D1ED51
:10405000007AFCEEE77A17EE903A9CB2012C02D07F
:10406000022C06D084B91148214664F0B3FD00202B
:1040700010BD0F4890F830375B0707D559F0D2FDD7
:104080000C4A052152F0F6FE0420F1E790F91C37A6
:104090001BB959F0C7FD084AF3E7A0F5A04007F0A7
:1040A000F5FF002814BF00200420E1E7B4830020BE
:1040B000987C002028180C0843180C0838B58B8B06
:1040C000C02B05460C4631D8B12B0BD8112B00F074
:1040D0009880142B00F0988021462846BDE838408F
:1040E0005AF0E4BBB23B0E2BF6D801A151F823F0F5
:1040F0005F410108D9400108D9400108D9400108B1
:10410000D9400108D9400108D9400108D940010827
:1041100055410108D940010879410108B74101081A
:10412000D9400108694101084B410108D42B08D04E
:10413000B3F5967F4BD0D02BCED1BDE83840FFF7FA
:1041400085BFBDE83840FFF769BF2146BDE838406C
:10415000FFF77EBE2146BDE83840FFF703BF21468A
:10416000BDE83840FFF730BF94ED000A2948FDF75D
:10417000FFFFF0B100201DE0274C94F8A53FC3B12C
:1041800004F50451A1F6DC202BF0C2FB88B104F544
:104190008053012283F85D2604F571610222A4F5A3
:1041A000804009F0BDFF0028E4D11C4B002283F8B9
:1041B0005D26042038BD184C94F8A53F002BF8D09C
:1041C00004F50451A1F6DC202BF026FBDEE7D1ED4F
:1041D000007A9FED137AF0EEE77AF4EEC77AF1EE0B
:1041E00010FA14D5D1ED017AF0EEE77AF4EEC77A41
:1041F000F1EE10FA0BD50B490222064809F090FFA8
:10420000B8E709490222F8E708490222F5E7022047
:10421000D0E700BF982C0020986C0020987C0020EC
:1042200000000034A87B0020C87B0020C07B002059
:1042300070B5434B03F63872D3F87C3F93428EB08F
:104240000C467BD1CD78272D28BF2725272200219A
:1042500004A8A8F057FC2A4604F10C0104A8A8F011
:1042600007FC059B9DF836400093069B0193E443B1
:10427000079B0293E4B2089B03938DF8364081F0CC
:104280002FFD14F0810F04F08705064601D1802D23
:1042900013D1684627F074FADFED2A7A2A4B20EE14
:1042A000270ADFED2A7AC3F8D06520EE270ABDEE93
:1042B000C00A10EE102AC3F8C42514F0820F01D1F1
:1042C000802D13D1684627F075FADFED1E7A1E4B5C
:1042D00020EE270ADFED1D7AC3F8D46520EE270A09
:1042E000BDEEC00A10EE102AC3F8C82514F0840FE2
:1042F00001D1802D13D1684627F06CFADFED117AD9
:10430000114B20EE270ADFED117AC3F8D86520EEB5
:10431000270ABDEEC00A10EE102AC3F8CC256306AA
:104320000CD5DDED0C7A9FED097A074B67EE877AA5
:1043300003F2DC52C2ED007AC3F8E0650EB070BD46
:10434000986C0020E02E6542987C00200000C84256
:1043500030B51F4C91B0084602A9FFF7D7FAD4F840
:104360007C2F04F638739A422FD19DF83C30072BEE
:104370002BD104F50054D4ED457ADDED056A9FEDAF
:10438000157AF8EEE77AE6EEC77AFDEEE77AC4ED45
:10439000457A59F047FCD4F8EC20D4F8143152682F
:1043A0009FED0D7A9B1A07EE903AF8EEE77A0546F4
:1043B00067EE877A17EE900AFCF7A6F8074ACDE970
:1043C00000010621284652F055FD11B030BD00BF56
:1043D000986C00200000C8420AD7233C5C180C08E7
:1043E00010B51D4B03F63872D3F87C3F9342044658
:1043F00096B008460FD108A9FFF788FA9DF8541027
:1044000003AA204658F05EFF38B959F00BFC134A56
:10441000042152F02FFD16B010BDBDF8503023F02E
:1044200004039BB2002BF6D0DDED0B7A9FED0C7AE6
:10443000039B009367EE877A0022FDEEE77A114630
:1044400017EE903A04A813F067FC236804A9D3F888
:10445000CC3020469847DEE7986C002070180C0896
:104460000000C84230B48D7A4B7A43EA0523CD7AF6
:1044700043EA0543562B04460A461BD008D8522B64
:1044800012D0542B13D02046114630BC59F0EABB51
:1044900003F18073863B23F07F43012BF3D8017C2B
:1044A000064830BC4BF078BF30BCFFF7C1BE30BC13
:1044B000FFF74EBF30BCFFF793BF00BFD48300208F
:1044C00000207047C82070470120704700207047C7
:1044D0000020704790F89C308B4286BF283150F8FE
:1044E000210000207047000090F89C308B4286BF6E
:1044F000283150F821000020704700000320704749
:10450000014B93F84E057047984C002070B5044657
:104510004C4808F08BFA18B1E36A43F40003E362F5
:10452000484808F083FA88B146205CF077FCDFED5C
:10453000467AB4EEE70AF1EE10FA07D8236B43F49B
:1045400000032363636B43F400036363E36A43F490
:10455000F843E3623D4BD3F87C0F03685B689847F0
:104560000138172814D8DFE800F03A420C444242E0
:104570004242133A3A3A3A3A3A13131313131313C3
:10458000133A334A92F880358BB392F881258AB377
:10459000304B93F8D43F012B3DD0022B44D02E4B0F
:1045A0001D68DDB12D4E284696F8BA1D47F0ACFDCA
:1045B000A0B1E36A43F48073E36296F9F4351BB16A
:1045C000236B43F48073236396F8BA1D284647F0A3
:1045D000D3FD18B1636B43F48073636370BDD4E99A
:1045E0000C2342F4E04243F4E0432263636301237B
:1045F00000E00023216B41F480622263626B42F48D
:1046000080606063002BC3D041F4406142F440629B
:1046100021636263BCE7E36A43F48003E362236BD4
:1046200043F480032363BAE7E36A43F48003E3625D
:10463000236B43F480032363636B43F4800363635E
:10464000ADE700BF982C0020000000B4986C00205B
:10465000985C0020987C0020C0900020984C00209E
:1046600013B54FF44470CDE9002113F037FF044631
:1046700028B1DDE9002159F015FD024B23602046E9
:1046800002B010BD701A0C0800207047002070475F
:10469000002070470020704700F5165030307047FA
:1046A00000487047F83F0C0800F58040D0F87C0FB8
:1046B00003685B681847000000F5804300F59E40E2
:1046C000D3F87C3F10301B1A584258417047000005
:1046D0009B20704730B500F5A04303F5C36353F842
:1046E000042CDFED286A07EE902AB8EEE77AD3EDC6
:1046F000007AF8EEE77A85B027EE267A67EEA67A9A
:104700000446002301A900F5A85003938DED017A1A
:10471000CDED027A04F58F550BF088FC04F5485274
:104720002432692128464EF041F904F54E526A219F
:1047300028464EF03BF904F5405393F9C22332B9B1
:10474000D3EDEE7AF5EEC07AF1EE10FA06DD04F55F
:10475000535234326B2128464EF028F904F5545454
:10476000203420467BF0A0FD28B104F130026D21F9
:1047700028464EF01BF90DF081FA0CF0C9FF05B088
:1047800030BD00BF0AD7233C10B54FF4801104465A
:1047900009F0B4FE10B12046FFF79CFF4FF48001F2
:1047A000204609F0ABFE28B124F06EFCBDE81040B5
:1047B00022F0FCBA10BD000030B591B0002300F526
:1047C000A855029302A9002304460DF107022846CA
:1047D0008DF807300DF03CF803A928460CF08CF852
:1047E00008B92E4B03933022002104A8A8F08AF9BF
:1047F000A3238DF8103095238DF8113081F078FACD
:1048000004F5A042CDF81300D2F81436ADF81B30F1
:1048100004F58053D2F81826CDF817104620D3F8A7
:10482000F816D3F8FC36ADF81D10ADF81F20ADF822
:1048300021305CF0F3FA10EE103A1520CDF8233059
:104840005CF0ECFA10EE103ACDF8273004F539534D
:104850009FED137AD3ED377A67EE877A284617EE05
:10486000903ACDF82B30029BCDF82F309DF80730D1
:104870008DF83330039B0D930DF0F0F904F5804370
:104880003022D3F8B83F8DED0E0A04A904F58F50FD
:104890000F934EF0C7F911B030BD00BF2292CA7F0E
:1048A0000000C84230B58FB035220446002168466A
:1048B000A8F028F9A3238DF8003095238DF8013056
:1048C00001238DF8023081F013FA04F5AB4304F5AF
:1048D00040551433CDF803001B68D5F8B007CDF868
:1048E0000710CDF80B3003681B699847ADF80F002F
:1048F000D5F8B00703689B689847ADF811001E48CB
:1049000001F064FDADF81300D5F8B00703685B69EA
:10491000984710EE103AD5F8B007CDF81530036877
:104920009B69984710EE103A04F58041CDF8193094
:1049300001F57B6335221B68CDF81D3004F5C043BB
:10494000D3F81801CDF82100D3F81C01CDF82500CB
:10495000D3F81401D3F8C432CDF82900CDF82D30A6
:1049600004F58F50D1F8A83FCDF8313069464EF0AC
:1049700059F90FB030BD00BF982C002030B587B07A
:104980001622044600216846A8F0BCF8A3238DF83F
:10499000003095238DF8013002238DF8023081F02C
:1049A000A7F904F5A045CDF803002046CDF807107F
:1049B00004F02CFC05F204638DF80B001B680393D4
:1049C000124B1B68D86A90F89C308DF81030036841
:1049D000DB69984795F8E9358DF812308DF81100AC
:1049E00024F052FB23F046FBD5F800368DF8130077
:1049F0008DF81430162295F8EA358DF81530694691
:104A000004F58F504EF00EF907B030BD942C002005
:104A100010B58AB02722044600216846A8F072F833
:104A2000A3238DF8003095238DF8013009238DF8EC
:104A3000023081F05DF9CDF803000420CDF80710B5
:104A40005CF0ECF910EE103A1320CDF80B305CF06E
:104A5000E5F910EE103A4620CDF80F305CF0DEF9A3
:104A600010EE103A1520CDF813305CF0D7F910EEA7
:104A7000103A0320CDF817305CF0E0F910EE103A50
:104A80001A20CDF81B305CF0C9F910EE103ACDF8C1
:104A90001F3004F59F43443327221B68CDF8233091
:104AA000694604F58F504EF0BDF80AB010BD000005
:104AB00013B5044600F58F5001904DF0E5FB0198C9
:104AC0004DF07CFC04F58053019893F910330BB141
:104AD0004DF01CFD204602B0BDE81040FFF798BF26
:104AE0007047000010B500F580430446D3F87C0FF2
:104AF00003685B68984704F50053014693F8D02497
:104B000004F58F504EF04EFA04F5A8500DF002FB5C
:104B100004F59070BDE810401BF0BABE9FED020A8C
:104B2000002245F0BFBE00BF0AD7233C184B70B52A
:104B3000044640F8043B5AF0E7FB164E164B636000
:104B4000542560195AF096FD66513035B5F5557FFC
:104B5000F7D104F555705CF055FD04F27C75FF2328
:104B600084F88C3784F894370C49284646F0AAF824
:104B70000B4B1A6812B10B4881F080F81D600123BD
:104B80002046094984F8C13746F09CF8204670BD9C
:104B9000F83A0020906A0C08A46A0C08C49E0D081C
:104BA0008C9A002068570C088C5A0C082DE9F041AB
:104BB00000F515519AB00D220C3104464CF020FC42
:104BC0000022BE48BE4E272145F0E4FD042100200E
:104BD0005CF0F2FC132101205CF0EEFC4621022087
:104BE0005CF0EAFC152103205CF0E6FC5CF050FA76
:104BF00046F06EFAB34A138843F0040313804FF073
:104C000000080AAF002110223846A7F07BFF0123DD
:104C10008DF830303388ADF8283005A973680B93D0
:104C2000384645F0BFFCC8B19DF91430002B15DDA6
:104C30005AF0EAFC9DF81410036801391B68C9B2E8
:104C4000984758B1051D284645F0F6FB30B9B368C2
:104C5000ADF8183006A9284646F0D8FE08F1060837
:104C6000B8F12A0F06F10C06CCD1974800220DF1BD
:104C70000B0145F0C9F906AD064620B345F0DCFB53
:104C800008BB924B0FCB85E80F0004A9284645F0DE
:104C900089FC002840F03A814FF004088C4B0FCB80
:104CA00087E80F0005A9384645F07CFC28B105A827
:104CB00045F0C2FB08B148F0010803A930468DF861
:104CC0000C8046F051FE834B0FCB85E80F0003A903
:104CD000284645F067FC002846D00998002204A920
:104CE00045F092F9064600283ED045F0A5FB054662
:104CF000002839D19DF80C30013BDBB2032B96BF65
:104D0000754A0346D35C8DF828303046394646F064
:104D10002BFE7248002205A945F076F9064668F098
:104D20003FFF78B168F03AFF90F8302090F82810F3
:104D300090F84830114490F840200A44D34214BF00
:104D40000125002586B130469DF90C8045F074FBA5
:104D500050B91DB1B8F1000518BF012539463046DC
:104D60008DF8285046F000FE04F517500022B7EEEB
:104D7000000A0121283045F095FD04F51650002267
:104D8000B7EE000A0221043045F08CFD01230093A8
:104D9000534A002304F508518E2045F0FFFC94F996
:104DA000DCC9BCF1000F1AD14E4E0FCE3D460FC5E7
:104DB0000FCE0FC50FCE0FC596E80F0085E80F0088
:104DC00062460421384645F0E5FC9FED470A474816
:104DD00046F018FB4648B7EE000A46F013FB0125E3
:104DE00004F50E51434A00950023383140F2051076
:104DF00045F0D4FC04F5165002213830FFF78EFE42
:104E000004F5145003212030FFF788FE04F51450F8
:104E100003212830FFF782FE04F5165003213430B9
:104E2000FFF77CFE04F5165002213C30FFF776FEBA
:104E300004F5145002213430FFF770FE04F51450CD
:104E400002213830FFF76AFE04F514500221303099
:104E5000FFF764FE04F5BF4058307EF0E9FE264AB5
:104E60001368D90709D42549156004F50D5320337B
:104E70000B6004F597531433CB6004F517501F49AA
:104E800002223830012545F0DBFC1D4A0095002345
:104E900004F58F51FD2045F081FC1A4B1A68D207AA
:104EA00005D4194A1D6004F5A15404341460164851
:104EB000012145F0E1FC1AB0BDE8F081C8570C08AB
:104EC000385A0C089C9000208C570C08300D0C08A8
:104ED000400D0C08500D0C08C4570C0897570C08CF
:104EE000847E0C08600D0C0800000000A4570C081C
:104EF000B3570C08F8990D088C2C002000220020D4
:104F0000B80F0D08902C00201822002004A845F0AE
:104F100093FA00283FF4C0AE4FF00C08BEE600BF85
:104F20000020704700207047002070470020704725
:104F30000020704770470000002070470020704735
:104F400084B001A880E80E0004B000207047000083
:104F500000207047704700001020704700487047DD
:104F6000B4660C0800487047C4660C0800207047FF
:104F700070470000012070470120704700207047F3
:104F8000002343608360C3600361436100230376B1
:104F90007047000010B50446FFF7F2FF0023637668
:104FA00010BD0000027E531CDBB2042B037600EB25
:104FB000820288BF002382ED010A88BF0376704712
:104FC00010B50446FFF7EEFFD4ED017A9FED107A9D
:104FD00094ED020A637E77EE877A042B77EE807A6F
:104FE00094ED030A94BF0133052377EE807A94EDA4
:104FF000040A637677EE807A637E94ED050A77EE95
:10500000807A00EE103AB8EEC00A87EE800A10BD32
:105010000000000003F034BE03F03EB803F098BA7D
:1050200003F048B801F088BC01F02CB801F0B8B921
:1050300001F0F8B9FDF7ACBBFDF73EB870B5234BF6
:10504000036000F540530446D3F84407204AC3F8F0
:10505000882508B113F04EFA1E4B236004F5005367
:1050600093F89C2142B9D3F898512DB1284620F0ED
:1050700015FF284613F03AFA04F5A050083078F0EE
:105080002BF904F5985010305DF03AFD04F6E46514
:1050900004F68466B54204D0183D284620F054FB3F
:1050A000F8E70D4BC4F8C83804F6282050F048FF44
:1050B00004F6FC1050F044FF04F65C1050F040FF82
:1050C00004F5136050F03CFF204670BDF04D0C0815
:1050D000AC2A0D08B8080D08E8D10C0838B54C4BBF
:1050E000044640F8043B61F05FFF04F1100010F04B
:1050F00047FA04F168004AF0E5F804F590701AF0F8
:1051000081FF04F58C600EF0ADFF04F2845013F0C3
:10511000F3F904F6C80021F079FF04F5666061F048
:1051200021FD04F5736046F015FF04F58F504DF036
:10513000ADFC04F59750143067F06CFC04F5985002
:1051400010305DF0C5FC04F59A500C3011F078FF7A
:1051500004F5A050083078F0ABF804F5A150043005
:105160004AF072FC04F5A350183063F0FBF804F524
:1051700080530025274A83F89C5404F5A55004F574
:10518000A4531C330C30136041F020FF294604F572
:10519000A8500BF08FF804F5DB50083072F0A6F938
:1051A00004F500502C3075F0B5F804F505500430C6
:1051B00077F0D8F904F50650283077F00DFE04F5A5
:1051C00008500AF0AFF904F50D50203072F070FE6F
:1051D00004F50E50383067F0B9FF04F5115038303F
:1051E00078F002FC04F5005304F5135083F8D05412
:1051F000094D283078F01AFD2B6813B1074880F06C
:105200003DFD2046064945F05DFD2C60204638BD39
:10521000B8080D08F4990020F8900020CC660C081E
:10522000C0070D082DE9F04F2DED028B04469FB00D
:10523000FFF754FFE24B236004F517503830FFF7B7
:1052400075FC04F536503C3004F500557AF0B8F89A
:1052500004F516531633C5F8E43D04F5385006231B
:1052600085F8E83D10305DF045F804F5A853C5F821
:10527000883E0E9304F514574FF4006304F5BF4BBA
:10528000C5F8943E10375A230BF1580B85F8143F9C
:10529000C5F88C7EC5F890BE05F67865C94BC5F893
:1052A0006031C94BC5F86431B7EE008AC74BC5F809
:1052B000683104F54150C5F8CC3185ED578A14307A
:1052C00051F05EF904F5415004F5405604F53959A2
:1052D000203051F055F94FF00008BD4B336709F10C
:1052E000380986F8888009F5FC70FFF749FEB94B4C
:1052F000B949336786F88980484645F0E3FCB74BE7
:10530000C6F890300E9BC6E925390023C6F8C43094
:10531000C6F8CC3004F54255012304F5435086F815
:10532000D4301035283012F0D7FCAD4986F8F8801B
:10533000284645F0C7FC04F5435039463C307AF026
:10534000F5FB04F54950394614307AF053F804F56A
:105350004E5039462C307AF0B3FF2C22414606F5E8
:10536000AA60A7F0CFFB04F554509E49203004F505
:10537000565845F0A7FC08F108089B4BC6F888353D
:1053800008F114007FF0DEFB04F5585304F5575A7A
:10539000243350460F9355F07BFF0F9B0AF1140AFC
:1053A0005345F6D10723C6F848370023A6F84C37F3
:1053B0004FF4CB7013F098F8C6F8440704F55D502D
:1053C00010307FF0BFFB04F55E5014307FF0BAFB65
:1053D000864B1A680AB9C3F80080854BC6F8883531
:1053E00004F55E504FF48051C6F8B057343010F0D9
:1053F000C9F904F56050343043F062F904F56150A6
:10540000343046F0B9FB04F5625008306AF0ECF82D
:1054100004F59D4004F58045243004F0CDFA754B29
:10542000C5F8A43E04F59D402C3004F0C5FA724B3B
:10543000C5F8AC3E04F59D40343004F0BDFA6F4B26
:10544000C5F8B43E04F59D403C3004F0B5FA6C4B11
:10545000C5F8BC3E05F56D63002204F59D40DA6099
:105460009A605A6083ED008A643004F0A5FA654BB7
:10547000C5F8E43E04F59D406C3004F09DFA624BA3
:10548000C5F8EC3E04F59D40743004F095FA5F4B8E
:10549000C5F8F43E04F59E40083004F08DFA5C4BEC
:1054A000C5F8083F04F59E40103004F085FA594BCA
:1054B000C5F8103F04F59E40283004F07DFA564BA5
:1054C000C5F8283F04F59E40303004F075FA534B80
:1054D000C5F8303F04F59E40383004F59E4804F08E
:1054E0006BFA08F144084E4BC5F8383F404604F0CB
:1054F00063FA4C4BC5F8443F04F59E404C3004F031
:105500005BFA494BC5F84C3F04F59E40543005F01A
:10551000FBFFFE2385F8883F052385F8A43F4FF065
:10552000FF3A424BC5F87C8FC5F8808FC5F8ACAF09
:10553000119305F6C4753E4B85ED008A04F59F4036
:1055400004F5A0454FF4007100932246374B1094A8
:1055500048300FF0FDFA05F27C531B4AC5F86CA5E4
:10556000DA600023C5F8C435C5F8C835C5F8CC35B0
:10557000C5F8D035C5F8D435C5F8D8350323C5F8F6
:10558000003605F21C6383ED008A2A4BC5F84436C9
:1055900004F5AC48284BC5F84C364046274BC5F8B7
:1055A0005436C5F84046C5F84846C5F850466830F8
:1055B00012F092FB04F5AD40043012F08DFB3FE099
:1055C000F04D0C08000080BF0000B4420000B4C2DF
:1055D00038670C0848670C0818DB0D088CD80D08D4
:1055E00034D80D08D0D20D08AC2A0D084094002004
:1055F0004C1B0C08F4700C08D8740C08C0760C080E
:10560000486F0C08FC710C0880720C0868710C085B
:1056100078700C08F86F0C0860740C0870730C0834
:10562000FC720C0870670C08EC730C08155001082C
:1056300020180C08195001081D50010821500108BC
:1056400004F5AD40203012F047FB774BC5F8B43677
:1056500008F1BC00A5F8B8A612F03EFB08F124083A
:10566000724B7349C5F818A74046C3F8008045F04F
:1056700029FB4FF6FF73A5F8603604F5AE406D4B7D
:105680006D49A5F87CA61C30186045F01BFB04F59D
:10569000AE403C304BF0A8FA684BD6F8B0271294D5
:1056A000CDE91334664BCDE91534664BCDE917349B
:1056B000654BCDE91934654BCDE91B34644B1D9323
:1056C0001EA911E903000CAB83E80300DDE91A0110
:1056D0000AAB83E80300DDE9180108AB83E80300A7
:1056E000DDE9160106AB83E80300DDE9140104AB34
:1056F00083E80300DDE9120102AB83E8030004F54F
:10570000C0464146CDE900274B460E9A584604F55F
:10571000C0487EF095F808F164084E4B736608F1B6
:105720003C0012F0D9FA4C49404645F0CBFA4B4BBD
:105730001F6817B14A4880F0A1FAC3F80080494BAE
:1057400073660E9B86F8687003F51B7304F5C14001
:10575000C6F8EC3086F86D7086F89170703012F0F3
:10576000BBFA04F5C24012F0B7FA04F5C24010309B
:1057700012F0B2FA1C22394606F59070A7F0C2F971
:1057800004F5C44804F5C34008F10C0808305DF086
:10579000EDFA404678F004FB334B3449C6F80C323E
:1057A000404645F08FFA324A3249116004F5C4434D
:1057B00044334FF0140CB8B20CFB00120137127CCA
:1057C000002AF8D12C4A10802C4A17680FB12C48B7
:1057D000B1E704F5C4404830136078F0CBFA294BA8
:1057E000C6F84832284BC6F85832642386F85C3233
:1057F000264BC6F8903204F5C440254BC6F89432C7
:105800002449583045F05EFA234BC6F858322046FA
:105810000123C6F8B87286F8C07285F8AC351FB09F
:10582000BDEC028BBDE8F08F0000FFFFDC8F002095
:1058300044DF0C08FC990020F4400D0825500108B5
:10584000295001082D500108315001083550010838
:105850003950010820670C08B0D60D0810A20020AE
:10586000E0660C08C86A0C08C8110C08A0110C08E6
:10587000B09000203C5C0C08AC90002068900020A8
:10588000FC660C0808120C0858670C08D07A0C0843
:10589000287B0C0818320D08A87C0C0810B57FF086
:1058A00031FD064C064B18602046FFF7BBFC204636
:1058B000044A0549BDE81040A4F0B6BB982C00206E
:1058C000942C002058EF00203D5001080069C0F3DF
:1058D000401070470F299DBF302303FB010050305B
:1058E00000207047014B93F995057047984C0020B4
:1058F000014BD3F8D00D7047984C002008B50368D1
:105900009B68984730B9044B93F8960FB0FA80F033
:10591000400908BD0020FCE7986C002008B5044849
:1059200006F010FE10B9034B93F8900F08BD00BFAE
:10593000982C0020986C0020022A10B50C4605D146
:10594000BDE810400948352208F0C6BC084BD3F822
:105950007C0F03685B689847A04205D159F054FE5C
:10596000BDE8104059F0DABD10BD00BF982C0020F2
:10597000986C0020012910B50C4614D0022907D0DC
:10598000D1B90E4BC3F8B81258F04CF90C4A05E0E7
:105990000A4BC3F8B81258F045F90A4ABDE810405E
:1059A000062151F067BA58F03DF9074A062151F037
:1059B00061FA024BC3F8B84210BD00BF988C0020BA
:1059C00087680C085C680C0870680C08012902D014
:1059D000022900D011B9024BC3F8BC12704700BFB6
:1059E000988C0020622910B400F3888047291ADCC3
:1059F000402900F0958008DC162951DC032904DDDC
:105A00004F4B01248C40234053B95DF8044B5AF0AE
:105A1000CDBCA1F196040123A3404A4C2342F4D00B
:105A20005DF8044B7047A1F148031A2BEDD801A48F
:105A300054F823F0215A01080B5A01080B5A0108A7
:105A40000B5A01080B5A0108215A01080B5A010888
:105A50000B5A01080B5A01080B5A01080B5A01088E
:105A60000B5A01080B5A01080B5A0108175B010871
:105A7000175B0108175B0108215A01080B5A01083E
:105A8000175B0108215A01080B5A01080B5A01083B
:105A9000215A0108215A01080B5A0108215A01080C
:105AA000A1F12703112BB0D8112BAED801A454F8C3
:105AB00023F000BF215A01080B5A01080B5A0108B4
:105AC0000B5A0108215A01080B5A01080B5A010808
:105AD0000B5A01080B5A01080B5A01080B5A01080E
:105AE0000B5A0108215A0108215A01080B5A0108D2
:105AF0000B5A0108215A0108215A0108B02904DC77
:105B0000952986DC6B2980D18AE7A1F1D003022B8D
:105B10003FF67BAF84E75DF8044B00235AF018BCD6
:105B2000094B012283F8B422A3F58043D3F8CC0DAE
:105B300000283FF475AF5DF8044B642159F0AABD0D
:105B400010004100A1008004988C002038B50B465D
:105B5000622B0446114600F39580472B13DC382B4B
:105B60007ADC262B4CDC102B00F0B680162B00F0D4
:105B70000781042B00F0C7800A4620461946BDE87D
:105B800038405AF051B9A3F148021A2AF4D801A0BA
:105B900050F822F0E15C0108795B0108795B0108AB
:105BA000795B0108795B01080B5D0108795B0108ED
:105BB000795B0108795B0108795B0108795B010871
:105BC000795B0108795B0108795B0108175D0108C1
:105BD000575D0108795B0108795D0108795B01086F
:105BE0005F5D0108115D0108795B0108795B0108BF
:105BF000C75C01088D5D0108795B0108EF5C010855
:105C0000A3F12702112AB7D801A050F822F000BF53
:105C1000C75C0108795B0108795B0108795B0108C1
:105C2000CB5C0108795B0108795B0108795B0108AD
:105C3000795B0108795B0108795B0108795B0108F0
:105C4000015D0108E95C0108795B0108795B0108E5
:105C5000FB5C0108F55C0108402B8DD1931E594275
:105C6000644C594184F8B31257F0DCFF624A94F84F
:105C7000B312624B002908BF1346614A062151F056
:105C8000F9F820E09B2B00F08E8007DC6B2B00F0F6
:105C90009480962B7FF470AF07211EE0AD2B7AD055
:105CA0000CDC9D2B7FF468AF0124002A00F081807A
:105CB000022A5BD14F4B83F8B24257E0A3F1D002E6
:105CC000022A3FF659AF012450E08A1E4D4B514243
:105CD000514183F8891FF6E70A21FFF72DFEF2E70D
:105CE0000A4601212046F8E70A460421FAE70A4657
:105CF0000321F7E70A460C21F4E70A460F21F1E7F2
:105D00000A460021EEE70B21E7E70A460D21E9E705
:105D10000A460521E6E7374CD1B102290DD101230E
:105D200084F8B032A4F50053D3F87C0F03685B6AA3
:105D3000984710B1344800F08DFD57F073FF334A97
:105D400094F8B012324B002908BF1346314A95E748
:105D500084F8B012E6E72046FFF70CFEB3E7012413
:105D600031B1022902D12C4B83F84C43204638BD77
:105D7000294B83F84C13F9E72046FFF727FEA2E7EB
:105D8000022AA0D1204806F081F99CE759F03CFC9A
:105D900059F0C4FB97E7022A95D19FED200A1A48D3
:105DA000FCF7E6F98FE7022A8DD1174806F0D8FAFA
:105DB00089E7104B83F8B222D8E7022A14D1114D9B
:105DC000D5F87C0F0368DB6B9847044628B10121A6
:105DD000A5F5804002F0CAFCC8E757F023FF104A3F
:105DE000042151F047F86EE70748002102F0BEFC9D
:105DF00069E700BF988C00209C680C0883500C0851
:105E0000A4680C08986C0020982C0020DF3B0C083C
:105E100040750C08B4680C08984C00200000000085
:105E2000C7680C0810B5084CD4F87C0F03689B6B4E
:105E3000984738B9D4F87C0F04F64C74001B18BF8F
:105E4000012010BD0220FCE7986C002008B502215B
:105E500003205BF0FBFA022108465BF0F7FA012110
:105E600004205BF0F3FA022115205BF0EFFA132017
:105E700002215BF0EBFA124806F0D8FDA8B1002130
:105E800046205BF0E3FA002149205BF0DFFA0021B5
:105E90004A205BF0DBFA002101205BF0D7FA0021F9
:105EA000BDE8084008465BF0D1BA012146205BF00E
:105EB000CDFA012149205BF0C9FA0121E8E700BFD2
:105EC000982C002002490348052208F029B900BF98
:105ED000A87B0020982C002038B5304B01241C7082
:105EE00090F90A302B2B0CD12D487DF09FFE2D48C8
:105EF00007F0E4FEBDE838402B4801220921FBF7FA
:105F000051BD284D9FED290AD5ED460A6421032095
:105F10005BF066F8D5ED460A9FED240A6421022065
:105F20005BF05EF89FED220A03205AF063FF9FEDBD
:105F3000200A02205AF05EFF9FED1E0A04205AF04C
:105F400059FF9FED1C0A15205AF054FF13209FEDB6
:105F5000190A5AF04FFF284606F068FDA0B100214B
:105F600046205BF0A1FA002149205BF09DFA002158
:105F70004A205BF099FA002101205BF095FA00219C
:105F800008465BF091FAB2E7214646205BF08CFAB6
:105F9000214649205BF088FA2146E9E7A0940020D9
:105FA000708C0020982C0020A48E0020000000009F
:105FB0000000C84200A08C4500F58040D0F87C0F5E
:105FC00003681B6C1847000000F5165393ED0D7A1B
:105FD00000F5C040B5EEC07AF1EE10FA03F13403DB
:105FE0005DBFD0F8EC30DFED086AD3ED017AD0F870
:105FF00004015FBFF8EEE77AE7EE267AFDEEE77A76
:1060000017EE900A704700BF0000C84200F500502C
:1060100090F8F40528B141F00101084214BF0120B5
:106020000020704713B50446FFF7F0FF58B104F5A0
:10603000005393F8EC1DC90705D503F6086393EDEB
:10604000000A02B010BD22B904F5C04494ED4F0A15
:10605000F7E704F5A04393F8D43F022BF4D104F5FD
:10606000AE40012201A93C304AF044FF0028EBD0A9
:106070009DED010AE5E7000000F5C04393F82821F3
:10608000FFF7D0BF10B54B68516800F5C0448B4294
:10609000D8BF0A46D4F82001CCBF1A46194623F0CF
:1060A0000FFEC4F8200110BD10B504464E4867F03D
:1060B000A9F910F0080217BF4C4BDFED4D7A93EDB4
:1060C000F17AD3EDF37A1FBF77EE877A9FED497AA5
:1060D000012267EE877A10F0010317BF434B9FED53
:1060E000447AD3EDF36A93EDF07A1CBF37EE667A0B
:1060F000DFED406A04F5165118BF27EE267AD1ED80
:106100000F6AF5EEC06A18BF0123F1EE10FA34DD14
:10611000394A9FED386AD2ED006A66EE866A01223E
:10612000F4EE676AF1EE10FA58BFF0EE667A04F505
:10613000C04090F8281129B373B1D0ED4B6AF8EE46
:10614000E66AF4EEC76AF1EE10FA58BFF0EE476A5D
:10615000FDEEE66AC0ED4B6A9AB190ED4B7AB8EE6F
:10616000C77AB4EEE77AF1EE10FAD8BFB0EE677AEC
:10617000BDEEC77A80ED4B7A03E0002AD7D1002B21
:10618000D5D110BDB3B1D0F8EC30D3ED016AF8EE43
:10619000E66A76EE876A90ED487AB8EEC77AF4EE52
:1061A000C76AF1EE10FAD8BFB0EE667ABDEEC77AD4
:1061B00080ED487A002AE4D0D0F8EC3093ED017AF3
:1061C000B8EEC77A77EE277A90ED487AB8EEC77ABC
:1061D000F4EEC77AF1EE10FA58BFB0EE677ABDEE72
:1061E000C77A80ED487ACCE750500020984C0020C8
:1061F000000000000000C8425452002000F5C040DA
:106200000023C0F82431704773B5164604460023B6
:106210006A463046009311F04DFE48B1DDED007A3C
:106220009FED277A67EE877AFDEEE77A17EE900A00
:1062300004F5C045C5F8240133785B0718D595F8F7
:106240002831ABB104F5AE40012201A93C304AF03F
:1062500051FE68B1D5ED4B7ADDED016A9FED187AFC
:10626000F8EEE77AE6EEC77AFDEEE77AC5ED497A11
:1062700004F5A043D3F80036042B1FD004F50054D6
:10628000B4F9EE25002A16DDD5F824319FED0D7AFC
:1062900083EAE371A1EBE37107EE901AF8EEE77A77
:1062A00067EE877A07EE102AB8EEC77AF4EEC77A5F
:1062B000F1EE10FA02D50023C5F8243102B070BD0A
:1062C0000000C8420AD7233C37B50B785A0704466A
:1062D0000D461DD500F5AE40012201A93C304AF023
:1062E00009FEA8B1D5ED017A2B78DFED1B6AF8EE37
:1062F000E77ADB0767EEA67A19D59DED017AB4EE51
:10630000E77AF1EE10FACCBF0120002003B030BDD7
:106310002B78D5ED017A13F0010FF8EEE77A04F54A
:10632000C0440FD194ED417AB8EEC77AE7E704F59F
:10633000C044D4F8EC3093ED017AB8EEC77AE7EEBA
:10634000667ADAE7D4F8EC3093ED017AB8EEC77AE2
:1063500077EE877AE6E700BF0AD7233C00F50053C3
:1063600000F58042B3F99E35D2F87C2F00EE103A4A
:1063700000F59E4310339A42B8EEC00A0ED100F5E4
:10638000A040D0F80036042B02D090F8AD352BB1E8
:1063900000F6D870D0ED007A30EE270A7047000082
:1063A000014608B501F5C041FFF7D8FFD1ED417AAC
:1063B0009FED057AF8EEE77AE0EE477AFDEEE77AB0
:1063C00017EE900A08BD00BF0000C84237B500F5BF
:1063D000C045044695F82831DBB100F5AE400122F6
:1063E00001A93C304AF086FD98B1D5ED4B7AD5ED48
:1063F0004C6A9FED0B7AF8EEE77AE6EE877ADDEDF0
:10640000016AE6EEC77AFDEEE77A17EE900A03B06E
:1064100030BD2046FFF7C4FFD5F82031181AF6E743
:106420000000C842014608B5FFF798FF01F5C041DA
:10643000D1ED4F7A37EEC00ADFED047A20EE270A5D
:10644000FDEEC07A17EE900A08BD00BF0000C842FA
:10645000F7B5044600F5C2400546103529460190BF
:1064600011F09CFF04F5A04704F5C14607F29453D0
:1064700070362A46314683ED000A019811F0C4FEB9
:1064800007F5B367DFED230A87ED000AB7EE001AC0
:10649000762023F075FB04F5395383ED7F0A2046FF
:1064A000FBF70AFE04F58043D3F87C0F03685B68B2
:1064B00098470B280DD008D80A2811D004F5C044FD
:1064C0000023C4F8243103B0F0BD0E38C0B2012857
:1064D000F4D829462046FFF7F7FE0028EED011E059
:1064E00029462046FFF7F0FE30B90B484FF48041B3
:1064F000FCF750F80028E1D12046FFF793FFB0F5F4
:10650000FA6FE6DD2A463146204603B0BDE8F0408A
:10651000FFF77ABE00000000982C002010B52DED8A
:10652000028B00F5C043D3ED457A93F81031DFEDCF
:106530001D8AB8EEE78ADA0728EE288A82B0044678
:1065400009D400F5805202F5EE62D2ED007AF8EE41
:10655000E77AA7EEE88A5B070FD504F5AE40012283
:1065600001A93C304AF0C6FC38B19DED010A30EE7D
:10657000480A02B0BDEC028B10BD204604F58054E1
:10658000FFF70EFF04F5EE6393ED000A07EE900AA5
:10659000B8EEC00AF8EEE77A28EEC00AA7EEA80A1D
:1065A000E5E700BF0AD7233C38B52DED028B00F597
:1065B000804200F59D43D2F87C2F6C339A4204460A
:1065C0004DD100F58053D3F8005700F50053B3F9CF
:1065D000EC35002B66DD04F5C85292ED017AF7EE3A
:1065E000007AB4EEE77AF1EE10FA5BD404F53A5291
:1065F000D2ED087AF6EE006A67EEA67A87EE871A81
:10660000B5EEC01AF1EE10FA4CD907EE905A9FED94
:10661000288AB8EEE70A07EE903A04F5AE4004F592
:10662000C044F8EEE70A20EE080A3C304AF06EFD5E
:10663000D4F824319FED1F1ADFED1F0A002BBCBFD9
:1066400007EE903AF8EEE77A4FF42970B8BFA7EE5C
:10665000880ABDEC028BBDE8384023F091BA05F002
:10666000ABFBF8B904F54053D3F8B00703681B69D6
:10667000984704F50053DFED100AB3F9EC3501EE4D
:10668000103A04F5AB4393ED050AB8EEC11A05467E
:1066900040F27F2023F074FABDEEC00A10EE103AEB
:1066A0001BB296E7BDEC028B9FED030A38BD00BF1D
:1066B0000AD7233C00007A440000000010B50446CD
:1066C0007FF00EFB04F50053D3F8002E801A41F240
:1066D000883290420FD802212046FFF797FC50B134
:1066E00004F5A044D4F80026042A04D103F6F45398
:1066F00093ED000A10BD9FED010AFBE700000000CA
:1067000030B52DED028B00F5C045DFED278A95F8F9
:10671000283183B004465BB3D5ED4B7A9FED230A55
:10672000F8EEE77A00F5AE4027EE800A012201A9D3
:106730003C304AF017FCD8B12046FFF735FFDDEDBD
:10674000017A85ED4C0A37EE800A20468DED010A6C
:10675000FFF7B4FFDDED017A30EE270A20EE280ABC
:10676000BDEEC00A10EE100A03B0BDEC028B30BDC6
:10677000D5F8EC20D5F8203152689B1A08EE103A73
:106780002046FFF7EBFDB8EEC88A2046A0EE288A27
:10679000FFF794FFBDEEC88AB8EEC88AA0EE288A3B
:1067A000BDEEC80ADEE700BF0000C8420AD7233C9E
:1067B00010B500F580430446D3F87C0F03685B6A8C
:1067C000984718B104F5C04494F8B00210BD000019
:1067D00038B500F5C0440D46D4F820310B44C4F858
:1067E000203194F828313BB1FFF7E2FF20B9D4F80B
:1067F0002C112944C4F82C1138BD000030B500F527
:106800000050D0F8E825D3070FD4094B08201D7895
:106810005C688D4204D1224214BF0120002030BDAB
:10682000013803F10803F2D1F9E70120F7E700BFCF
:10683000186B0C0810B500F580430446D3F87C0FA4
:1068400003685B68984701462046BDE81040FFF7A3
:10685000D5BF000037B500F5C0440546D4F8043173
:10686000C4F820310023C4F82431FFF7E3FFD0B18E
:1068700005F5AE40012201A93C304AF03BFB90B146
:106880002846FFF795FF70B9DDED017A9FED087A94
:1068900067EE877A0123FDEEE77A84F82831C4EDAC
:1068A0004B7A03B030BD002384F82831F9E700BFEC
:1068B0000000C84238B504460D46FFF7BBFF30B1B3
:1068C0000321284611F0D2FA80F00103D8B204F572
:1068D000C04484F8290138BD73B500F5C0444A6846
:1068E000C4F820210B780D46D90741BFD4F8EC300D
:1068F0005B689B18C4F8203194F82931064623B10F
:1069000000F5C2411031FFF7D5FF2B785B070FD59B
:1069100006F5AE40012201A93C304AF0EBFA38B14D
:10692000012384F828316B68C4F82C3102B070BDA3
:10693000002384F82831F9E7F0B52DED028B0446E9
:1069400083B004F5C0450E468DED010AFFF7C4FF84
:10695000DFED340A9DED010A40F24310B7EE001A54
:1069600023F00EF9D5F824315B4207EE903AF8EEA9
:10697000E77A04F5175767EE807A2046FDEEE77A4E
:10698000B0EE408A17EE901AFFF722FFD7ED0C7A8F
:10699000F5EEC07AF1EE10FA07F130073EDDD5F8DA
:1069A0002431002B3ADD2046FFF710FD07EE900A58
:1069B000DFED1D6AB8EEE77AD7ED007A67EEA67ACA
:1069C000B4EEE77AF1EE10FA28D531462046FFF70B
:1069D00083FF324604F5C2412046FFF715FCD5F887
:1069E00024315B4207EE903AF8EEE77A204667EEF4
:1069F000887AFDEEE77A17EE901AFFF7E9FEB5EE1A
:106A0000C08AF1EE10FA09DDD5ED497AB8EEE77AE1
:106A1000C7EE087AFDEEE77AC5ED497A03B0BDEC22
:106A2000028BF0BD000000000000C8C2F0B500F508
:106A3000C04487B094F8103103F00503052B0746D6
:106A40000BD04BF0D5FA4FF4AE724FF480114BF0EF
:106A500087FA0025284607B0F0BD1E486A46032184
:106A600011F014FA0028F4D01B4801AA032111F0F8
:106A70000DFA05460028ECD0184BDFED190A93ED0E
:106A8000000A40F26D10B7EE001A23F079F804F511
:106A900088730FCBB0EE401A02AEDFED111ADDEDB8
:106AA000010A9DED000AB7EE002A86E80F0022F0E9
:106AB00099FFDFED0C7A20EE270A3046FDEEC07A12
:106AC000032217EE901A11F00DF931463846FFF700
:106AD00003FFBFE7888D0020A88D002030820020B2
:106AE000000000000000C842F7B50E46022104462F
:106AF000FFF78CFA68B304F5A045D5F80036042BEF
:106B000027D12046FFF796FE18B304F5AE473C3771
:106B100001236A4604F5C24138464AF0D5F8C0B1AF
:106B200004F5C241012301AA103138464AF0CCF8DD
:106B300078B19DED017ADDED007A77EEC77A96EDBA
:106B4000007A37EE277A05F5B76586ED007AC5ED50
:106B5000007A03B0F0BD0000F0B52DED048B00F518
:106B6000005489B000F5736694F8BA1D0391054688
:106B7000304645F0BFFA03990746304645F0CCFA57
:106B8000042F0399B0EE408A1FD1002305A88DED94
:106B9000050A0693079325F061FB05A905F5C15089
:106BA00023F07EFADFED9A7A8DED050AB4EEE71A4E
:106BB000F1EE10FACDED060A8DED071A05DB05F5AD
:106BC000805393F87C37DF070CD494F8EC3D002217
:106BD00062F3000384F8042E84F8EC3D09B0BDECA8
:106BE000048BF0BD94F8EC3D98075CBF43F00203C2
:106BF00084F8EC3D04F6086758BF04F55F6305F5BB
:106C0000385158BF83ED008A083187ED001A2846B5
:106C1000FFF76AFF94F8043E092B00F2898004F61E
:106C20000C63D3ED000A9FED7B9AB0EE480A22F088
:106C300095FE00BB04F55F6394F8BA1DD3ED008A9E
:106C4000304645F087FA07EE900A9FED737AF8EE2A
:106C5000E77A78EEC88A67EE877AF0EEE88A67EE20
:106C6000897AF4EEE78AF1EE10FAC2BF94F8043E96
:106C7000013384F8043E04F60C6394F8BA1DD3ED96
:106C8000008A304645F066FA07EE900AF8EEE77A99
:106C90009FED627A67EE897A78EEC88A67EE877A26
:106CA000F0EEE88AF4EEE78AF1EE10FA02DD002356
:106CB00084F8043E04F60C6383ED008A94F8EC3DFE
:106CC000DA078BD52846FFF729FC04F6086393ED15
:106CD000008A05F5C04330EE488A93F82831002B2E
:106CE0004CD005F5AE40012205A93C304AF002F92E
:106CF000002849D17EF0F4FFD4F8002E41F288310B
:106D0000821A8A42034604F6F45204F6F85144D932
:106D100082ED008A284681ED008A0221FFF776F98C
:106D200018B105F5BF456A6E2A66C4F8003E55E7FE
:106D300094F8EC3D43F00103590784F8EC3DB9D4D5
:106D400005F5A042D2F80026042AB3D10221284634
:106D5000FFF75CF90028ADD043F0040384F8EC3D64
:106D60003868F9F7D1FB05F556560836CDE900012C
:106D70002B4A0621304650F07DF89BE72846FFF766
:106D800059FD0028ADD1B5E704F6086393ED000A7C
:106D90009DED058A38EE408AACE79FED200A92ED22
:106DA000007ADFED207A28EE008AA7EE278A82EDAE
:106DB000008AC4F8000ED1ED007A38EE678AF3EE4F
:106DC0000E7AB0EEC88AB4EEE78AF1EE10FA7FF7D9
:106DD00005AF94F8EC3D5B070ED504F6086405F5A5
:106DE00056562068F9F790FB0836CDE900010E4AA7
:106DF0000621304650F03EF805F537502422002198
:106E00002C3009B0BDEC048BBDE8F040A5F07ABE93
:106E1000000000340AD7233CCDCC4C3DCDCC4C3EB9
:106E2000D86A0C08CDCC4C3FF56A0C0838B52DED6E
:106E3000028B0D460446FFF771FB002320462B70A2
:106E4000B0EE408AFFF73AFC0221204638EE400AB5
:106E5000FFF7DCF828B104F5005494F8EC0D00F0CD
:106E60000100BDEC028B287038BD000070B50B78B6
:106E700003F00503042B05460C46164615D105F50F
:106E8000C0454BF0B5F8B2B24FF480114BF068F842
:106E9000D5F8EC20636852689B1A13F5FA7FC8BFD7
:106EA0006360237843F00103237070BDF8B500F5EB
:106EB000805300F5A047D3F87067D7F8BC55B542AA
:106EC000044619D00E4A1268D26A92F89C209AB1F0
:106ED00000F5C241751B25221031FFF7C7FF07EEF1
:106EE000905AB8EEE70ADFED077A04F5395020EE44
:106EF000270A38307CF02CFAC7F8BC65F8BD00BF13
:106F0000942C00200AD7233C2DE9F04100F5A04E37
:106F100000F5C0449EF8AF8505468C4600F5C24694
:106F200004F1F007B8F1000F4ED004F588730FCBD1
:106F300087E80F0001238EF8B0359CE80F0004F5B8
:106F4000887787E80F00D4F8183105F5C247103765
:106F500093B9D4F81C317BB9D4F80831D4F8142192
:106F6000C4F81831D4F80C31C4F81C3122B9D4F863
:106F70000411384610F0B6FE394628222846FFF79D
:106F800075FF94F8101111F0040102D1384610F089
:106F90006DFF05F5C1413A467031304611F06AF98E
:106FA00020B196E80F00F03484E80F00284604F082
:106FB0009BFB2846FFF74CFA284604F0C1FE284602
:106FC000BDE8F041FEF7F8BF96E80F0087E80F0034
:106FD00001238EF8AF358EF8B085AEE7F8B500F531
:106FE00000530446B3F94635002B0D4635DB0B78CC
:106FF00013F0020F14BF4FF0FF33012304F5C04616
:1070000006F1F00786F8C83004F5C2430FCB87E8D5
:107010000F0095E80F0006F5887787E80F0004F564
:10702000C241572210312046FFF720FF2046FFF7CC
:1070300011FC2046FFF70CFA204604F081FE04F50F
:10704000A042002382F8B035C6F8CC3082F8B535BE
:107050002046BDE8F84004F047BB4FF0FF33CDE7D2
:107060002DE9F043354B1B6885B00546D86AFAF721
:1070700069FA00285FD105F5005393F9683D5A1C61
:1070800052D0002B05F58C6611DD95F87124242172
:1070900007EE903A01FB026292ED0B7AF8EEE77A86
:1070A000B0EEC77AB4EEE77AF1EE10FA3CDC05F503
:1070B000805305F5A85793F87C3713F0010429D0C5
:1070C000C3F340089B0732D495F8141495F858443C
:1070D0004FF0B00909FB015191F8F1314CBB022B83
:1070E00018D9684610F0F8FD694638460AF026FBC4
:1070F000044678B195F8143409FB03534246D3F89B
:107100000012684610F0EEFD0AF0B8FD69460AF07C
:1071100003FA044630460DF079F838460AF01AF9B9
:107120002846FBF70BFA204605B0BDE8F0830024A3
:10713000F0E74446EEE70020F6E700BF942C00207D
:1071400038B50C4B1B680546D86A0C46FAF7FAF9B5
:1071500010B10024204638BD0AF090FD21460AF007
:10716000DBF904460028F4D005F5AC40243025F0C6
:1071700063FEEFE7942C0020F0B500F5A043002259
:1071800083F8AF2583F8B02500F5C246044600F524
:10719000C04700EE101A96E80F0087B007F1F0051F
:1071A00085E80F0002ADB8EEC00A324628461749FE
:1071B00044F0EAFD95E80F0007F5887686E80F00B1
:1071C00004F5C24140F25712103120460191FFF7F9
:1071D0004DFE01992046FFF76DFB01992046FFF710
:1071E0007BFB04F500532046B3F94635002BB4BFB2
:1071F0004FF0FF33012387F8C830FFF729F9204605
:1072000007B0BDE8F04004F09BBD00BF0C65002056
:1072100010B50349044644F0B7FD204610BD00BF39
:107220000C650020F8B500F5C24300F5C0450446E2
:107230000E460FCB05F1F00787E80F0006F10801B5
:107240002046FFF761FEB28802EB820202EB820267
:10725000920012B204F5A043002AD8BF4FF4C872BE
:10726000A3F8AA25D5F8EC20D5F814115068091A0E
:10727000C3F87C1591680A31C5F81811D2680A3232
:10728000C5F81C210022C3F8902583F8AC2583F8AB
:10729000C025C3F8802503F27452002111604FF01D
:1072A000FF32C3F86C2594F8711404F58C62242025
:1072B00000FB012203F2A453D26A1A60F8BD000059
:1072C00070B50E4608310446FFF71EFEB38804F57C
:1072D000A04543B3642213FB02F3C5F87C35B5F92E
:1072E000AA35002BD8BF4FF47A7304F53750D8BFB6
:1072F000A5F8AA35242200212C30A5F003FC04F5C2
:10730000C04304F5BF4093ED4F0A314658307CF03E
:107310008DFBD5F80036072B0CD120460421BDE8A3
:107320007040FAF779BED5F87C35002BD7DC40F6F3
:10733000B833D2E770BD00000B7A00F5C04013F0FF
:10734000020F14BF4FF0FF33012380F8C83070479D
:107350007FB501F1080305460E460FCB6C4684E865
:107360000F0005F5C241204610F020FE21462846B8
:10737000FFF7CAFD31462846FFF7DEFF04B070BDB7
:107380007FB501F1080304460E460FCB6D4685E834
:107390000F0004F5C241284610F008FE2946204699
:1073A000FFF7B2FD20463146FFF7C6FF337907EEFF
:1073B000903A337E9B0748BF9FED0A7AF8EE677AD2
:1073C00004F5C04448BF67EE877A9FED077A67EE01
:1073D000877A0123FCEEE77AC4F8E030C4ED307A16
:1073E00004B070BD0000803B00A00C477FB501F1E8
:1073F000080304460E460FCB6D4685E80F0004F5E2
:10740000C241284610F0D2FD29462046FFF77CFDF8
:1074100020463146FFF790FFB38804F5C0444FF48F
:107420007A725343C4F8D8300123C4F8E03004B072
:1074300070BD00002DE9F34100F5C245044610354A
:1074400000F5C1400E467030294610F06FFD04F57E
:10745000A047D0B94FF0FF33C7F86C3506F10807E5
:10746000384610F069FC032802463CD1F1682846F2
:1074700010F038FCB28804F5C0432046C3F8E02081
:1074800002B0BDE8F041FEF7B9BE1AF097F9FAF77D
:1074900053FB012812D94FF0FF33C7F86C351AF0AF
:1074A0008DF990F8F432DFED150AB02202FB0300EB
:1074B00090ED3C0A284610F0E7FFCFE704F580582E
:1074C000D8F8000722F030FB04F5B853C7F86C0574
:1074D000D3ED007A9FED0A0ADFED080AF8EEE77AAD
:1074E00027EE800AE6E701AA0021384610F030FCBA
:1074F0000028BFD001990022B9E700BF00007A44FC
:107500000AD7233C7FB501F1080304460E460FCB92
:107510006D4685E80F0004F5C241284610F046FD8F
:1075200029462046FFF7F0FC20463146FFF704FFCE
:1075300004F5C0440023C4F8E03004B070BD00007E
:1075400037B504460D467EF0CBFBE060D5ED027A00
:10755000F5EEC07AF1EE10FA15DD9FED127A67EEC6
:10756000877AFCEEE77AC4ED027A56F05BFBA268FC
:107570004FF47A73B2FBF3F30B4A062103B0BDE874
:1075800030404FF077BC65F08BFD0023009395F9F8
:107590000D2095F90E3095F90C1065F01DFDA060D9
:1075A000E3E700BF00007A44586B0C082DE9F04374
:1075B0002DED028B85B004460AF060FB09F0B0FCAB
:1075C00004F5805304F5A04593F8F8390BB9002869
:1075D00077D0D5F86C35013373D1D5F89035002BC1
:1075E0004BD07EF07DFBD5F89035C01AB0F5FA6F20
:1075F00067D394F81424DFED617A9FED618A4FF030
:10760000B00808FB024292ED840A20EE270A22F01D
:10761000A3FA05F27459D9ED007A30EE670A22F028
:107620009BFADFED587A20EE080A04F5565720EE53
:10763000270A22F039FAFDEEC07A083717EE906A71
:10764000C5F86C65D9ED007A67EE887A17EE900A76
:10765000F8F75AFFCDE9020194F8143408FB03430C
:10766000D3F80C02F8F750FF474ACDE90001334642
:10767000062138464FF0FEFB23E004F59070FAF740
:107680005BFA02281DD994F81434B02202FB03439C
:1076900093ED837AF1EE047AB4EEE77AF1EE10FA24
:1076A0000FDD3A4B1B68D86A0368DB6998470128ED
:1076B00003D07EF015FBC5F89005D5F89035002B6A
:1076C0008FD104F54053D5F86C15D3F8B0074A1C98
:1076D000036849D01B6B98472D4807F051FB20B138
:1076E00004F5AC40243027F043FE2046FEF79AFE16
:1076F000D5F87C358342064639DA07EE906A9FED6D
:10770000257AF8EEE77A04F5565767EE877A083758
:1077100017EE900AF8F7F8FE1F4ACDE90001384647
:1077200006214FF0A7FB01264FF0FF33C5F86C355B
:1077300085F8AC6504F5C04C04F5C24494E80F002C
:107740000CF1F0070CF5887487E80F0084E80F004F
:10775000124865F021FE002385F8AF35304605B0AC
:10776000BDEC028BBDE8F0835B6B9847B4E708483B
:1077700007F0E6FA0028C0D1F1E700BF35FA8E3CE9
:10778000E02E65420000C842686B0C08942C002073
:10779000982C00200AD7233C8C6B0C0850500020FA
:1077A0002DE9F04F00F5A0492DED028B4FF0FF338E
:1077B00000F5C04AC9F86C350AF588730F460646CD
:1077C0000FCBBC8897F8048089B004AD240A85E803
:1077D0000F001FD006F5C14770372946384610F014
:1077E000DDFD29463846B0EE408A10F0A7FCDFEDFB
:1077F000567AB4EEE78AF1EE10FA0BDBE3B200EE54
:10780000903ADFED527AF8EE600A20EE270A284619
:1078100010F03AFE06F5405B99F8B025DBF8B007AA
:107820009FED4B0A036806F5C2479B6A32B306F523
:10783000C1412A467031984706F50051B1F97635B5
:10784000002B1EDD07EE903A09F29452F8EEE77A2B
:1078500092ED007AB4EEE77AF1EE10FA11DD06F55A
:10786000C1412A467031384610F004FD00BB0024A7
:10787000204609B0BDEC028BBDE8F08F2A463946A0
:10788000D9E7B8F1000F1CD1002C3CD1B1F9742517
:10789000DBF8B00700EE102A026809F5B163126A3E
:1078A000D3ED000AB8EEC00A9047B0EE408A0CE073
:1078B000002CDCD197E80F000AF1F00585E80F00F5
:1078C000D6E707EE908AB8EE678A2946384610F068
:1078D00065FDB4EEC08AF1EE10FA17DBB9F8603638
:1078E00003932946384610F059FDBCEEC00A06F550
:1078F0005650039B174A8DED000A062108304FF0C1
:10790000B9FA0124B4E79FED128ADEE706F5C1411A
:107910002A467031384610F0ADFC04460028A6D047
:10792000B9F8603603932946384610F037FDBCEEAF
:10793000C00A06F55650039B074A8DED000A062142
:1079400008304FF097FA93E700000034E02E6542CC
:1079500000000000A86B0C08C66B0C0838B500F5D9
:10796000005500F5C043B5F978150029ACBF0122D8
:107970004FF0FF320029B8BF4942044683F8C820BF
:1079800089B204F001FB04F5AB4393ED057AB5F938
:107990007435002BCABF07EE903ADFED0E7AF8EE91
:1079A000E77AFCEEE77AF8EE677AB4EEE77AF1EE82
:1079B00010FA08D804F556500830074A06214FF04F
:1079C00059FA012038BD204604F0F6F90028F1D11B
:1079D000F8E700BF00000000E46B0C08F8B500F504
:1079E000C14600F5C245703610350446294630467A
:1079F00010F09CFA04F5405750B304F5A043D3F8B7
:107A00006C154B1C24D0D7F8B00703681B6B984744
:107A100004F5C045D5F8E030012B46D0D5F8E0306C
:107A2000022B06D12046FEF7BBFCD5F81431984254
:107A300042DD2046FEF7B4FCD5F81431C01A002808
:107A4000B8BF4042B0F5FA7FCCBF0020012034E03F
:107A5000294604F5C24010F0A1FCDFED187AB4EE1F
:107A6000E70AF1EE10FA16D53046294610F066FB0B
:107A70009FED137ADFED130AF6EE007AE0EE077A57
:107A800028469FED110AFDEEE77AF8EEE77A27EE39
:107A9000800A10F0F9FCD7F8B0079FED0C0A0368D4
:107AA0002A469B6A31469847B2E72046FEF778FCA3
:107AB000D5F814319842B1DB0120F8BD00004843ED
:107AC000A00CB345000096430AD7233C00000000F9
:107AD00073B5374CD1ED026AD4ED417A9FED357A1A
:107AE000F8EEE77A0546D7EE876A0E46F5EEC06AED
:107AF000F1EE10FA08DD56F095F82F4A06214FF006
:107B0000B9F9012002B070BDD1ED037AF5EEC07A6B
:107B1000A4F67424F1EE10FA94ED006A12DDF4EE8E
:107B2000C67AF1EE10FA0DD556F07CF805462068BD
:107B3000F8F7EAFC214ACDE90001062128464FF07A
:107B400099F9DEE7DFED1E7A337CB4EEE76AF1EEF9
:107B500010FA54BFB0EE677AB0EE467A0BB9002047
:107B6000D0E7B5EEC06AF1EE10FA0CDC86EE876A5B
:107B700003EB830307EE903AF8EEE77AF4EEC67A69
:107B8000F1EE10FAEBD52C7C002CE8D17EF0A8F8B1
:107B90006B69C01A337C4FF47A7253439842DED932
:107BA00001232B747EF09CF868612046AAE700BF91
:107BB000988C00200AD7233CFC6B0C080D6C0C0839
:107BC0000AD723BC38B5054677F0F4FB76F032F9D6
:107BD000044640B97EF084F8EB68C01AAB6898425E
:107BE00084BFAC600124204638BD000038B504468F
:107BF0000D467EF075F804F5C0439FED067AC3F894
:107C0000E400D5ED027A67EE877AFDEEE77AC3ED00
:107C1000387A38BD00007A4410B504467EF060F82A
:107C200004F5C043D3F8E420801AD3F8E020904252
:107C30004FF0000084BFC3F8E000012010BD000039
:107C400000F5C04300F5AB41D3F8E02091ED057A93
:107C500022EAE27207EE902AF8EEE77A0020B4EE0C
:107C6000E77AF1EE10FA44BFC3F8E0000120704754
:107C700010B500F5005300F5C044B3F94635002BAC
:107C8000B4BF4FF0FF33012384F8C83000F5C24081
:107C90000FC804F5887484E80F0010BD38B5044699
:107CA0002DED028BF0EE408AB0EE608A09B3012917
:107CB0005ED0B5EEC08AF1EE10FA69DDDFED357AFF
:107CC000B4EEE78AF1EE10FA62D8FCEEC87A04F559
:107CD000565017EE903A304A062108304FF0CAF855
:107CE000FDEEC87A04F5005417EE903A84F8133587
:107CF0003CE0F8EE000A21F031FE40B104F580448A
:107D00004FF0FF33C4F8AC3FBDEC028B38BD04F537
:107D10000053B3F91C2507EE902AF8EEE77AF4EE4B
:107D2000E87AF1EE10FAC4D8B3F91E3507EE903AAE
:107D3000F8EEE77AF4EEE87AF1EE10FAB9DBDFED6F
:107D4000157A68EEA77A04F58043FDEEE77A04F52C
:107D5000565017EE902AFCEEE87AC3F8AC2F0621B5
:107D600017EE903A0D4A08304FF084F80120CBE727
:107D7000FCEEC07A00F5565017EE903A084A0621FC
:107D8000083004F514544FF075F8C4ED0A8AEDE795
:107D90000020B9E70000C842536C0C082C6C0C089A
:107DA000406C0C08D1F80D3000EE903AD1F8093053
:107DB000097A00EE103AFFF771BF000070B58B88AA
:107DC000012B04460D4611D100F590763046F9F7A7
:107DD000B3FE02280AD994F81414B02303FB0161FE
:107DE0002046DC31BDE87040FFF7AAB909F046FF34
:107DF00005F10801BDE8704009F08EBBF0B500F553
:107E0000A0460027A24B86F8B57589B004460846FF
:107E10000D4683F8297124F021FE50B3012386F822
:107E2000AC3504F54053D3F8B0070368DB6B9847D3
:107E300004F5C04386F8B37503A8C3F8CC700FF0FF
:107E40004BFFB6F860164FF6FF73994208BF3946EC
:107E5000013104F5AC4001AA89B2243026F00AFEB3
:107E600028B1BDF80600A0F115035842584186F824
:107E7000AD056B885D2B00F0038132D81F2B29D80C
:107E80000F2B01D800202AE0103B0F2BFAD801A2BB
:107E900052F823F0877F01089D7F0108A77F010822
:107EA000B17F0108C57F0108937F0108757F010834
:107EB000857E0108857E0108857E0108857E010892
:107EC000857E0108857E0108857E0108D57F010831
:107ED000BB7F0108532BD5D1012086F8B30509B02B
:107EE000F0BDBD2B18D8BB2B4BD8B22B7CD00CD8F7
:107EF000702B74D0722BC5D1D5ED027AFDEEE77AE6
:107F000004F5C044C4ED387A3BE0B32BBAD129461E
:107F10002046FFF753FF34E0C33B9AB2112AB1D891
:107F2000112BAFD801A252F823F000BF2380010823
:107F3000857E010823800108857E0108857E010871
:107F4000857E010823800108857E0108857E010861
:107F5000857E01085F800108857E0108857E010815
:107F6000857E0108857E0108F37F0108857E010872
:107F700013800108002386F8E93529462046FFF7DB
:107F800051F90120ABE705F108012046FEF7BCFFDF
:107F9000F7E729462046FFF793F9F2E729462046FE
:107FA000FFF7D6F9EDE729462046FFF7E9F9E8E7BC
:107FB00029462046FFF71AFAE3E729462046FFF74D
:107FC000A1FADEE704F59E4129222831204606F079
:107FD000A7F8D6E729462046FFF72CFAD1E729462D
:107FE0002046FFF703FECCE729462046FFF7DAFEDE
:107FF000C7E7AB88012BC4D803F0010386F8AE3580
:1080000004F55650AB88234A062108304EF032FF63
:10801000B7E7A988003918BF0121204600F0A6FB68
:10802000AFE704F5C346EB6804F5C044083694F89E
:10803000011273B92B6963B96B6953B930465AF0B1
:10804000C3FE04289DD194F8011230465AF0C6FEB2
:1080500097E705F1080230465AF0FEFF91E704F574
:10806000C04304F5C34095ED041AD5ED020A95ED21
:10807000030A93F80112002208305AF0D1FE80E77B
:1080800004F59E4029461030FFF75AFA79E700BF01
:10809000988C0020646C0C0800F5804200F59E432B
:1080A000D2F87C2F10339A4201D1FFF7A7BE0120EE
:1080B0007047000010B500F5804200F59E43D2F8ED
:1080C0007C2F10339A4204460ED100F59E410822BF
:1080D000283106F025F804F55650044ABDE8104052
:1080E000062108304EF0C6BE10BD00BF746C0C08EF
:1080F00070B58EB009AD044628460E460FF0ECFD73
:1081000004F5A0434FF6FF72B3F86036934208BF00
:108110000023013304F5AC4007AA99B2243026F0BD
:10812000A9FCB0B104F5C04416B10023C4F8C430B2
:1081300095E80F0001AE86E80F00D4F81C310093DB
:1081400004F5887494E80E00034802F073FD0EB045
:1081500070BD0120FBE700BFC87B002070B505465D
:1081600005F5C046002103F00FFFD6F8CC407CB9DE
:10817000284603F021FE10B90024204670BDD6F831
:10818000C430012BF8DD7DF0ABFDC6F8CC00F4E780
:10819000D6F8E01061B17DF0A3FDD6F8CC30C01A5E
:1081A000D6F8D8309842E7D90023C6F8E03001214C
:1081B0002846FFF79DFF04460028DDD005F5565000
:1081C000054A0621083005F5A0454EF053FE002370
:1081D00085F8B535D1E700BF9C6C0C0838B50A4668
:1081E0008B88190A137EDB0748BF01EB8101044627
:1081F00048BF490003F0C8FE04F5A043002583F8FA
:10820000B555204603F0D8FD10B90025284638BDE5
:1082100004F5C043D3F8E01041B1D3E930128A42EB
:10822000F3DD012AF1DDC3F8E05001212046FFF71C
:108230005FFF05460028E8D004F55650024A0621A3
:1082400008304EF017FEE1E7B46C0C0838B505466F
:1082500005F5C044898803F097FED4F8E03083BB6D
:10826000D4F8C430002BB8BF5B42012B02DC0024E1
:10827000204638BD94F8C92094F8CA3072B9002B52
:10828000F5D005F55650D4F804216423062192FB5D
:10829000F3F308300C4A4EF0EDFD01E0002BF0D175
:1082A0000121C4F8E0102846FFF722FF0446002809
:1082B000DDD005F55650054A062108304EF0DAFDAE
:1082C000D6E70021EFE700BFCC6C0C08EA6C0C0885
:1082D0002DE9F0434B881F2B8BB004460A4631D85A
:1082E0000F2B07D804F55650974A042108304EF05A
:1082F000C1FD88E0A3F110010F29F3D801A050F8C7
:1083000021F000BF17840108E1840108ED84010811
:10831000FB84010815850108258401080B840108E8
:10832000E5820108E5820108E5820108E58201088D
:10833000E5820108E5820108E5820108218501083E
:1083400007850108702B00F0F9800CD8532B00F042
:10835000ED805D2BC6D100F59E4010300BB0BDE81E
:10836000F043FFF72FBCB32B08D8B12B4BD8722B9F
:10837000B8D10BB0BDE8F043FFF762BCD42B3BD8BB
:10838000BB2BAFD9A3F1BC02182AABD801A151F87D
:1083900022F000BF0784010807840108E582010874
:1083A000E5820108E5820108E5820108E58201080D
:1083B00007840108E582010807840108E5820108B5
:1083C000E5820108E582010807840108E5820108C9
:1083D000E5820108E5820108078401080784010895
:1083E00007840108E5820108E58201080784010885
:1083F000E582010807840108DF2B04D040F6B8327B
:1084000093427FF46FAF01202CE020460BB0BDE813
:10841000F043FFF7CBB8114620460BB0BDE8F04360
:10842000FFF7BEB904F5A04504F5BF46D5F8002610
:1084300004F5C14704F5C248072A06F1580607F1BA
:10844000700708F1100804F5C2430ED104F5AB44DF
:1084500078340194D5F87C2500923946424630465E
:108460007BF0A8FB0BB0BDE8F0830DF127010022E3
:10847000364807938DF82720FEF7D8FC05F5B7623C
:10848000D2ED007AD5F89C9505F28C52D2ED000A17
:1084900005F5B36230EE670A92ED001A8DED060A1B
:1084A00004F5C4400C30CDED050A8DED041A75F0CD
:1084B000B7FC0546204600F0A9FE9DF827209DED5B
:1084C000041ADDED050A9DED060A079BCDE90202BF
:1084D000CDE900954246394630467BF0C1FAC1E706
:1084E0002046918803F050FD0020BBE7114620464E
:1084F0000BB0BDE8F043FFF771BE20460BB0BDE8FE
:10850000F043FFF72BBE114620460BB0BDE8F04309
:10851000FFF79CBE20460BB0BDE8F043FFF71EBA44
:1085200020460BB0BDE8F043FFF758BA00F59E4077
:1085300010300BB0BDE8F043FFF7CABA0BB0BDE88E
:10854000F043FFF769BB00BF046D0C08982C0020B6
:1085500070B500F5804200F59E43D2F87C2F1033B1
:108560009A4205460E4602D00024204670BDFFF711
:10857000AFFE04460028F7D005F556503188083084
:1085800052F068FEF1E7000021F04003152B04D003
:10859000A1F15E0358425841704701207047000026
:1085A000102946D8DFE801F0090D1115191D212504
:1085B00029452D31354139393D0000F59E404C307B
:1085C000704700F59D402430704700F59D402C30E9
:1085D000704700F59D403430704700F59D403C30B9
:1085E000704700F59D406430704700F59D406C3049
:1085F000704700F59D407430704700F59E4008308C
:10860000704700F59E401030704700F59E402830BE
:10861000704700F59E403030704700F59E4038307E
:10862000704700F59E404430704700F59E4054303E
:10863000704700207047000000290DDB074890F8C4
:10864000E82DCBB29A4207D3D0F8E43D0122595C21
:10865000A0F5005005F040BE704700BF984C0020C8
:108660002DE9F34100F5005300F5565593F8B83D58
:1086700003F0010603F0020803F004075B07044659
:1086800005F1080535D01F4A062128464EF0F2FBB9
:1086900026B104F543503C3077F09AFCB8F1000F56
:1086A00004D004F54950143077F00EFA27B104F5E0
:1086B0004E502C3078F0B6F804F5C044012384F80D
:1086C000B132114A114B1249B8F1000F08BF1A46D6
:1086D000002F08BF1946CDE900210E4A0621002EC1
:1086E00018BF134628460C4A4EF0C4FB02B0BDE842
:1086F000F0810A4A0621284602B0BDE8F0414EF05A
:10870000B9BB00BF316D0C08266D0C0828470D0859
:108710002D6D0C08206D0C08426D0C08546D0C0872
:1087200010B5044600F543503C3077F07DFC04F56D
:108730004950143077F0F4F904F54E502C3078F0AD
:10874000ABF804F5C04393F8B1225AB1002283F884
:10875000B12204F55650044ABDE810400621083005
:108760004EF088BB10BD00BF746D0C0809B1FFF757
:1087700077BFFFF7D5BF000000F580430A4AD3F862
:108780007C1F91420DD093F8893F43B900F59E427A
:108790001032914203D100F5A04090F8AE35184652
:1087A00070470023FBE700BFE47B002010B50446C0
:1087B0007DF096FA054BD3F89C3FC01A642804D884
:1087C0002046BDE8104056F099BE10BD986C0020C0
:1087D00010B500F53654D4ED0A7AF5EEC07AF1EE14
:1087E00010FA8AB04FF0000304F1280444D907932B
:1087F0000893099306AB019307AB009303AA05AB5B
:1088000004A900F5A85008F00DFF30B3DDED080A0B
:108810009DED070AA1F0B4FDDDED090AA1F0B0FD60
:10882000D4ED007A9DED047A77EEA76AB4EEE70AFC
:10883000F1EE10FAF4EEC76AACBF01200020F1EEB1
:1088400010FA0CD802309DED037AF4EEC77AF1EEFF
:1088500010FA0CD8003818BF01200AB010BDF4EE91
:10886000C77AF1EE10FA9CBF0130C0B2EBE70128E5
:1088700094BF00200120F0E70020EEE710B5074B81
:108880001A7A4AB901241C724BF0C4F9224611210C
:10889000BDE810404AF076BF10BD00BF608F0020D9
:1088A00010B5074B1A7A4AB100241C724BF0B2F98A
:1088B00022461121BDE810404AF064BF10BD00BF40
:1088C000608F0020F0B5054685B0684605F5A856CE
:1088D0000FF002FA6946304608F0D6FFA0B13348DF
:1088E000334C344F75F09CFA40B105F53653D3ED57
:1088F0000A7AF5EEC07AF1EE10FA07D8002328467E
:108900002380FB73FFF7CCFF05B0F0BD2846FFF7CF
:108910005FFFA0B363787BBB23780133DBB2082B06
:10892000237002D1304608F0E9FE2378092B02D1EA
:10893000304608F0DBFE2378092B1DD94FF48573F0
:1089400023804BF067F9022210214AF01BFF7DF0D3
:10895000C7F96368C01A47F23053984209D905F540
:108960005650154A022108304EF084FA7DF0B8F9CD
:1089700060602846FFF782FF6378FB73C4E72678C0
:10898000002EF9D0013E6378F6B22670002BF3D0AA
:10899000002EF1D166704BF03DF9324610214AF0BD
:1089A000F1FE2846FFF77CFFE6E700BFA48E00201B
:1089B000608F00200D900020886D0C0800F5A0400D
:1089C000D0F80036042B14BF90F82C060120704715
:1089D00073B500F580450192A5F8941F04467DF01B
:1089E0007FF9C5F8980FD5F87C0F03685B68984746
:1089F00085F8920FD5F87C0F03685B6898470F28BD
:108A0000019A0BD80F2827D8DFE800F01C261C1C81
:108A10001C1C1C1C1C264E260A260A0A18281BD1C0
:108A200004F50056019296F98835ABB1D5F87C0F64
:108A300003685B68984785F8920F96F98835019A24
:108A4000022B29E01F4B93F8B23203B304F59D418A
:108A50006431204605F064FBD5F87C0F95F8926FE1
:108A600003685B68984704F55654864204F108048D
:108A700020D0D5F87C0F03689B689847124A0346BC
:108A80000421204602B0BDE870404EF0F3B904F571
:108A9000005393F98835022BD8D004F59D41042B5F
:108AA0000CBF6C312431D4E72046FFF787FF002844
:108AB000D2D1B5E7054A0421204602B0BDE8704096
:108AC0004EF0D8B9988C0020986D0C08BA6D0C083F
:108AD000F0B5044604F5804685B00F46154656F0BD
:108AE00093FCD6F87C0FA6F8947F03685B689847E0
:108AF00018281ED8DFE800F00D0D0D0D0D0D0D0D21
:108B00000D1D53690D0D58581D1D1D1D1D1D1D1DCD
:108B10000D00314BD3F80026012A21D104F5005372
:108B200093F88935023B012B1AD904F5405383F899
:108B30008425D6F87C0F294A294B052D18BF1346EA
:108B4000026803939268904704F5565408340090E5
:108B5000039B244A042120464EF08CF905B0F0BD59
:108B6000214B93F8B2323BB104F59D412A46643162
:108B7000204605F0D5FADCE704F5005393F9893572
:108B8000032B03D1204603F05BFAD2E7022BEBD094
:108B9000042B15D104F59E412A461031E8E7204602
:108BA000FFF70CFF0028C4D104F5005393F9893571
:108BB000032BE7D0022BD7D0042BEBD0012BB8D15D
:108BC00004F59E412A462831D2E704F5005393F973
:108BD0008935042BADD1DDE7987C0020D06D0C08E1
:108BE00007520C08D86D0C08988C002070B500F561
:108BF000565504460835124A0421284604F5804695
:108C00004EF038F90023A6F8943F04F5005393F88A
:108C1000D034032B12D196F8921F3022204605F053
:108C20005BFBD6F87C0F03689B689847054A0346B0
:108C300006212846BDE870404EF01CB970BD00BF4B
:108C4000EC6D0C08036E0C0800F5405310B50022C3
:108C50000529044600F5565083F8842500F10800E4
:108C60000CBF054A054A042104F580444EF002F980
:108C70000023A4F8943F10BD1C6E0C082D6E0C0848
:108C800030B50B4687B00446052A19D8DFE802F054
:108C9000182C0353186000F5A043D3F80036042BBA
:108CA00022D02E4D95F8A53FF3B105F50451A1F65C
:108CB000DC2026F0B1FA28B1294B012283F82C26BA
:108CC00007B030BD05F50451A1F6DC2026F0A4FD67
:108CD00050B104F59E4104221031A5F5804007B043
:108CE000BDE8304005F01CBA04F5A043D3F80036C7
:108CF000042BE5D004F5005393F95335022B0BD127
:108D0000164991F8A53F3BB101F50451A1F6DC20CD
:108D100026F082FA0028CFD104F59E4104222831A2
:108D2000204605F0FDF904F51450133007B0BDE8F6
:108D3000304042F09DB80B4A112101A87CF092F816
:108D400004F5C04001AA0121643077F057FEB7E76F
:108D500007B0BDE8304003F073B900BF986C002045
:108D6000987C0020486E0C0870B52DED048B0446ED
:108D70007CF0AAFF4F4BB4F8BE101A884E4E8A42C0
:108D800005464E4A06D01980002330601370BDECB2
:108D9000048B70BD33684A49C31A8B4276D90123CC
:108DA000137056F031FC56F0E9FA356056F02CFCA1
:108DB00056F0E4FA04F5405393F8833523B104F5F3
:108DC000C040643077F06EFD56F000FB0428DED919
:108DD00056F01AFB0021204603F05CFC00212046DF
:108DE000F0EE409A03F060FC01212046B0EE409A7C
:108DF00003F022FE00212046B0EE408A03F05EFC24
:108E000004F5C4400C30F0EE408A75F013F8DFED45
:108E10002D7A0028B0EE690A4FF0040008BFB0EECA
:108E2000678A57F0E7FFB0EE490A132057F0E2FFD8
:108E3000B0EE680A152057F0DDFF04F5C045B0EE2E
:108E4000680A1A2057F0D6FF64354620B0EE480A6B
:108E500057F0D0FF284677F0B3FD08BB0121084644
:108E600058F0CAFA9FED170A022057F0C3FF9FED92
:108E7000150A032057F0BEFF204604F001F8BDECB0
:108E8000048B2046BDE8704004F018BF1278002A19
:108E90003FF47DAF44F6206293427FF678AF80E7DF
:108EA0002846FDF719F804F5C04393F96E302B2BD3
:108EB000D4D06CE76C8F0020708F00206E8F002064
:108EC000400D03000000000000F5804200F59E43C5
:108ED000D2F87C2F10339A4204D100F5A04090F8CC
:108EE0002C06E8B10F4B93F8D00403F58043A0F1B2
:108EF0002702012A93F8C0320FD92C2809D00A285A
:108F000009D0A0F13102504250410A2B18BF002075
:108F100070470120F9E7012070470A3B5842584149
:108F2000704700BF984C002008B500F5005393F837
:108F3000B82342B193F8F4332BB1FFF7C5FF80F0AB
:108F40000100C0B208BD0120FCE700002DE9F04798
:108F500000F50055A74F95F8F483044600F5C4408A
:108F60008AB00C3074F05CFFD7F80036042B06464C
:108F70004FD000284DD0B7F86216A7F5A040FFF7F4
:108F800003FB014620B197F828164B1E5942594160
:108F900004F50E57DFF870A23837384664F062FDEA
:108FA0009AF8C0320A2B814603D1A6BB00238AF867
:108FB000C03295F8B833002B39D195F9BE338E4DB8
:108FC000012B03D0063BDBB2012B11D895F8D0342E
:108FD0000A2B0DD104F58046D6F87C0F03681B6A76
:108FE000984728B1D6F8801F2B22204605F098F824
:108FF0009AF8C0320A2B04BF37238AF8C03295F89A
:10900000D0340A2B02D1372385F8D0340AB0BDE81A
:10901000F0870121BCE740EA0803DBB2002BC8D18E
:10902000AAF5C04000F0F2F80028BFD0C1E7002E3A
:10903000ECD004F5BF4058307AF088FC0028E5D128
:109040002046FFF741FF0028E0D1B9F1000F00F002
:10905000BF806A494A46384664F0DCF895F9BE8319
:10906000B8F1010F06D040F38580A8F10603DBB20A
:10907000012B7FD85FFA88F8B8F1010F4ED104F5C3
:10908000804204F59E43D2F87C2F10339A4209D1D6
:1090900004F5A04393F82C3623B195F85335013BE2
:1090A000012BB3D904F59E410A222831204606AE91
:1090B00005F036F830460EF00FFE95F9D12392BB3D
:1090C000B8F1010F2FD004F5C048B5F9D233D8F864
:1090D000EC10DFED4B5AD1ED017A002BF8EEE77A78
:1090E00051DD07EE103AF8EEC76AE6EEA57A304693
:1090F000FDEEE77A17EE901A0EF0F4FD00233846E5
:10910000CDE9043364F04AFD04A965F0A7FA00280C
:1091100058D0049B0893059B099316E004F59E41E3
:109120000A223831C2E72046FCF74EFF07EE900ACC
:109130006F4604F5C24221463846B8EEE70AFEF70C
:1091400067F897E80F0086E80F0095F9BE33012B0A
:1091500010D031462046FDF7ADFB31462046FDF7E5
:109160003DFF95F9BE33072B04D104F5405401238C
:1091700084F882354AF04EFD4A4609210AB0BDE81E
:10918000F0474AF0FFBAD5EDF06A95EDF35A95ED48
:10919000F17A35EE076A36EEC57AB4EEC67AF1EEAC
:1091A00010FA8DBF37EE067A05F2B45393ED007ACC
:1091B00027EE257A8ABFF6EE006AE7EE257AE7EE1B
:1091C000267A94E7D8F8EC309A680892DB68A3E72F
:1091D000B8F1000F3FF41AAF95F8F433002B7FF489
:1091E00015AF04F55650074A052108304DF042FEF0
:1091F000C0E700BF987C0020984C0020546E0C08FB
:109200000000C8425D6E0C08988C002010B5044622
:1092100000F5C4400C3074F00DFE04F5A04404F2D7
:10922000046494ED007A48B1DFED067AB4EEE77A93
:10923000F1EE10FAACBF0120002010BDDFED027A84
:10924000F4E700BFCDCCCC3D6666663F00F58043B9
:10925000D3F87C1F00F59E435433994204D100F5A6
:10926000A04393F8F8259AB900F59E43103399422C
:1092700010D100F5A04393F8F8254AB1D3F80026A1
:10928000032A07D1B3F86226A2F116035A425A41C3
:10929000104670470022FBE72DE9F84F00F58042A9
:1092A00000F59E43D2F87C2F10339A42054600F514
:1092B000A04704D100F5005898F92C3533B90023A4
:1092C000C7F8EC3587F8E935BDE8F88F7CF008FD84
:1092D000D7F8A045814634B1041B40F6C3139C4225
:1092E00094BF002401242846FFF790FF834620B155
:1092F000002487F8E84500263EE005F5C4400C3020
:1093000074F08EFD82460028F2D005F5BF4658362F
:1093100030467AF01BFB00283FD097F8E865BEBBCB
:109320003CB305F5805141F27072D1F8F836002B4C
:10933000B8BF5B42934206DCD1F8FC36002BB8BFC5
:109340005B42934227DD05F5AC41683105F5C2402B
:109350000FF024F8DFED457AC7F8EC95B4EEE70A94
:10936000F1EE10FA4FF000034CBF01260026C7F8BB
:10937000F035012387F8E83505F59070F8F7DCFB48
:10938000022835D9002C44D10023C7F8EC359BE7DF
:109390005C465E46EDE73446EBE730467AF0BEFACF
:1093A000064638B1002CA6D04FF4FA73C7F8F03552
:1093B0005446A0E7D7F80036012B03D0032B0FD07B
:1093C0003446D9E708F2CC53D3ED007AF5EEC07AF3
:1093D000F1EE10FAF4DD97F8F835002BF0D1E3E761
:1093E0002846FFF733FF0028EAD1002CDCD1C3E781
:1093F00005F5085A98F84E13504606F009FB002868
:10940000C2D098F84E13504606F0FAFB0028B9D1A6
:10941000BAE7D7F8EC3513B9C7F8EC9554E7D7F8A5
:10942000F025A9EB03039342FFF44EAF97F8E9351B
:10943000002B7FF449AF012287F8E92598F82C35F5
:10944000DB0705D50C2105F5C4400844F8F7AAFA56
:1094500005F5565008302EB1054A0221BDE8F84FF7
:109460004DF008BD034A3146F8E700BF00009642C0
:10947000746E0C088A6E0C082DE9F04F2DED028BEE
:10948000054685B0002305F5005803937CF028FCC1
:1094900008F5A563D3ED007AF5EEC07AF1EE10FA87
:1094A000C4BF9FEDC27A67EE877A05F5907BC8BF8F
:1094B000FCEEE77A07465846CCBF17EE906A962630
:1094C000F8F73AFB022840F2FF8095F814349FED3C
:1094D000B87AB02202FB0353D3ED837A67EE877A22
:1094E000FCEEE77A17EE903A9E428CBF00260126EA
:1094F000B8F91C35022BB8BF022307EE903AB8EE3C
:10950000E78A03A9F6EE087A05F5A85028EE278A1F
:1095100008F098F9044640B1DDED037AF4EEC87A1C
:10952000F1EE10FAACBF012400245846F8F704FB12
:1095300005F5C449012809F10C0905F5A04A18D818
:10954000484674F06DFCA0B19CB90AF2046292ED39
:10955000007ADFED987AB4EEE77AF1EE10FA08DDE2
:10956000DDED037AF4EEC87AF1EE10FAACBF012417
:109570000024484674F054FC0090002800F002815A
:1095800095F8142405EB0212D2F8C02172B15846A6
:109590000192F8F7D1FA012800F29880019A41F27D
:1095A0008731BA1A8A428CBF00220122DAF89C1550
:1095B00001B11AB9002C40F08B80344605F580418A
:1095C00005F59E42D1F87C1F103291421AD198F9CC
:1095D0005425002A40F0848000228AF8EA25DAF82F
:1095E0000026042A00F0AC80072A00F0BF80032A7E
:1095F00008D12846FFF72AFE20B100248AF8E94561
:10960000CAF8A0459AF8EA2502B18CB907EE904A4B
:109610009FED697AF8EE677A0AF2046267EE877A5C
:10962000D2ED006A9FED657AE6EE877AC2ED007AA8
:109630002846FFF7EBFD0446A8B19AF80806CAF8D9
:109640009C7508B9CAF80C7605F5804105F59E426F
:10965000D1F87C1F1032914205D1DAF8A02502B171
:1096600008B9CAF8A0759AF830278AF8084664F352
:10967000C3028AF830276EF01FFD21466EF0F8FC19
:109680004F4A28465471FFF707FE2846FBF776F944
:1096900034B198F8D2241AB97CF022FBC8F8D4046B
:1096A00088F8D2442846FFF7B1FD00287BD1484610
:1096B00074F0C0FB80F00100C0B28AF8100605B05B
:1096C000BDEC028BBDE8F08F002611E700226DE7AC
:1096D0001FF0DAFC1EF0CEFC00287FF46EAF6DE7C1
:1096E000524207EE902A05F61862F8EEE77A92EDFC
:1096F000007AF4EEC77AF1EE10FA13DD01228AF84F
:10970000EA25CAF8F4750AF20462DFED2E7A92EDCA
:10971000007AB4EEE77AF1EE10FA7FF760AFC2EDAF
:10972000007A5CE79AF8EA25002A3FF458AFDAF8A5
:10973000F42540F6B831BA1A8A423FF64DAF4EE7EB
:1097400005F5BF4058307AF0E9F800283FF45AAFE9
:109750000AF28C5292ED007ADFED1A7AB4EEE77AD3
:10976000F1EE10FA7FF74EAF009C4BE70AF28C52F5
:1097700092ED007AFEEE007AB4EEE77AF1EE10FA9E
:10978000F2D43FE7DAF80026002C18BF3446012A4D
:1097900007D005F5BF4058307AF0B6F800283FF4FE
:1097A00031AF00242EE7002087E700BF0000B4425D
:1097B0000000C8429A99993E9A99193E9A99593F40
:1097C0000D900020CDCC4C3E00207047002070470B
:1097D000012070470020704701207047034BD3F8E9
:1097E0000006431E58425841704700BF987C002035
:1097F00030B587B002A80EF06FFA32487AF084F8DC
:1098000020B131493148FDF767F81FE02D487AF063
:1098100085F8E8B12E4C04F12405234604F110022A
:10982000A4F11001A4F5947000957AF09DF8CDE9AB
:109830000045A4F66C3292ED000A264904F11003AB
:10984000A4F11002A4F594707AF050F807B030BD7E
:109850001C4802A97AF0A0F808B102A9D2E71B4877
:1098600002F0AAFA0028CCD11B4C94F810315B0707
:1098700020D4D4F82431002BC3D0134AA2F1200104
:10988000A2F110000EF0F6FC0028BAD1134C0F48DC
:10989000D4ED007AB7EE000A04F6783130EE670AAC
:1098A000FDF74AF8094804F6583204F67831FCF717
:1098B000E9FBCBE7A4F5C040FDF7B8F80028C5D117
:1098C000D7E700BF708C0020A88D0020982C0020C6
:1098D000988D0020845A0020988C0020308200202F
:1098E00008B50A4890F8C535013B012B03D8A0F50F
:1098F0000050F9F785F90648F9F7A6F80448F9F792
:1099000045F9BDE808400248F9F774BC984C0020BE
:10991000982C0020124A904208B50ED002F108019E
:1099200088420AD002F11001884206D002F13801C3
:10993000884202D05C32904206D10A4B93F97D05F1
:10994000B0FA80F0400908BD03681B6A984728B147
:10995000054B93F8820580F00100F4E70120F2E75F
:10996000447B0020984C0020985C0020104A9042D4
:1099700008B518D002F10801884214D002F1100194
:10998000884210D002F1380188420CD05C329042FB
:1099900009D003681B6A984738B1064B93F88205D3
:1099A00080F0010008BD0020FCE70120FAE700BFBD
:1099B000447B0020985C0020024A0260024A426018
:1099C000704700BFDC6E0C089841002008B50368A2
:1099D000DB6D98470648D0F87C2F00F608739A4252
:1099E00005D0BDE80840A0F58040FEF799BE08BD4F
:1099F000986C00202DE9F843484C04F2745300227F
:109A00001A60A4F1F003C11A4B42A4F500584B416F
:109A100088F8243804F28453002584F85855A4F8B3
:109A2000AE5584F8B25584F8705584F8E95584F839
:109A3000EA55C4F8D855C4F8D455C4F8D055C4F87C
:109A4000E0551A604368D3F8FC31A4F8A83504F552
:109A5000885306460FCB04F5805909F1F00787E8D3
:109A60000F0084F8B15584F8C055C9F8CC507CF08B
:109A700037F944F87C0C336830465B6998474FF0FF
:109A8000FF3384F8B40584F8B55588F8845589F80F
:109A9000295184F8B35544F8543C336830469B6DE3
:109AA00098470546002836D0336830469B6B984768
:109AB00084F8F805D8F8B0070368DB6B9847A4F57D
:109AC000D75076F0EDFBA4F5A04002F04FFDA8F6CC
:109AD000484064F02DF894F82C36CBB1A4F5A040A2
:109AE000FFF794FBA0B909F5037074F0A3F978B9F6
:109AF00054F8840C03685B6B984748B954F092F8AB
:109B0000074A06214DF0B6F904F2246025F030FC36
:109B10000448F8F7D1FA2846BDE8F883987C00207D
:109B20009C6E0C08982C002070B503681B6E0E46C6
:109B300015469847044650B995F900303BB9054899
:109B4000054B00683246C06A29461CF041F92046A0
:109B500070BD00BF942C0020C06E0C0810B50E4CD8
:109B6000204676F099F904F5AC7075F011FF04F514
:109B70002C7076F03FFE094B03F5A042002182F8DD
:109B8000701502F27452002103F540531160012256
:109B900083F8482010BD00BF945D0020982C002061
:109BA00008B52DED028B1520B0EE408A57F022F952
:109BB000B0EE480ABDEC028B1A20BDE8084057F011
:109BC00019B9000008B5084890F97D350121A0F5C4
:109BD000005033B102F030FFBDE80840462057F096
:109BE00009B902F051FFF7E7984C002004207047B4
:109BF000004870474EA90D08004870474EA90D084F
:109C0000037A73B1D0ED037AFDEEE77A17EE903A5E
:109C1000084AC2F81436437A3BB10369C2F81836D1
:109C200070474368D3F8F831F2E74368D3F8FC3162
:109C3000F4E700BF987C002008B50023038100F101
:109C40001401406807F014FE012008BD70B56E4E87
:109C50002DED048B06F59F4304460121304693ED1C
:109C6000119ADFED6A9A02F015FD0121B0EE408AEB
:109C7000304602F019FDC8EE297A06F500556068F5
:109C8000B5F9A03504F1140108EE903AF8EEE88A2F
:109C9000B5F9A23568EEA78AC0EE297A08EE103A27
:109CA000B8EEC88A28EE278A07F0E2FD95F9A635B6
:109CB00063B39FED577AF0EEE87AF4EEC77AF1EEEF
:109CC00010FA23D5227A6368002A55D10122227224
:109CD0000022E26094ED037ADFED4E7AD3F8F8319A
:109CE0004D4A4E4867EEC77A9FED4D7A67EE877A08
:109CF000B0EE490AFDEEE77A17EE901A0B44C2F86F
:109D000014360023012276F057F808E00023434878
:109D10002372F0EE490AB0EE680A76F049F80420A2
:109D200057F068F895F9A63543B19FED397AF0EE12
:109D3000C87AF4EEC77AF1EE10FA28D40023394835
:109D40006372F0EE490AB0EE480A75F08BFC1320FE
:109D500057F050F8B5F9A435002B03DD324E96F9D3
:109D6000C23363BB28482021F8F714FC002843D1F4
:109D7000254802F0CBFA42E0D3EDC56A96ED467A6B
:109D8000D4ED037AE6EE877AC4ED037AA2E7637A2C
:109D90002BB9012363726368D3F8FC3123611E4B36
:109DA0002169C3F818166368D3F8FC010023091A67
:109DB0001A461C48B0EE490A75F03AFDC7E7012182
:109DC000A6F5405002F07AFC80EE297AB5F9A43568
:109DD000002106F56B7007EE903AF8EEE77AF0EEA8
:109DE000490A27EE870A76F005FCBDEC048B204675
:109DF000BDE87040FFF7D4BE0348F9F761F807EEFD
:109E0000900AB8EEE70AF0E7982C002000A08C45F5
:109E100000000034E02E6542987C0020945D002014
:109E20000000C842EC5E0020985C00202DE9F04F55
:109E30002DED0C8BDFF8A4A39FEDDDDA9FEDDD9A0D
:109E400097B00AF59F4300F11405044601215046DE
:109E500093ED11BA02F01EFC01215046F0EE408A4B
:109E600002F022FC01215046B0EE408A02F026FCAE
:109E7000DFEDD17A88EEA77A0AF5005601A8B6F987
:109E8000A0350AF5A04B0AEE903AF8EEEAAAB6F928
:109E9000A235DFEDCA8A6AEE87AA88EE277A0AEE33
:109EA000103AB8EECAAAB6F9A4359FEDC58A2AEED3
:109EB00007AA80EE277A09EE903AF8EEE99A6AEE60
:109EC0008D7A69EE879AF0EEEACAF4EEC8CACDED53
:109ED000017AB0EECACA6AEE0D7AF1EE10FAF0EE2F
:109EE000E9BAB4EEC8CACDED027A58BF4FF0010905
:109EF00069EE8D7A48BF4FF00009F1EE10FAF4EEEA
:109F0000C8BA9AED460ACDED037A54BF4FF0010866
:109F10004FF00008F1EE10FA54BF0127002722F09D
:109F2000A3F801A9284621F0BFFB284621F0AEFC8A
:109F3000284621F025FC20EE090A284620EE280AB2
:109F4000BDEEC00A10EE103ACBF8143621F032FC08
:109F500020EE090A20EE280ADFED9A8ABDEEC00A3B
:109F6000CDED0D8A10EE103ACBF818360DF1280B16
:109F70004FF07E53594660680A93CDED0C8ACDEDC3
:109F80000B8A07F075FC0021504602F055FDB0EE3B
:109F9000C00AB4EEC80AF1EE10FA16D55046FFF723
:109FA00035F990B9F4EEC8CAF1EE10FA0DD5B4EE59
:109FB000C8CAF1EE10FA08D5F4EEC8BAF1EE10FAFC
:109FC00044BF9BE80F0085E80F000AA821F0C2FCFF
:109FD000294612A88DED141A8DED120ACDED130A43
:109FE000CDED151A21F0C8FC0DF1100A51460EA84E
:109FF0008DED101ACDED048ACDED058ACDED068AE2
:10A000008DED0E0ACDED0F0ACDED111A21F086FA75
:10A01000B6F9A035DFED6C7A01EE103AB6F9A2354B
:10A0200009EE103AB6F9A43508EE903AB8EEC11A26
:10A03000B8EEC99AF8EEE88A21EE271A29EE279A97
:10A0400068EEA78AF4EEC8CAF1EE10FA21EE0D1AF6
:10A0500029EE0D9A68EE8D8A07D594F82430DFED4D
:10A06000597A002B18BFB0EE671AB4EEC8CAF1EEE9
:10A0700010FA07D594F82530DFED527A002B18BF7F
:10A08000B0EE679AF4EEC8BAF1EE10FA07D594F87C
:10A090002630DFED4C7A002B18BFF0EE678A9AE885
:10A0A000070007AE86E80700F1EE410AC2209DEDE9
:10A0B000070A1FF065FDC3208DED070AB0EE491AAF
:10A0C000F1EE490A9DED080A1FF05AFDB0EE681A3C
:10A0D000F1EE680A8DED080AC4209DED090A1FF013
:10A0E0004FFD514630468DED090A21F053FF12A96C
:10A0F00028468DED120ACDED130A8DED141A21F0CC
:10A10000D3FA284621F0C2FB304BDDED076A93ED10
:10A11000407A9FED280AC6EE877A3046DDED086A60
:10A12000CDED077AD3ED967A86EEA77ADDED096A52
:10A130008DED087A86EEA77A8DED097A21F094FFED
:10A14000B9F1000F01D0CDED07AAB8F1000F01D091
:10A150008DED08AA0FB1CDED099AF0EE4B0A9DEDF9
:10A16000070A1B4875F024FE042056F043FEF0EE6B
:10A170004B0A9DED080A174875F074FA132056F043
:10A1800039FE0021F0EE4B0A9DED090A124876F0E7
:10A1900031FA2046FFF704FD84F8249084F82580E6
:10A1A00084F8267017B0BDEC0C8BBDE8F08F00BFB3
:10A1B00035FA8E3CE02E654200A08C450000C84276
:10A1C0000000003400000000CDCC4C3E985C002024
:10A1D000945D0020EC5E002044600020982C00205C
:10A1E00010B50446FFF7EEFC0B4B93F9A625022AA7
:10A1F0000DD1B3F9A425002A09DD03F5805393F9A5
:10A20000C23323B12046BDE81040FFF70FBE204601
:10A21000BDE81040FFF71ABD984C00200A20704797
:10A220000048704769790C080048704769790C0844
:10A2300001207047012070470120704701207047BE
:10A2400001207047034BD3F80006031F58425841C2
:10A25000704700BF987C0020F8B51A4E06F5885369
:10A260000FCB06F5805505F1F00405F5887584E8F7
:10A270000F0085E80F00002706F2246086F8B47509
:10A2800025F0B6FA104B1C68E56A2B6828465B6817
:10A290009847A8B195F84D3093B1E36A9B8F7BB195
:10A2A00053F0C0FCE36A094A9B8F06214CF0E2FDA3
:10A2B000E36A06F22460998F25F086F8E36A9F87A7
:10A2C0000120F8BD987C0020942C0020AC6F0C0875
:10A2D00010B50A4C94F82836012B0BD104F22460F7
:10A2E00022F030FBB4F86236152B03D104F6D87097
:10A2F00079F0EAFB0023C4F8A03510BD987C00205B
:10A3000008B507F0BBFC90F87C32DB0704D5BDE84C
:10A310000840024825F008B908BD00BFBC820020F3
:10A3200010B5304C94F82836012B0ED0A4F1D8018A
:10A330000822A4F5A04003F0F3FE53F073FCBDE83F
:10A340001040294A06214CF095BDB4F86236162B10
:10A3500005D0152B36D1D4F80036072B0AD1234867
:10A3600004F06CFA214804F0B9FBBDE810401F4826
:10A3700004F0C8BAA4F5A040F9F7ACF8A4F5A040E1
:10A38000F8F7A6FFA4F54053D4F8141693F9E42582
:10A3900064235A4304F6D87079F0F2FAC4F814062C
:10A3A00004F6D87079F02EFC30B1BDE810409FED76
:10A3B000100A462056F01EBDA4F5A040BDE810408E
:10A3C000F8F766BD1E2B18BF4FF0FF33074818BFC4
:10A3D000C4F86C35F9F77EF80448F8F779FF0348BC
:10A3E000ECE700BF987C0020C46F0C08982C00207C
:10A3F0000000000010B5144BB3F86236532B04462E
:10A400001ED102F013FF9FED110A462056F0F2FC18
:10A410009FED0E0A492056F0EDFC9FED0C0A4A20F4
:10A4200056F0E8FC462056F0C5FD492056F0C2FD26
:10A430004A2056F0BFFD2046BDE81040FFF78EBB16
:10A44000BDE81040FFF74CBA987C002000000000E7
:10A4500008207047004870475C700C08004870473F
:10A4600068700C080120704708B50248FEF7F8F83C
:10A47000012008BD982C0020014800F059B900BF08
:10A480007C7B002010B50446FFF72AFA2046BDE881
:10A490001040FFF797BB000001207047004870474D
:10A4A000DC700C0800487047E4700C08012070470D
:10A4B0000120704710B5054B03F5C24403F5C243B4
:10A4C0000FCB103484E80F00012010BD982C002021
:10A4D00008B50B4800F5A04200F500530321D3F85E
:10A4E000DC3D93FBF1F3C2F81436F8F759FF04484A
:10A4F000F8F7EEFEBDE808400148F8F7C9BC00BF18
:10A50000982C00200720704700487047C4530C085F
:10A510000048704758710C080120704701207047AF
:10A52000012070477047000008B5002303720361E3
:10A530000248FCF78FF9012008BD00BF982C0020CD
:10A5400010B5194CD4F8C43DB3F9083023B9D4F888
:10A55000D03DB3F90830F3B1002303720361D4F89E
:10A56000C40D55F041F904F6DC53D3ED007A0F48E1
:10A57000F8EEE77A27EE800ABDEEC00A10EE103A38
:10A58000C0F81436A0F5A040F8F70AFFBDE8104067
:10A59000074801F031BB037A002BE0D0A4F500504E
:10A5A000F8F798FFF2E700BF984C0020987C002055
:10A5B000982C002070B54E4DDFED4E7A95F814348E
:10A5C0009FED4D7A2DED048BB02606FB035393EDE2
:10A5D000848A9FED4A9A28EE278A05F5B853BDEE86
:10A5E000C88A93ED030AF8EEC87A044667EE897AC2
:10A5F00097EE870A1FF0B0FA237AF0EE408A002B1C
:10A6000062D105F50053D3F8C43DB3F90830002BEF
:10A610005AD1284601F07AFE002855D195F8143415
:10A6200095F8581406FB035393F8F12100294BD1F8
:10A63000012A49D993ED837AF0EE087AB4EEE77AED
:10A64000F1EE10FA40DBDFED2E7AB0EEE80AB4EE60
:10A65000E70AF1EE10FA37D5236993B37BF040FB9C
:10A660002369C01AB0F5FA7F32D8237A002B3CD088
:10A67000244DA5F1200696E80F0085E80F0094ED23
:10A68000038AA5F110013046B8EEC88A0DF086FEA7
:10A6900028EE098ADFED1C0A284670EE200AB0EE8B
:10A6A000480A0DF0F1FE194B9FED190AD3F8B007D7
:10A6B000BDEC048B03682A4631469B6ABDE87040B6
:10A6C00018477BF00DFB20612369002BCDD0C5E737
:10A6D000104D84ED038A012323720023236105F1C9
:10A6E00010030FCB85E80F00BFE7BDEC048B70BDF6
:10A6F000982C00200000C84235FA8E3C0AD7233C33
:10A70000DB0FC93FA88D002000007A44985C002030
:10A7100000000000888D0020052070470048704729
:10A72000CC710C0800487047DC710C0801207047A0
:10A7300038B52DED028B4D4C9FED4D8AD4F8C40DEC
:10A7400055F052F8D4F8DC3D07EE903AF8EEE77A8F
:10A7500004F5405527EE800AA4F50050BDEEC00A6E
:10A7600010EE103AC5F81436F8F71AFED4F8C80DF2
:10A7700055F03AF8B5EEC00AF1EE10FACBBF04F28C
:10A78000345304F55E63D3ED007AD3ED007A394893
:10A79000CBBF20EE270A20EE270A20EE080A28EE7B
:10A7A000400ABDEEC00A10EE103AC5F81836F8F7A8
:10A7B000C1FD04F2345393ED007AD5F8180604F580
:10A7C0005E6327EE087AD3ED007A27EE888AFDEEE5
:10A7D000C77A17EE902AFDEEC87A17EE901A1FF08E
:10A7E0006FFAC5F818062348FDF7C6FF20B1D5F863
:10A7F00018365B42C5F818361F4B93F8903F63B18B
:10A8000094F98835022B08D1002301214620C5F890
:10A810001436C5F8183656F047FE54F0F5FE5F21A1
:10A8200055F09AFFF8B155F067FF02281BD195F853
:10A83000B135C3B905F2845304F2D45493ED007AD0
:10A84000D4ED007AB4EEE77AF1EE10FA0BD50123DD
:10A8500085F8B135BDEC028B084A0948BDE838409F
:10A8600004214CF007BBBDEC028B38BD984C002096
:10A870000000C842982C0020986C0020E4710C085D
:10A880002062002010B50446FFF72AF82046BDE8F4
:10A890001040FFF797B90000062070470048704746
:10A8A00060720C080048704770720C0801207047F5
:10A8B0000120704701207047012070477047000059
:10A8C00008B50248FBF7C6FF012008BD982C002000
:10A8D00038B50F4C04F50055D5F8C40D54F084FF7D
:10A8E00005F6DC52D2ED007AF8EEE77A04F5A043E3
:10A8F00027EE800A2046BDEEC00A10EE102AC3F8EB
:10A900001426F8F74DFD2046BDE8384001F074B933
:10A91000982C00200F20704700487047E4720C0804
:10A9200000487047EC720C08012070470120704706
:10A930000120704701207047012070477FB50B4D03
:10A9400005F54053002283F8822505F5C2430646EB
:10A950000FCB6C4684E80F0000232846B3602146E5
:10A96000FCF73CFB012004B070BD00BF982C002018
:10A9700010B53C4CD4F8D035002B2CDD7BF0B0F971
:10A98000D4F8D035C01A40F6B733984223D8A4F58E
:10A990004053D4F8C405D3F8DC2D51421FF090F990
:10A9A000C4F81406A4F5A040F8F7FAFCD4F8D4359E
:10A9B000002B14DC2C48F8F78BFC2C4890F88235DF
:10A9C00093B30121A0F5405002F036F8BDE81040E5
:10A9D000462056F00FBA2448F8F77CFDE6E77BF0F6
:10A9E0007FF9D4F8D435C01A40F6B7339842E1D88D
:10A9F0001F4BDFED206A93ED007AD4F8C80503F60B
:10AA0000AC03D3ED007A27EE267A67EEA67ABDEE88
:10AA1000C77AFDEEE77A17EE102A17EE901A1FF0AC
:10AA20004FF9C4F81806C8E7A0F5805090F913351F
:10AA3000012B04DCBDE810400B48F8F729BAD4F824
:10AA4000E035002BF6D07BF04BF9D4F8E035C01A96
:10AA500040F6B7339842EDD804F2DC5494ED000A86
:10AA6000B4E700BF987C0020982C0020985C002060
:10AA7000CC5100200000C842D0ED027A0348FCEE21
:10AA8000E77A17EE903A99B201F07EBA982C00203E
:10AA900084B010B503AC84E80E000B4821466F2249
:10AAA000FCF7E4F99DF80C1011F0040102D12046E6
:10AAB0000DF0DCF904482146FCF790FABDE810409F
:10AAC000012004B0704700BF982C0020B0EEC00AEF
:10AAD000FDEEC07A38B54FF6FF7205460C4617EE0C
:10AAE000900A00211FF0ECF807EE900A002CF8EE17
:10AAF000E77A054BC5ED027A14BF4FF0FF32012211
:10AB000083F8C82038BD00BF988C0020FEF770BEC7
:10AB10000C2070470048704760730C08004870476D
:10AB20003DA90D08012070470120704701207047A2
:10AB3000012070470120704708B50C48FDF798F8D0
:10AB40000A480B49FBF7B6FE0848F7F707FF40B184
:10AB500006484FF48051F7F71DFD10B10348FBF78D
:10AB600079FE024800F0C0FD012008BD982C0020AD
:10AB7000A88D002008B50D48F8F7ACFC0B48F7F796
:10AB8000EDFE50B109484FF48051F7F703FD20B1B5
:10AB9000BDE80840054801F02FB80448F8F798FBD5
:10ABA000BDE808400148F8F773B900BF982C0020B1
:10ABB00008B50A484FF48051F7F7ECFC38B1084863
:10ABC0000022D0F8201100F588700DF08BF8BDE858
:10ABD00008400248002101F0D7B900BF982C00209E
:10ABE000988C0020881A10B51EF092FF104BD3F8F5
:10ABF000C4200028B8BF4042002AB8BF524248F6DD
:10AC0000A041B2FBF1F24FF47A7102FB01118842CC
:10AC10000CDC93F81021D20606D503F5887403F5F1
:10AC200080730FCB84E80F00012000E0002010BDEE
:10AC3000988C002084B0F0B52DED048B87B011AC5A
:10AC400084E80E004D4FDFED4E8A0546D7F8B00779
:10AC500007F5405696ED370A0368B0EEC00A5B6A06
:10AC60009847B4EEE80AF1EE10FAB0EE408A07DA3F
:10AC7000012007B0BDEC048BBDE8F04004B0704784
:10AC800007F5445120460DF095FA02A8CDED030AD0
:10AC90008DED020A21F0DCF804A88DED040AB0EE77
:10ACA000480ACDED050A20F0CDFF15A920468DED0F
:10ACB000000ACDED010A0DF07DFA02A88DED020A21
:10ACC000CDED030A21F06AF8B4EEE80AF1EE10FACD
:10ACD000CEDBB4EEC08AF1EE10FA9FED2A9ADFEDDA
:10ACE0002A8ADFED2A9A2BD802A8694620F09AFF1B
:10ACF00004A88DED040ACDED050A21F005F868469B
:10AD000020EE098A21F000F896F9C83007EE903A53
:10AD1000F8EEE77A28EE288AA7EEA90A1EF01CFFB3
:10AD200020EE090ABDEEC88A20EE280A18EE101A95
:10AD3000FDEEC07A284617EE902AFFF753FF98E7FA
:10AD400038EE400A38EE088A80EE080A9FF0B0FC20
:10AD500002A8B0EE408A20F0D7FF96F9C830F0EE96
:10AD6000007AB0EE697AA8EE677A07EE903AF8EECC
:10AD7000E77AA7EE270A1EF0EFFEC0E7985C0020F6
:10AD800000000034E02E65420000C842DB0FC93FDE
:10AD900010B504460848F7F7E1FD20B92046BDE8A4
:10ADA0001040FEF725BD04484FF48051F7F7F2FB41
:10ADB0000028F3D010BD00BF982C00200020704761
:10ADC00000487047D4730C0800487047DC730C08C7
:10ADD000002070470020704738B5154C054600210B
:10ADE000204601F057FC042056F004F800212046CC
:10ADF00001F05AFC132055F0FDFF0021204601F020
:10AE00005DFC2846FEF7CCFE2046012101F014FE31
:10AE1000462055F0EFFF6B6804F5A044D3F8F831F5
:10AE2000C4F814366B68D3F8FC31C4F8183638BD52
:10AE3000982C0020FEF792BE0B2070470048704708
:10AE4000976C0C080048704750740C08012070473C
:10AE500001207047012070470020704770B50B4CEF
:10AE600004F5C2430FCB04F5C04606F1F00585E8B2
:10AE70000F002046FBF7A8F801462046FCF77CF9B6
:10AE8000002386F88031012070BD00BF982C00207F
:10AE900038B53148F8F71EFB2F48F8F719FA2E4855
:10AEA000F7F7F6FF2C481021F7F774FBE0B12B4AB7
:10AEB000D2F80431D2F814219342D4BF00230123E5
:10AEC000264C94F8802172B973B304F580730FCBCC
:10AED00004F1F00585E80F00A4F5C040FBF7B8FACF
:10AEE000012384F8803138BD1D4AB2F9AC1D002918
:10AEF000F9DD02F580429FED1B7AD2F80431D2F8D9
:10AF0000F4209B1A07EE903AF8EEE77A67EE877A1C
:10AF100007EE101AB8EEC77AF4EEC77AF1EE10FA1F
:10AF2000CCBF01230023CBE7A4F58043642193F930
:10AF3000E42512FB01F2D3F8DC1DA4F580548A420B
:10AF4000A8BF0A46D4F81406C3F8DC2D51421EF0FF
:10AF5000B7FEC4F81406C6E7982C0020988C002091
:10AF6000984C00200AD7233C38B52D4DB5F97835DB
:10AF700083EAE371A1EBE37189B241B1002B05F5DE
:10AF80008043B4BF4FF0FF32012283F8C820254C24
:10AF9000254800F0F9FF94F8B235FBB995F953351F
:10AFA000022B1CD1214D95F8A53FA3B105F5045105
:10AFB000A1F6DC2024F030FC68B10123282205F53D
:10AFC0007161A5F5804084F85D3603F0A9F828B9D1
:10AFD000002384F85D36012384F8B23538BD012B97
:10AFE0000ED1A4F5A04000F0E7FE48B1A4F5A040C2
:10AFF000FBF7ECF90028B8BF4042B0F57A7FD1DB0F
:10B0000095F95335042BE9D1084D95F8A53F002B50
:10B01000E1D005F50451A1F6DC2024F079FCCBE762
:10B02000984C0020987C0020982C0020986C0020E0
:10B030000220704700487047C4740C0800487047ED
:10B0400032A90D08034B0022C3F81426C3F81826B2
:10B05000704700BF987C002038B5094D044628464B
:10B06000F7F7F2FC2846F7F791FD2046F7F7A6FD23
:10B070002846F8F7BFF82046BDE83840FEF7A2BDE5
:10B08000982C00200D207047004870473C750C0834
:10B090000048704744750C08012070470120704734
:10B0A000012070470023C37480F8243001207047CA
:10B0B0000148002100F068BF982C00202DE9F041E4
:10B0C000B34DD5E942322DED088B1343D5F8042159
:10B0D000134388B006460FD1AE48F8F7FBF9AD48E8
:10B0E000F8F7F6F89FEDAC0A462008B0BDEC088BE7
:10B0F000BDE8F04155F07EBE06F0C0FD90F87C3210
:10B10000DB07E9D5B6F90830F17C09EE103AB6F95B
:10B11000103008EE903AB8EEC99AF8EEE88AA5F534
:10B120008057002940F0D6809FED9CAA29EE0ABAEC
:10B130000122FDEECB7AA5F5C04017EE903AC7F894
:10B140007C35FAF76FFF706800F57F700790B0EEFE
:10B15000408A20F0D9FDDFED927A20EE270A1EF01A
:10B1600079FC0798F0EE409A20F018FEA5F5C04053
:10B17000F0EE40AAFEF74AF805F58074002876D173
:10B1800094E80F0006F1140C8CE80F0094E80F000F
:10B1900005F1F00C8CE80F0005F5887C8CE80F00B9
:10B1A000D5ED457A7F48F8EEE77AF0EE680A77EE5B
:10B1B0008B7AB0EE690AFDEEE77AC5ED457A0DF0BF
:10B1C00063F9002387F8E93596F91230714803EBEB
:10B1D000830303EB83039B000121A7F8AA35F6F74D
:10B1E0001BFF97F8F885B8F1000F73D16E4B9FEDF8
:10B1F0006F7AB3F91C3507EE903AF8EEE77A67EE0E
:10B20000877AF4EEE7AAF1EE10FA63DD52F00AFD58
:10B21000044619EE900AF5F777F9CDE9040118EE26
:10B22000900AF5F771F9CDE9020119EE100AF5F768
:10B230006BF95F4ACDE90001062120464BF01AFE6A
:10B240007AF04EFDC7F86885C7F854057AF048FDD6
:10B250000123C7F8640529EE8A0AF3741EF024FC62
:10B26000BDEEC00A10EE103AC7F86C3532E07AF045
:10B2700037FDD7F80C36C01A42F2107398427FF6A9
:10B280007FAFF0EE087AF4EEE7AAF1EE10FA7FF75E
:10B2900077AFBCEEC88A18EE103A9BB208EE103AAF
:10B2A000B8EEC88AB4EEC89AF1EE10FA48D852F057
:10B2B000B9FC404A06214BF0DDFD94E80F0005F58E
:10B2C000887C8CE80F000123F3740321A5F5C040AE
:10B2D000F6F7A2FE2F4803F053FD28B12D480321B5
:10B2E000F6F79AFE0023F374D7F80036012B40F0EE
:10B2F000B080D5F80431B2699FED28AA9B1A07EEF9
:10B30000903AD7F86C350133F8EEE79A5AD0DFED72
:10B310002A7AE9EE0A7AF4EEE79AF1EE10FA0ADAFE
:10B32000264906F114000DF039F8F4EEC08AF1EE6A
:10B3300010FA00F28E8017480321F6F76DFE88E0C0
:10B3400052F070FC1E4A06214BF094FD94E80F0069
:10B3500006F1140C8CE80F0094E80F0005F5887CCA
:10B360008CE80F00D5ED457A39EE488AF8EEE77A99
:10B37000F0EE680AE8EE0A7A6046B0EE690AFDEE81
:10B38000E77AC5ED457A0DF07FF80121F1749DE76C
:10B39000988C0020982C0020000000000000C8427B
:10B3A000E02E6542A88D0020984C00209A99993E85
:10B3B0008D750C084C750C08000048C3988D002052
:10B3C00068750C08B6F90A3007EE903AF8EEE77A9D
:10B3D00006F1140467EE8A7AF4EEE79AF1EE10FAB9
:10B3E00051DB424920460CF0A9FEDFED417ADFF83F
:10B3F00014C1B6EE008AA0EE278A94E80F00BDEED5
:10B40000C88A9FED3C0AB8EEC88A8CE80F0028EE87
:10B41000008AF0EE680AB0EE480A60460DF034F893
:10B42000D5ED457AF8EEE77A28EE0A0AE9EE0A7ACF
:10B43000FDEEE77AC5ED457A1EF036FBBDEEC00A9B
:10B4400010EE103AC7F86C35D7F80036012B3FF4F0
:10B450005EAF294803F074FC18B127480321F6F7C2
:10B46000DBFDD7F80036012B17D1234803F0E6F9AE
:10B47000214803F033FB204808B0BDEC088BBDE841
:10B48000F04103F03FBA194920460CF087FFF4EE73
:10B49000C08AF1EE10FAA4D9D6E796F824302BB979
:10B4A000164861F079FF012386F824301248F8F736
:10B4B00011F81148F7F70CFF0F48F7F7E9FC1048AF
:10B4C00090F884356BB1002380F884353322022153
:10B4D000A0F5405008B0BDEC088BBDE8F041FDF789
:10B4E000F7BA08B0BDEC088BBDE8F081988D00205C
:10B4F000A00CB3450AD7233C982C002050500020C4
:10B50000985C0020A88D002010B50446FEF754FA80
:10B510002046054B40F8143B0CF0DEFB2046034967
:10B520003FF0D0FB204610BD40760C08D8750C08C3
:10B530000320704700487047A4760C080048704705
:10B54000B0760C08F8B52B4D06460027A5F54050FF
:10B55000A5F88075F7F724FF7368A5F58052D3F836
:10B56000F811D2F8DC3D994205F5005423DBC4F80C
:10B57000143673689FED206AD3ED7F6A02F234536C
:10B5800093ED007AF8EEE66A27EE067AF4EEC76AE3
:10B59000F1EE10FA18DBBDEEC77A17EE103A174835
:10B5A000C4F81836FDF7E8F820B1D4F818365B4235
:10B5B000C4F81836F8BD5B429942D8DD012385F8FE
:10B5C0008035C4F81476D4E702F55E62D2ED007AD5
:10B5D00067EE867AF4EEE76AF1EE10FA93BFFDEEBD
:10B5E000E77A012385F8813517EE903A88BF00236A
:10B5F000D5E700BF985C00200000C842982C0020CE
:10B6000070B500212DED028B04463448344D01F015
:10B6100041F832480021F0EE408A01F045F895F8F3
:10B620008035B0EE408AD3B1B0EE680A042055F000
:10B63000E1FB95F8813593B3B0EE480A132055F03D
:10B64000D9FB2648002101F039F82046FEF7A8FA78
:10B65000BDEC028B2046BDE87040FEF7B3BA05F59D
:10B660000056A5F54050F7F7EFF9D6F81436002B41
:10B670000CDCD6F81436002BDBDA042055F0CEFBB8
:10B68000B4EEE80AF1EE10FACED4D2E7042055F079
:10B69000C5FBB4EEE80AF1EE10FAEADDC4E7114D9D
:10B6A0000E48F7F773FAD5F81836002B0CDCD5F8EE
:10B6B0001836002BC5DA132055F0B0FBB4EEC80ADB
:10B6C000F1EE10FAB8D4BCE7132055F0A7FBB4EEA6
:10B6D000C80AF1EE10FAEADDAEE700BF982C0020B0
:10B6E000985C0020987C002000F5C0400023C0E951
:10B6F000303380F8C93080F8CA30704700F5804395
:10B70000D3F8AC3F002BCBBF07EE903A00F51450B6
:10B71000B8EEE70ADFED037ADCBF90ED080A20EE11
:10B72000270A70470000C8422DE9F0412DED028B39
:10B7300000F5A85784B09FEDCA8A054603A938468C
:10B740008DED038A06F07EF8B0B19FEDC67ADDED8F
:10B75000037A05F5AC4367EE877AD3ED086A9FED6F
:10B76000C27AE6EE877AF4EE487AF1EE10FA48BF34
:10B77000F0EE487AC3ED087A2846F7F73FF805F56A
:10B780008044B0EE408AF0EE000A9FEDB50A1EF04C
:10B79000CFFA04F6C473D3ED007A38EE678A05F564
:10B7A0000056E0EE087AC3ED007A94F8903F002B43
:10B7B00040F09780D4F87C2F05F59D436C339A4276
:10B7C00005D005F59D4374339A4240F08A800821E4
:10B7D0002846F6F7DFFE804640B106F5A463D3EDB8
:10B7E000007A9FEDA27A67EE877A75E002212846FB
:10B7F000F6F7D0FE0146002857D0D6F8CC3D1B8B7B
:10B800002846414608EE103A01F016F9D6F8CC0D5C
:10B810004369B8EE488AB0EE401A3BB3012B2AD0F8
:10B82000DFED937AF0EE671A06F5A46393ED000A54
:10B830009FED8E7AF4EEC17AF1EE10FA20EE070A4F
:10B840004FF0640124DBB6F81C2512FB01F2B0EEC8
:10B85000672A07EE902AF0EE400AB8EEE70A1EF0DB
:10B86000C1F8BDEEC00A10EE103AECE0DFED807AD0
:10B87000F1EE481AD8E78DED010A53F027FF07EEE5
:10B88000900ADFED7B1A9DED011AF8EEE77ACBE71F
:10B89000B6F81E3513FB01F300EE903AB0EE482ADD
:10B8A000F8EEE00AF0EE671AD9E7B6F91C25B6F90A
:10B8B0001E359B1A07EE903A2846B8EEE78A01F04B
:10B8C000BBF8B6F81C35642213FB02F307EE903A7E
:10B8D000F8EEE77AE8EE007AFDEEE77A17EE903AB6
:10B8E000B1E005F5A043D3F80036042B40F0A0806A
:10B8F00005F5BF40583078F051F8C4F8A80FD4F8D7
:10B900007C0F03689B6B984700285ED094F8BC3F7F
:10B91000002B5AD0D4F87C3F05F59D452435AB4229
:10B9200053D0D4F8A83F9FED537A07EE903AD4F85D
:10B93000B83FF8EEE77A384627EE878A07EE903A66
:10B94000F8EEE78A68EE878A06F088F9C8EE807A12
:10B9500004F57C639DED037A77EE877AB6EE007A84
:10B96000B4EEE78AF1EE10FA4CBF77EEC87ADFED5D
:10B97000407A77EE877A93ED007AFDEEE77AF8EE7B
:10B98000E77AB4EEE77AF1EE10FA0ADD37EE676A8D
:10B99000DFED396AB4EE666AF1EE10FA48BFF0EEF8
:10B9A000477A04F57C63C3ED007AD4F8A83FDFED55
:10B9B0002F6A07EE103AB8EEC77AA7EEA67ABDEE68
:10B9C000C77A17EE103AC4F8A83FD4F87C0F036882
:10B9D0001B6B984740B1B4F9B42F002AC2BFD4F80A
:10B9E000A83F9B18C4F8A83FB6F91E25B6F91C1548
:10B9F000D4F8A80F64235A4359431EF061F9C4F8E0
:10BA0000A80F06F67863D6F8880E93ED4A8A06F0FA
:10BA100025F9C8EE007A04F57B649DED037A77EE94
:10BA2000C77AC4ED007A04B0BDEC028BBDE8F081AA
:10BA3000D4F87C2F05F59E4338339A4206D1D4F8CA
:10BA4000AC3F002B02DDC4F8A83F58E705F59E4344
:10BA500010339A427FF4C1AE2846FFF74FFE00E74D
:10BA6000CDCCCC3DCDCC4C3ECDCC4C3F0000C842E3
:10BA7000000000000AD7233C9A99993F30B500F5A1
:10BA8000A85587B0002304462846039304930593E2
:10BA900004F0A8FF002846D003A9284605F000FFBF
:10BAA000002840D004F5C15393ED007ADFED226AFF
:10BAB0008DED017AB0EEC77AD3ED037AB4EEE67A73
:10BAC000F1EE10FACDED027A06D5F0EEE77AF4EE5B
:10BAD000E67AF1EE10FA2DD401A820F0B1F903A90D
:10BAE00001A820F0F5F804F5145393ED0A7AB5EEA9
:10BAF000C07AF1EE10FAC4BFDFED107A27EEC00A6B
:10BB000004F58044C8BFA7EE270A03F12803CABF83
:10BB100001230023FDEEC07A84F8BC3FCCBF17EEB2
:10BB2000903A002304E004F58044002384F8BC3FED
:10BB3000C4F8B83F07B030BD000000340000C84270
:10BB40002DE9F04100F5C0472DED028B07EE901A6C
:10BB5000D7F8CC3000F5C245B8EE678A04461035F8
:10BB600000F54056C3BB00F58043D3F87C2F00F5A9
:10BB70009E4310339A4204D000F59E4338339A42D4
:10BB80002AD104F5A04393F8B0352BB3294604F528
:10BB9000C2400CF003FCD6F8B0070368F0EE408A10
:10BBA0005B6AB0EE480A9847F0EE087A60EE277AB2
:10BBB000F4EEE78AF1EE10FA0EDDBDEC028BD6F85A
:10BBC000B0079FED0C0A036804F5C1412A469B6A41
:10BBD000BDE8F04170311847B0EE480ABDEC028B69
:10BBE000D6F8B00797F9C82003682946DB6ABDE894
:10BBF000F04118470000000070B504462DED028B9F
:10BC000004F5C0467AF060F8D6F83831444AC31AD1
:10BC1000934205466CD907EE903AB8EE670ADFED1D
:10BC2000417A9FED411ADFED410A20EE270A40F2EA
:10BC300095101DF0A5FFC6F8385104F50055DFED4D
:10BC40003C7AD5F8C83DB3F9083008EE103A95F9BA
:10BC50007A35B8EEC88AF0EE408A28EE278A0BB112
:10BC6000B1EE488A9FED337ADFED337AB4EEC78ABE
:10BC7000F1EE10FA4CDAD6ED4D6AF4EEC76AF1EE49
:10BC800010FAB4EEE78AACBF01230023F1EE10FAFC
:10BC90003BD996ED4D7AB4EEE77AF1EE10FA34D84E
:10BCA0002046FAF7D7FD95F97B3500EE103A05F5F9
:10BCB0006A6305F6A865D5ED000A93ED001AB8EEA3
:10BCC000C00A40F2A710F1EE600A20EE080A1DF04B
:10BCD00057FF28EE800ADFED198A20EE280A204659
:10BCE000FDEEC07A17EE901AFAF772FD86ED4D8AD6
:10BCF0002046FAF7D9F92046F7F7CAF8BDEC028BCF
:10BD00002046BDE87040F7F7E3BA002BC8D1CAE778
:10BD1000B4EEE78AF1EE10FAC5D90023B9E700BF07
:10BD20009F860100BD3786359A99193ECDCCCC3D12
:10BD30005304693900000034000000B40000C84218
:10BD400070B5054600F5AC404FF0FF31243022F0CD
:10BD5000E7FE431C064605F5A04404D104F5B16492
:10BD6000124B236070BD05F5C24105F5C14010318D
:10BD700070300CF0E3F99FED0E7AF6EE007AE0EE0B
:10BD8000077A04F5B164FDEEE77A17EE900A301AEF
:10BD90001DF0BEFE07EE900A9FED067AF8EEE77AF8
:10BDA00067EE877AC4ED007ADCE700BF0000B4429A
:10BDB000A00CB3450AD7233C00F54050D0F8B0079B
:10BDC00003689B6B18470000F7B500F54053054624
:10BDD000D3F8B00703681B69984707462846FFF762
:10BDE000EBFF05F5C0440646D4F8C400002862D134
:10BDF0003EB1D4F80431C4F8D0303E4BC4F8D4304E
:10BE00000120C4F8BC701DF083FED4F8C43094F94E
:10BE1000C82000FB0230C4F8C4003EB300230193E5
:10BE200094F82831002B4AD005F5A04393F8D43F6D
:10BE3000022B44D105F5AE40012201A93C3045F06A
:10BE400059F800283BD0D4ED4B7ADFED2B6AB8EEE1
:10BE5000E77ADDED017AE7EE667AB1EE047AF0EE8C
:10BE6000E77AF4EEC77AF1EE10FA33D494F8C930D9
:10BE7000002B3DD1D4F8C430D4F8D420002BB8BF67
:10BE80005B42934234DBD4F80411D4F8D030C4F8C8
:10BE9000D010CB1A03F2F31340F2E630834202F5DE
:10BEA000D2328CBF0023012302F5F07284F8CA302D
:10BEB000C4F8D4201CE0D4F8BC30F81AA1E7D4F8B8
:10BEC0002021D4F804319B1A03F2F31340F2E63236
:10BED0009342CBD8012384F8C930002384F8CA30B8
:10BEE000D4F8C43003F5D23303F5F073C4F8D4307A
:10BEF00003B0F0BDE0A501000AD7233CF7B500F57B
:10BF00008047044697F8A53FCBB300F5C043D3F86C
:10BF1000182112B9D3F81C318BB32046FAF7C6FFAB
:10BF200004F5C24006461036314601900CF036FA50
:10BF300004F5A04505F2945304F5C1413246703131
:10BF4000019883ED000A0CF05FF905F5B365DFEDAC
:10BF50000D0A85ED000AB7EE001A76201DF010FEDE
:10BF600004F5395383ED7F0A2046FFF72DFFD7F8FC
:10BF70007C0F0368DB6A03B0BDE8F040184703B0EC
:10BF8000F0BD00BF00000000012938B5044600F5EF
:10BF9000C04512D800F5005395F81021B3F9463585
:10BFA00083EAE371A1EBE37189B2012998BF3C21D7
:10BFB000920731D5FF2385F8C83007EE901AF8EEC6
:10BFC000677A2046C5ED377AFFF7BAFDD5F8CC3051
:10BFD00043BB2046FFF7F0FE50B904F5AB4393EDA9
:10BFE000067AF7EE007AB4EEE77AF1EE10FA19DD90
:10BFF00079F076FE04F58043C5F8CC00D3F87C0FC9
:10C0000003681B6A984768B104F556500021BDE8E3
:10C01000384008304FF01EB9002BB4BF4FF0FF334B
:10C020000123C8E738BD000010B500F5AE441C344C
:10C0300020465CF00DFE2046BDE810405CF078BE66
:10C0400010B500F5A043044693F830379A0717D48B
:10C050005B0700F556504FF002014CBF094A0A4AEF
:10C0600008304AF007FF04F5AE401C305CF0C4FD18
:10C0700004F535500121BDE81040343063F06AB951
:10C0800010BD00BF24770C083E770C0870B500F592
:10C09000A046054696F91C479CB196F83037C3F385
:10C0A00080045B0729D4B6F92237002B0BDC284625
:10C0B000FFF7C6FF05F535500121343063F04AF92A
:10C0C0000124204670BD2146F9F7D6FFB6F9223784
:10C0D00007EE903AF8EEE77AB4EEE70AF1EE10FADE
:10C0E000E5D5D6F89C35002BE1D005F55650044A2D
:10C0F000042108304AF0BEFEE3E70024E1E700BF78
:10C1000054770C0808B52DED028B08EE901A30B369
:10C11000F2B1B0F9083008EE103AB8EEC88AF8EE7D
:10C12000E88A9FED100ADFED100A28EE800ADFEDA5
:10C130000F8A4FF4D470B7EE001A1DF021FDC8EE3F
:10C14000280A1DF079FC20EE280ABDEC028B08BD00
:10C1500053F040FB07EE900AB8EEE78ADFE79FED69
:10C16000020AF2E70AD7233C0000000000A08C4539
:10C1700037B500F50054054694F9A735002B52D089
:10C1800053F042FA53F036FAC4F8C40D53F03CFAB7
:10C1900053F01CFAC4F8C80D53F036FA53F020FAE5
:10C1A000C4F8CC0D53F030FA53F024FA41F2941154
:10C1B000C4F8D00DD4F8C40D53F070FAD4F8C80DFB
:10C1C00041F2941153F06AFAD4F8D00D41F294116F
:10C1D00053F064FA284600F029FC48BBD4F8CC0D93
:10C1E000642153F057FA53F00FFAD02154F0B4FA07
:10C1F000C4F8D40D53F008FAD22154F0ADFAC4F8C3
:10C20000D80D05F525500C304921019055F032F834
:10C2100001984A2155F02EF80198462103B0BDE857
:10C22000304055F027B853F0EFF953F0C5F9ABE7BC
:10C2300005F5C043D4F8CC0D93F8B432642173B142
:10C2400053F028FA6421462054F00CFF6421492061
:10C2500054F008FF64214A2054F004FFC3E753F070
:10C260001DFAEFE710B500F500541E21D4F8C40DF7
:10C2700053F018FAD4F8C80D1E2153F013FAD4F86D
:10C28000D00D1E2153F00EFAD4F8CC0D1E21BDE8BE
:10C29000104053F007BA000007B500F0C7FB014695
:10C2A00058B90190462054F0FFFD0199492054F0FF
:10C2B000FBFD01994A2054F0F7FD0021042055F0C0
:10C2C000C5F80021132055F0C1F80021462055F093
:10C2D000BDF80021492055F0B9F800214A2055F059
:10C2E000B5F80021152003B05DF804EB55F0AEB8A9
:10C2F00010B5044655F0F0FA54F040FF204601F026
:10C30000DDFCBDE8104055F0EFB9000038B500F590
:10C310000055044695F9A7350BB1002038BD012121
:10C32000F6F738F990B104F58043D3F87C2F04F583
:10C330009E434C339A4209D004F59D432C339A42D4
:10C3400004D004F59D433C339A42E6D12046F6F7EB
:10C3500005FB0028E1D0D5F8D03DB3F90800DDE7B2
:10C3600038B52DED028B00F5804393F8903F002BFC
:10C3700040F0B9805D4A00F59E43D2F87C2F4C33E3
:10C3800000F556549A4204F1080408D0584A032193
:10C39000BDEC028B2046BDE838404AF06BBD00F58D
:10C3A00000559FED546AD5F8C42DB2F90830002B22
:10C3B000B8BF5B429BB207EE903A138B06EE903A01
:10C3C000F8EEE66AF8EEE77A66EE866AF4EEE67A6A
:10C3D000F1EE10FA17DCD5F8C82DB2F90830002BB1
:10C3E000B8BF5B429BB207EE903A138B07EE103A50
:10C3F000B8EEC77AF8EEE77A27EE067AF4EEC77A57
:10C40000F1EE10FA01DD3C4AC1E700F5C0501430EE
:10C4100020F038FADFED397A20EE270AF3EE0E7AB3
:10C42000B4EEE70AF1EE10FA01DD354AAFE7042079
:10C4300054F0C4FF132054F0C1FF152054F0BEFF88
:10C440004D2054F0BBFF4E2054F0B8FF4F2054F065
:10C45000B5FF502054F0B2FF152054F0DFFC9FEDE3
:10C46000298AB0EEC00AB4EEC80AF1EE10FA0BD574
:10C47000102054F0A3FF562054F0A0FF112054F0D8
:10C480009DFF572054F09AFF032054F0D7FCB0EEE4
:10C49000C00AB4EEC80AF1EE10FA0FD5022054F02B
:10C4A000CDFCB0EEC00AB4EEC80AF1EE10FA05D524
:10C4B000182054F083FF192054F080FFD5F8C40DE4
:10C4C000811D0C303FF0BCFAD5F8C80D811D0C3031
:10C4D0003FF0B6FAD5F8D00D811D0C303FF0B0FA20
:10C4E000094A052154E7BDEC028B38BD986C002049
:10C4F00068770C08CDCC4C3E88770C08E02E65425E
:10C50000B0770C0800000034CC770C0810B500F5AB
:10C51000005494F97E359BB1D4F8CC0D53F0D0F88B
:10C52000D4F8CC2DB4F9803530B1B2F90600984278
:10C53000ACBF0020012010BDB2F906008342F7E72E
:10C540000120F8E710B50446FFF7E0FF60B104F5FD
:10C55000804479F0C5FBD4F89C3FC01AB0F57A7FCF
:10C5600094BF0020012010BD0120FCE770B50546F6
:10C57000FFF7E8FF05F5005408B3D4F8C43D9A89E5
:10C58000DA80D4F8C83D9A89DA80D4F8D03D9A8907
:10C59000DA80D4F8C43D00261E81D4F8C83D1E813F
:10C5A000D4F8D03D1E8105F58043D3F87C0FC3F845
:10C5B000B46F03685B689847D4F8CC3D1E8105F5DD
:10C5C000C4400C3071F02CFC80B3002653F01CF8F2
:10C5D000437A13B953F018F8837A94F97E25012A27
:10C5E00023D106B10BB32846FFF7ACFF05F5804415
:10C5F00094F8963F38B30133DBB20A2B84F8963FA8
:10C600000CD105F556501F4B1F4A042108304AF043
:10C6100031FC1E4A012384F8903F937294F8963FB0
:10C620000A2B02D90A2384F8963F70BD2846FCF7EE
:10C63000EDFD0028C9D152F0E7FF52F0A9FF061E18
:10C6400018BF0126C2E7002BEFD0013BDBB2032B62
:10C6500088BF032384F8963F94F8963F012B09D1B5
:10C6600005F556500A4B084ABDE8704004210830D1
:10C670004AF000BC002BD8D1044A84F8903F937252
:10C68000D3E700BF5FCE0D08DC770C080D900020CB
:10C69000BF790C0800F500500A4690F9AE1DD0F89D
:10C6A000C40DFFF72FBD000000F500500A4690F9B9
:10C6B000AF1DD0F8C80DFFF725BD000000F50050F4
:10C6C0000A4690F9B01DD0F8D00DFFF71BBD000051
:10C6D00010B54FF480610446F5F75CFF04F5005394
:10C6E00028B1BDE81040D3F8CC0D53F06FB9BDE8C8
:10C6F0001040D3F8CC0D53F073B900002DE9F04190
:10C7000000F500530546D3F8D03DB3F9088000F595
:10C71000C044B8F1000F02D1012384F8503205F56E
:10C72000C4470C37384671F07BFB0646F8B9B8F5BC
:10C730007A6F2EDD79F0D4FAD4F84C32804693B17A
:10C74000C31A40F6B73293420FD905F5A04501222E
:10C7500031463846F5F700F9C4F84C6284F8506267
:10C76000C5F8448501E0C4F84C02BDE8F08118F535
:10C770007A6F0EDA79F0B4FAD4F84C326BB1C01A91
:10C7800040F6B7339842F0D9012200213846F5F738
:10C7900009F90023C4F84C32E7E7C4F84C02E4E797
:10C7A00070B52DED028B044652F02EFF52F0E6FDDF
:10C7B00030B9BDEC028B2046BDE87040FFF7D6BE15
:10C7C00004F5804595F8903F1BB979F089FAC5F8D2
:10C7D000A00F2046FFF79AFE18B179F081FAC5F84C
:10C7E0009C0F2046FFF7C2FE2046FCF79DFB04F598
:10C7F00000560023C5F8B43F96F982356BB3D6F8DE
:10C80000CC3DB3F90830322B27DD30B3323B1BB2BD
:10C8100007EE903AB8EEE78ADFED227A04F5A850E9
:10C8200028EE278A04F018F848B3B6F91E3507EE4B
:10C83000903A06F5A46696ED007AF8EEE77A77EE80
:10C84000C77A27EE888ADFED187A28EE278ABDEEB0
:10C85000C88A18EE103AA5F8B43F2046FFF74EFFFD
:10C86000D5F87C0F03685B689847BDEC028B0146E6
:10C8700004F5C4405830BDE8704055F021BC96F92D
:10C88000113596F913259B1A07EE903AF8EEE77AE0
:10C8900027EE888ABDEEC88A18EE103AA5F8B63F92
:10C8A000DBE700BF0AD7A33C0000C84270B500F523
:10C8B00000540546D4F884350BB9002041E094F9C2
:10C8C0001035002BF9DA00F58043D3F87C0F0368AC
:10C8D0005B6898470138172832D801A353F820F035
:10C8E000DDC9010819CA010841C901080FCA0108B8
:10C8F00005CA0108F1C90108E7C9010841C90108D1
:10C9000041C9010845C90108D3C90108C9C90108BD
:10C91000BBC80108FBC90108FBC9010841C90108DE
:10C9200041C9010841C9010841C9010841C90108BB
:10C9300041C9010841C9010841C9010823CA0108C8
:10C94000012070BD05F5A045B5F86266162EB4D07D
:10C95000D4F8841511F0020301F0010205D0A6F10C
:10C96000150CDCF1000343EB0C0311F0040043EA67
:10C97000020303D0A6F11F046042604143EA0002B3
:10C9800011F0080007D01F2E1AD0A6F111000228BE
:10C990008CBF0020012011F0100340EA020005D0F6
:10C9A000102E0FD0A6F1520253425341034311F40B
:10C9B000006014BF95F82C16014643EA0100C0E759
:10C9C0000120E8E70123F1E7D4F88405C0F3401023
:10C9D000B7E7D4F88405C0F38010B2E7D4F8840533
:10C9E000C0F3C010ADE7D4F88405C0F30020A8E779
:10C9F000D4F88405C0F34020A3E7D4F88405C0F33D
:10CA000080209EE7D4F88405C0F3003099E7D4F87D
:10CA10008405C0F3403094E7D4F88405C0F3803037
:10CA20008FE7D4F88405C0F3C0308AE700F50050E2
:10CA300090F81005C009704738B504460D4652F00D
:10CA4000E3FD0368DB689847C8B104F50053D3F8E9
:10CA5000CC0D6DB152F0BEFE07EE900AB8EEE70ABB
:10CA600004F5C04494F8B3320BB1B1EE400A38BDBE
:10CA7000B0F9083000EE103AB8EEC00AF0E79FEDCA
:10CA8000010AF4E70000000038B52DED028B0446E2
:10CA90000D4652F0B9FD0368DB68984700283FD087
:10CAA000214BD3F8CC3D5B69012B07D0BDEC028B49
:10CAB00029462046BDE83840FFF7BEBF4FF48061ED
:10CAC0002046F5F767FD0028F0D004F50053DFEDB0
:10CAD000177AD3F8CC0D93F91335028B08EE903A00
:10CAE00000EE102AF8EEE88AB8EEC08A68EEA78A4F
:10CAF00052F07AFEB6EE001AA0EE011A04F5C04418
:10CB0000DFED0B0AB0EE680A1DF068F894F8B33256
:10CB100028EE000A0BB1B1EE400ABDEC028B38BD25
:10CB20009FED030AF9E700BF984C00200AD7233C89
:10CB30000000000073B500F5A046044696F8D43F07
:10CB4000022B00F5736512D100F5AE40012201A958
:10CB50003C3044F0CFF950B1019BC5F89C322846D7
:10CB60003FF06EFB2046F9F7F7FF02B070BDD6F834
:10CB70000036042B05D12046F9F7D0FC8DED010AD3
:10CB8000EAE704F5C043D3F83C310193E4E7000041
:10CB900070B500F580460446D6F87C0F03689B6BA1
:10CBA0000D46984748B9D4ED460A9FED1D0A642109
:10CBB0002846BDE8704054F013BAD6F87C0F04F54F
:10CBC0009E4104F500521031884292F8123592F9D4
:10CBD000DC2521D104F5A04090F8AC1551B94AB13B
:10CBE000D3B204F5A041D1F800160139012998BF4C
:10CBF000D3B209E004F5C04191F9541061B1D0F805
:10CC00000006042808D1CBB207EE903AD4ED460ACC
:10CC1000B8EE670A6421CBE7002AF5D0E1E700BF50
:10CC2000000000002DE9F04100F58048044604F5BD
:10CC30009E43D8F87C0F4C33984203D100252846F8
:10CC4000BDE8F08103689B6B984750B104F5A043A1
:10CC500093F8305715F0010503D0012283F8F82529
:10CC6000EDE704F5BF40583076F0CCFF054608B13B
:10CC70000125E4E704F5A04696F8F835002BDDD051
:10CC8000D8F87C0F03689B6B984718B9002386F887
:10CC9000F835D4E794F8143494F85874B02202FBB1
:10CCA000034393F8F121BFBB012A0AD993ED837A9C
:10CCB000F1EE047AB4EEE77AF1EE10FAACBF012798
:10CCC0000027D8F87C2F04F59E4310339A4202D1F6
:10CCD00096F8AC3523B104F59E4354339A4241D1C2
:10CCE00004F50053204693F9D085FCF78FFAA8B9D4
:10CCF000204601F027FC0028BAD0002386F8F8353A
:10CD000094F8712404F58C63242101FB023306F2AC
:10CD1000A456DB6A336092E72F46D2E778F0E0FF53
:10CD2000D6F80C364FF4FA62C01A642313FB0823BA
:10CD300041F28832934238BF13469842D8D92046F0
:10CD4000F9F770FBB0F5FA7FD2DD04F5805341F2BC
:10CD50006E72D3F8FC3603F6B7339342C8D8002F6F
:10CD6000C6D093E704F5C043D3ED4F7AB2EE047A10
:10CD7000F0EEE77AF4EEC77AF1EE10FA86DA002FD9
:10CD80003FF476AF04F5A85003F066FD00283FF4A9
:10CD90007DAF04F5005304F5085093F84E1302F0EC
:10CDA00071FFF1EE047AB4EEE70AF1EE10FAFFF645
:10CDB0005FAF6BE7F8B52DED048B044608461746C8
:10CDC0001D46BDF9286054F029F804F50054384692
:10CDD000B0EE408A54F022F8B4F9AC25002AF0EE07
:10CDE000408A39DAC2F1640307EE903A9FED217A66
:10CDF000F8EEE77A67EE877A60EE278A04F5B56485
:10CE0000D4ED007A9FED1C1ADFED1C0A38EEC80A3B
:10CE1000BC2020EE270A1CF0B3FE38EE288AB0EEC4
:10CE2000409A94ED000A9FED141ADFED140A28EEE3
:10CE3000000ABD201CF0A4FE2846B0EE408AB0EEE9
:10CE4000490A53F0D7FFB0EE480ABDEC048B3046D8
:10CE5000BDE8F84053F0CEBFD0D002F1640307EE36
:10CE6000903A9FED047AF8EEE77A67EE877A28EE3B
:10CE7000278AC3E70AD7233C00A08C4500A08CC5B5
:10CE800000B52DED048B042083B053F0C7FF0320C1
:10CE9000B0EE408A53F0D2FFDFED189A9FED181ADA
:10CEA000DFED180A8DED011AF0EE408AB0EE480A67
:10CEB000A8EEA90ACF20CDED000A1CF061FEB0EE6D
:10CEC000409AB0EE480A9DED011ADDED000AA8EE89
:10CED000E90AD0201CF054FE1820B0EE408AB0EED3
:10CEE000490A53F087FFB0EE480A192003B0BDECA1
:10CEF000048B5DF804EB53F07DBF00BF00003442AB
:10CF000000A08C4500A08CC5F8B52DED088B00F570
:10CF1000005600F5C04596F9963D13F0040F03F056
:10CF2000010203F0020440F0F580D5F8B8727B1ED0
:10CF30005F425F41002A00F0EF804D2053F06EFF0A
:10CF40004E20F0EE409A53F069FFB0EE408AB6F9F9
:10CF5000AE35DFED87AA0AEE103A1520B8EECAAA60
:10CF600053F05CFF2AEE2AAA20EE0AAA002C00F059
:10CF7000DB80F0EE488AB0EE699AB5EEC0AAF1EE19
:10CF800010FA40F3D6809FED7B1ADFED7B0A38EE76
:10CF90000A0A4FF480701CF0F3FD9FED761ADFED66
:10CFA000760AB0EE408A40F2011038EECA0A1CF050
:10CFB000E7FDF0EE408A96F9973D632B15DC07EE0E
:10CFC000903A9FED6E7AF8EEE77AB4EEC79A67EE84
:10CFD000AA7AF1EE10FAF4EEC78A98BF29EE279AE2
:10CFE000F1EE10FA98BF68EEA78AD5F8B83296F934
:10CFF000944D96F9956D022B00F0B48024B2002C6C
:10D0000001DC002E6EDD032053F018FFDFED5C7AAB
:10D01000B4EEE70AF1EE10FAB0EE40AA62DB002FA0
:10D0200000F0A2809FED571ADFED570A40F227105B
:10D0300030EE000A1CF0A4FD9FED541ADFED520AF9
:10D04000B0EE40BA4FF494703AEE410A1CF098FDED
:10D0500070EE007AB0EE4BAA07EE104AF8EEC7AABF
:10D060009FED4BBA9FED431ADFED430A6AEEA7AA84
:10D07000B0EE690A40F22B10AAEE8B0A1CF080FD7C
:10D0800007EE906AF0EE409AB8EEE70A9FED391A83
:10D09000DFED390A2AEE40AAB0EE490A4FF4967045
:10D0A000AAEE0B0A1CF06CFDB0EE409AB0EE480AF6
:10D0B0009FED301ADFED300A40F22D10AAEE8B0AF8
:10D0C0001CF05EFDB0EE408AB0EE680AAAEE0B0AD4
:10D0D0004FF497709FED271ADFED270A1CF050FDE3
:10D0E000F0EE408AB0EE690A102053F083FEB0EEF5
:10D0F000490A562053F07EFEB0EE480A112053F044
:10D1000079FEB0EE680ABDEC088B5720BDE8F84008
:10D1100053F070BE01270DE7042053F07FFEB0EE00
:10D12000408AF1EE409A12E7DFED178AB0EE689A76
:10D1300023E79FED101ADFED100A39EECA0A4FF40B
:10D1400082701CF01DFD9FED0B1ADFED0B0AF0EE57
:10D15000409A40F2051039EE0A0A1CF011FDB0EEBB
:10D16000409A28E700244CE7F0EE407A74E700BFCD
:10D170000AD7233C00A08C4500A08CC5000000B459
:10D18000000000340000C8420000000000004842D7
:10D190006666E63E38B52DED028B00F50055044677
:10D1A000D5F8D80DA0B304F5804393F8902F7ABB3F
:10D1B00093F8963F63BB52F0D3FB07EE900AB8EEAC
:10D1C000678A462095F9105553F028FE002DF0EEA1
:10D1D000408A20DA04F5BF40583076F095FBE8B974
:10D1E0009FED101ADFED100A40F25110B1EE680AFF
:10D1F0001CF0C6FCB4EE408AF1EE10FAC8BFB0EEE7
:10D20000480ABDEC028B6E20BDE8384053F0F2BDF9
:10D210009FED058AD5E79FED040AEBE79FED010A34
:10D22000E8E700BF0000C8420000000010B52DED87
:10D23000028B4369002B4AD0037C0BB1013303748A
:10D24000037C002B41D0182B1FD803EB4303C3EB07
:10D2500003139B001CB2002307EE903AB8EEE78A56
:10D260000420B0EE480A53F0C5FD07EE904A1320A3
:10D27000B8EEE70A53F0BEFDB0EE480ABDEC028BF3
:10D280001520BDE8104053F0B5BD4A2B02D8C3F1BC
:10D290003203DAE7632B01D8643BD6E77C2B08D84E
:10D2A000643B03EB4303C3EB03139B001BB200245B
:10D2B000D2E7AE2B02D8C3F19603F2E7C72B01D811
:10D2C000C83BEEE700230374F1E71C46C4E7BDEC5E
:10D2D000028B10BD10B59FED1C7AD0ED017AF4EEF3
:10D2E000C77A0023F1EE10FA044643722BDB90ED6F
:10D2F000007AB4EEE77AF1EE10FA24D908F030F9AA
:10D30000217A07F081FDD4ED010AF5EE007A60EE96
:10D31000A77AB4EEE70AF1EE10FA14D494ED001AED
:10D3200040F2A5101CF02CFCF7EE007AB4EEE70AF0
:10D33000F1EE10FA07D494ED007AC7EE007A0123DB
:10D340006372C4ED037A10BD00000034437A7BB3EE
:10D3500091F9003090ED037A07EE903AF8EEE77A13
:10D3600067EE877A9FED137AF4EEC77AF1EE10FA42
:10D37000D8BFF0EE477AFDEEE77A17EE903A0B70E1
:10D3800092F9003090ED037A07EE903AF8EEE77AE2
:10D3900067EE877A9FED087AF4EEC77AF1EE10FA1D
:10D3A00058BFF0EE477AFDEEE77A17EE903A137029
:10D3B000704700BF0000C8C20000C842437AF0EEC8
:10D3C000407A5BB190ED030A9FED051ADFED050A87
:10D3D00027EE800A4FF4E6701CF0D2BB704700BF06
:10D3E0000000C8420000C8C2F8B504460E46174601
:10D3F00078F076FC054604F59F40483007F08EFE35
:10D4000004F5A044D8B3462053F008FDDFED3D7A83
:10D41000B4EEE70AF1EE10FA10DB97F9002094F968
:10D42000F935193A934209DAD4F8FC25AA4205D015
:10D43000C4F8FC55013384F8F93544E0462053F034
:10D44000EDFCDFED317AB4EEE70AF1EE10FA3AD8EE
:10D4500096F90020002A36DAC2F1FF2294F9FA3553
:10D4600002F57F02E73293422DDAD4F8FC25AA4276
:10D4700029D0C4F8FC55013384F8FA3523E0D4F8F8
:10D48000FC35EB1AB3F57A7F1DD3462053F0C6FC6A
:10D4900094F9F93507EE903AF8EEE77AB4EEE70A38
:10D4A000F1EE10FA01DD002B22DC462053F0B6FC31
:10D4B00094F9FA3507EE903AF8EEE77AB4EEE70A17
:10D4C000F1EE10FA18D497F9000094F9F92500212B
:10D4D000821A1CF005FC387096F90000002806DA64
:10D4E00094F9FA15002201441CF0FAFB3070F8BDE3
:10D4F000C4F8FC55013B9EE7002BE4DDC4F8FC5565
:10D50000013BB9E700000034000000B410B52DED78
:10D51000028B00F5005282B092F9103592F8112575
:10D520008DF80630002B0446B0EE408A8DF80720B7
:10D5300004DAFFF7BBF908B98DF8060004F5A0433B
:10D54000D3F80026012A4CD0072A4AD004F5BF4060
:10D55000583076F0D9F9002858D104F536500DF13D
:10D5600006010DF107021830FFF7F0FE2046FFF725
:10D570003BFF9DF906309DF90720DFED258A934298
:10D58000A8BF134607EE903A04F53954B8EEE70AFF
:10D59000383420EE280A20468DF8063075F0ACFBB2
:10D5A0009DF9073000EE103AB8EEC00A204620EE92
:10D5B000280A75F0ABFB9DF9073001EE103A9DF992
:10D5C000063000EE903AB8EEC11AF8EEE00A40F2EA
:10D5D0004D20B0EE480A1CF0D3FA02B0BDEC028B2D
:10D5E00010BD03F25C52D2ED007AFDEEE77A03F54E
:10D5F000AC6317EE902AD3ED007A8DF80720FDEE8C
:10D60000E77A17EE903A8DF80630A6E70023FAE79E
:10D610000AD7233C70B5044600F53655183504F595
:10D6200080462846FFF756FED6F87C0F03685B6DF0
:10D63000984740B1462053F0F1FB2846FFF7BEFE65
:10D64000462053F0D7FBD6F87C0F03681B6D984734
:10D6500040B1462053F0E2FB2046FFF757FF46203B
:10D6600053F0C8FB2046FFF7DDFA10B304F5005570
:10D6700095F97C3543B101212046FFF7DDF9BDE87E
:10D680007040462053F0B6BB04F5BF4458342046E2
:10D6900076F03AF950B1204676F0BEFA30B195F9FD
:10D6A000103500EE103AB8EEC00AE8E79FED010A27
:10D6B000E5E770BD0000000010B504462DED028BBB
:10D6C000462053F0ABFB2046B0EE408AFBF79EFDB0
:10D6D00080BB04F5C4400C3070F0A2FB50B304F5DD
:10D6E000A853D3ED968A1BF0CFFC90F8EC349FED55
:10D6F000137A0C2202FB0300D0ED807AE8EEC77AA1
:10D70000F4EEC77AF1EE10FA0CDC04F5005494F94B
:10D71000133507EE903AF8EEE77AF4EEC87AF1EEB8
:10D7200010FA07D5BDEC028B0548BDE81040012179
:10D7300004F018BDBDEC028B10BD00BF0AE81C410F
:10D74000984100202DE9F04100F500550646D5F836
:10D75000D43D9BBB002706F58048D8F87C0F0368B2
:10D760009B6B98470446002851D006F5A85003F05B
:10D7700073F880B308F6A873D3ED007A9FED407A72
:10D78000F8EEE77A67EE877AFDEEE77A17EE903AE1
:10D790001BB295F9C3250AB19A421FDA95F9C14522
:10D7A000FCB906F5A043D3F80036013B062B2ED872
:10D7B000DFE803F01E2D24602D2D1E0051F024FF04
:10D7C0000368DB6898470028C4D0D5F8D40D52F020
:10D7D000C7F847B2BFE795F91335DAE795F9C245BF
:10D7E000DFE724B29C42ACBF95F9C0450024D8E7DE
:10D7F00095F9C435002B18BF1C4608E095F9C435CF
:10D800002BB13046FBF722FD08B195F9C44587EAF4
:10D81000E773A3EBE773DBB2A342C8BF3C4607EE56
:10D82000904A0320B8EEE70A53F0E4FA07EE907A44
:10D830000220B8EEE70A53F0DDFA95F9F535D6ED9A
:10D84000460A00EE103A6421B8EEC00A032053F0F5
:10D85000C7FB95F9F535D6ED460A00EE103A0220E1
:10D86000B8EEC00A642153F0BBFB3046BDE8F0417E
:10D87000FFF706BB06F5C04393F95330BAE700BF84
:10D880000AD7233C38B504462DED048B462053F0CF
:10D89000C5FA584BDFED587A93F9613D08EE903A9E
:10D8A000F8EEE88A152068EEA78AB0EE408A53F0B9
:10D8B000B5FA9FED527A20EE280A04F5C045C0EE75
:10D8C000077A28466430C5EDAA7A73F079F810B16A
:10D8D0000023C5F8A832B5EEC08AF1EE10FA43D5A0
:10D8E0002046FFF7A3F800287ED02046FEF7DEFF93
:10D8F000002879D0D5EDAA7A9FED419A9FED411A83
:10D90000DFED410AB0EE480AA7EE890A4FF43B70FA
:10D910001CF036F9D5EDAA7A9FED3A1ADFED3A0AF6
:10D92000F0EE408A40F2ED20B0EE480AA7EEC90AB8
:10D930001CF026F9B0EE408A04F5C4450C352846A3
:10D9400070F078FAD0BB284671F088FB022827D106
:10D950000321492053F0A8FDBDEC048B0321BDE851
:10D9600038404A2053F0A0BD3ED9D5EDAA7A9FEDAC
:10D97000249A9FED261ADFED230AB0EE480AA7EE9F
:10D98000890A40F2F2201CF0FBF8D5EDAA7A9FED4F
:10D990001F1ADFED1C0AF0EE408A40F2F320C3E7C5
:10D9A0009FED180A492053F025FABDEC048B9FED3A
:10D9B000150ABDE838404A2053F01CBAB0EE680A98
:10D9C000492053F017FAB0EE480A4A2053F012FAF1
:10D9D00020464921FFF7DCF8BDEC048B20464A21A4
:10D9E000BDE83840FFF7D4B89FED068AF0EE488ACC
:10D9F000A2E700BF984C00200AD7233C00A08C452A
:10DA000000004842000000000000C8C20000C842F8
:10DA1000F8B52DED028B00F5C046044696F951305D
:10DA2000002B32DD00F5804200F59E43D2F87C2FBA
:10DA300010339A4229D196F95030002B25DD00F59C
:10DA4000BF40583075F0D2FFF8B104F5C4400C3037
:10DA500070F0E6F9C8B9124F9FED128A04463D688E
:10DA60002D190ED0B5F9080052F0EAFF48B196F929
:10DA70005130012B0CD1B5F90800B0EE480A53F033
:10DA8000B9F91434B4F5A07FE9D1BDEC028BF8BD2F
:10DA9000022BF6D1B5F90800032153F005FDF0E79C
:10DAA000A89400200000000037B500F5A04304460C
:10DAB00093F858350BB39FED120A15204F2553F0FC
:10DAC00099F920460095502313221521FFF772F98A
:10DAD000152053F031FC80B9284653F02DFC60B975
:10DAE0009FED070A4E2053F085F99FED050A4D2062
:10DAF00003B0BDE8304053F07DB903B030BD00BF86
:10DB00000000000070470000F8B52DED048B00F513
:10DB100080440546D4F87C0F03689B6B984738B95E
:10DB2000D4F87C2F05F59D4364339A4240F0C080C1
:10DB300005F5C4400C3070F07DF9002800F0B88085
:10DB40002846FBF763FB002800F0B28005F5A044EF
:10DB5000D4F81436002BB8BF5B42B3F52F7F00F327
:10DB6000A780D4F81836002BB8BF5B42B3F52F7FDF
:10DB700000F39E8005F5C04778F0B2F8D7F8783109
:10DB8000C31AB3F5FA7F0646C0F0928005F5C85374
:10DB900093ED017AF2EE007AB4EEE77AF1EE10FA44
:10DBA00000F1868004F5C46494ED007AB4EEE77A5F
:10DBB000F1EE10FA7CD405F5405393ED8D8AD3ED48
:10DBC000E48A05F525540C34B0EE480A04212046B9
:10DBD00053F086F9B0EE680A1321204653F080F91D
:10DBE00078EEC89A4D21B0EE690A204653F078F9D4
:10DBF00038EE289A4E21B0EE490A204653F070F9CB
:10DC0000B0EE680A4F21204653F06AF9B0EE680A78
:10DC10005021204653F064F905F50055B0EE480A4E
:10DC20001821204653F05CF9B0EE480A192120462D
:10DC300053F056F995F9963D03F00202DB075CBFFD
:10DC4000F1EE489AB0EE489A6AB3B0EE498AF0EE27
:10DC5000698AB0EE690A1021204653F041F9B0EE0E
:10DC6000680A5621204653F03BF9B0EE490A1121CB
:10DC7000204653F035F9B0EE480A5721204653F0BC
:10DC80002FF9D7F87C31C7F87861F31A42F2107295
:10DC900093420DD9C7F87C61BDEC048B2046BDE8EA
:10DCA000F84053F003BD9FED048AF0EE488AD0E7B8
:10DCB000BDEC048BF8BD00BF0000000073B5044646
:10DCC00053F00AFE054653F09DFD2046FFF7DAFDAE
:10DCD0004E23009313224D2304212046FFF76AF8B8
:10DCE0004F2315211322009320465023FFF762F89B
:10DCF0002046FFF709F92046FFF78AFE4FF400514E
:10DD00002046F4F747FC10B12046FFF7CDFE04F59E
:10DD10000056D6F8640D50B104F5804204F59E43D8
:10DD2000D2F87C2F4C339A4201D153F03DF853F096
:10DD3000FFFC52F053FF284653F06CFD96F9383D36
:10DD40002BB1204602B0BDE87040FFF7DDBE02B047
:10DD500070BD000037B5044604F5C04553F0BCFD66
:10DD6000643553F04FFD284672F02AFE002868D132
:10DD700004F5A043D3F80036042B04D104F5BF40CA
:10DD8000583075F0EDFD2046FFF744FC04F5804265
:10DD900004F59E43D2F87C2F4C3304F5C4459A42D7
:10DDA00005F10C0523D0284670F044F8F8B99FED32
:10DDB000320A462053F01EF89FED2F0A492053F0F7
:10DDC00019F89FED2D0A4A2053F014F8284671F0F7
:10DDD00045F902280BD10321462053F065FB0321AE
:10DDE000492053F061FB03214A2053F05DFB20469C
:10DDF000FFF762FC2046FFF7A5FC2046FFF7CAF9B3
:10DE000020464621FEF7C4FE284670F009F890B976
:10DE10000190284671F022F968B102281CD10199BD
:10DE2000462053F0ADFA0199492053F0A9FA01991F
:10DE30004A2053F0A5FA204603B0BDE83040FFF772
:10DE40003DBF2846F8F748F804F5C04393F96E3013
:10DE50002B2B8DD003B030BD9FED070A462052F02A
:10DE6000C9FF9FED050A492052F0C4FF9FED020A49
:10DE70004A2052F0BFFFDEE700000000F6F732BE96
:10DE80000148FAF771BF00BF982C002008B5044A7A
:10DE90000F2343F0F9FE80F00100C0B208BD00BFBF
:10DEA000EC780C08F8B500F540570446D7F8406701
:10DEB00077F016FF04F58042B2F9945FAB1E9BB277
:10DEC000012B04F500537CD904F5A041D1F80016CC
:10DED000042976D0012D92F8905FD2F89C1F08BFDC
:10DEE000D2F8981FC5B1411A07EE901A03F5B26136
:10DEF00091ED007ADFED476AF8EE677A27EE267A31
:10DF0000F4EEC77AF1EE10FA06DD03220221204674
:10DF1000BDE8F840FAF7DCBD93F9941503291DD14B
:10DF2000D2F87C2F04F59E4110318A4270D1002E28
:10DF30006ED0801B07EE900A03F5B263B8EE677AE5
:10DF4000DFED346AD3ED007A67EEA67AB4EEE77AB5
:10DF5000F1EE10FA5CDD05220321D8E7012955D046
:10DF6000022955D19EB1821B07EE102A03F5B26239
:10DF7000D2ED007ADFED276AB8EE477A67EEA67A2F
:10DF8000B4EEE77AF1EE10FAE5DC022940D197F819
:10DF90002426002A3CD0D7F82826CAB31E4A126885
:10DFA000B2B3801A03F5B26307EE900A93ED007ADC
:10DFB000DFED186AF8EE677A27EE267AF4EEC77A74
:10DFC000C6E703F5B261D1ED007A93F9881503290C
:10DFD0001CBF03F28C53D3ED007A032D0FD1FCEE5E
:10DFE000E77A4FF47A7317EE902A801B5A439042D7
:10DFF0000ED205212046BDE8F840FAF725BE022DD5
:10E0000006D192F8903F1BB90321F3E7002EAAD165
:10E01000F8BD00BF00007A441C94002070B500F5E4
:10E020000056044696F98835032B00F580450FD03D
:10E03000B5F9943F63B900F5A043D3F80036042B3B
:10E0400017D095F8903FA3B103220121FAF7C0FC45
:10E05000B5F9943F012B0CD195F8903F1BB196F97F
:10E060008835032B05D120460321BDE87040FAF71F
:10E07000BDBD70BD70B500F6C806044630461AF046
:10E08000CFFF04F55653083358B3174A18460121F9
:10E0900004F5A85548F0EEFE284602F083FA04F590
:10E0A0008053032283F8142740F20112A3F80828B2
:10E0B000B4F9A4301BB9B4F8A230A4F8A430B4F871
:10E0C000A41030461BF086F8284602F06BFB802334
:10E0D000C4F8743404F58C600121BDE8704006F08A
:10E0E00061BA024AD2E700BFF4770C0821780C0825
:10E0F00038B50B6805465B6808460C469847074BE1
:10E10000D87023682046DB689847014605F5A5507E
:10E110000C30BDE8384039F0FFB800BF0D9000204A
:10E120002DE9F74F00F580470446D7F87C3F8B4236
:10E130000D4616460CD100F5005494F8D0349342A5
:10E1400040F0B5804FF00109484603B0BDE8F08FBC
:10E150000B6808465B69984704F5565808F10808AB
:10E160008146B0B143F044FF40F203124FF48011F6
:10E1700043F0F6FE524A0621404648F07BFE1A2E36
:10E180001FBF504A137843F0040313704FF0000987
:10E19000DAE74D4B1B68DB6A93F89C305BB304F500
:10E1A000005393F8B82332B3B3F8D423D20722D55F
:10E1B00093F8F433FBB12046FAF786FED8B1A6F106
:10E1C0002703DBB20A2B06D8012202FA03F340F23E
:10E1D000234213420FD12B6828469B6898473B4A3D
:10E1E00003460521404648F045FE364A137843F081
:10E1F00004031370A8E7022E2BD0D7F87CBFD7F802
:10E20000803FC7F87C5F04F50059C7F880BF04F56C
:10E21000C04A99F8D024009328469AF8C0328AF868
:10E22000C02289F8D0640193FBF7E4FB38BB284A8D
:10E230000421404648F01EFE009BC7F8803FC7F807
:10E240007CBF9AF8C03289F8D034019B8AF8C0327A
:10E2500095E72B6828465B68984701462046FFF7FC
:10E2600015FE81460028C8D12B6828469B68984730
:10E27000184A03460521404648F0FCFD64E758462D
:10E28000FBF7A4FBD7F87C0F03685B68984799F805
:10E29000D024014604F58F5044F084FED7F87C1F4B
:10E2A0002046FFF725FF0021404650F0D7FA1A2EEE
:10E2B0001FBF044A137843F00203137042E700BF04
:10E2C0003C780C082C900020942C002054780C08EA
:10E2D000C0780C0880780C0873B505460A4801928E
:10E2E0000E46FAF75DF9019A044630B10146284618
:10E2F00002B0BDE87040FFF713BF2846314643F037
:10E300000BFC204602B070BD982C0020FFF7E4BF44
:10E310004FF40023F7B50446C0F8B83D00F543506C
:10E320003C3071F0BDFD04F54950143071F034FB00
:10E3300051F06AF99922292152F050FA51F064F90A
:10E3400051F00AF904F5A35018305AF0F1F904F528
:10E35000A5500C3038F0C4FF04F580432046D3F8B4
:10E360007C1FFFF7C5FE2046FDF796FF04F58C6085
:10E3700006F060FB04F580534FF48042C3F8DC21C3
:10E38000192104F573603EF02DFA04F59F404830E2
:10E3900006F08AFC04F59850103054F0BFFB04F5E9
:10E3A000565504F538500835103054F039F82846E1
:10E3B0004CF0B4FF04F56250083061F017FD0AF02C
:10E3C00015FE4FF4806303630AF010FE0BF086FE27
:10E3D00004F51451103104F5085004F5005601F00D
:10E3E000E5F88023C6F850330423C4F8A43104F5BB
:10E3F000907011F09BFE2046FDF734FF04F5C340FA
:10E40000083055F07DF904F55E50343007F08CFF8C
:10E4100004F53550343060F0D9FF324B32491F6873
:10E42000B86A03684FF47A72DB6A984701203CF0BF
:10E43000A3F804F59E411A2244312046FFF770FEEE
:10E440002A4A0621284648F015FD2046FFF712FE0D
:10E4500004F5AC4024301FF0F7FE04F5A0434FF460
:10E460008072C3F81827224B0093224B019302AB12
:10E4700013E9060004F58F5044F0ACFB77F030FC54
:10E4800004F54055C5F840072046FDF731FFD6F8A2
:10E49000B41D29B1786A03680222D3F88030984706
